:020000040000fa
:08000000c07d040001000000b6
:020000040000fa
:100200005406040000000000820604000000000004
:10021000cfee2100807f2200000188000000000056
:10022000050007000c0007001a3c02000000000057
:100230000040da000000fe004440a900c0c02900d0
:100240000000e0000300320010002000a001880040
:100250004440a80000000600a0bc2d0001002000c2
:100260001600370062004000e080480091018800dd
:100270009001ba0062004000e080480091018800cf
:100280009002ba0062004000e08048000002eb00eb
:100290006028e10005003a008301e900070033000f
:1002a000038009000059eb00040037006128e100d9
:1002b000010032000082eb00050007009101880078
:1002c0001001ba000200e000e6ff3a00000005005d
:1002d000910188008002780062004000e0804800c0
:1002e0003559ba008301e900080032002559ba00e7
:1002f0008301e900050032000400e000f4ff320051
:1003000015d9ba008301e900f1ff3a0000000600a8
:100310001004b100070035009001b1000400340062
:100320007000b100030035009001b10001003c00f5
:100330001000050000000500ea874700889fbe0006
:100340008a9fbe008c9fbe008e1f780080067800ba
:10035000010678008204780000047800010037006c
:100360000804e8001800fb00980207000000e00005
:10037000fbff3a0098407800d0c2b30080cf500015
:100380000400320000c0e900d0ef9f0080cf500091
:1003900002003a00d1ef9f000804e8000900e000e5
:1003a00046003500e18f5400440032004002200036
:1003b000808f540041003c000900e0000d00340033
:1003c000f08f54001a003a0000c3b300984f100099
:1003d00017003a009840900080c7b30080cf5000cb
:1003e0001200320080c5b30080cf500010003a00e8
:1003f0000e00370000c3b300984f10000200320017
:10040000a90020000a0037009840900080c7b30080
:1004100080cf5000040032008900200080c5b30066
:1004200080cf500002003a00090120000884e80053
:10043000d8b79f0000c3b300984f100002003a00e5
:10044000d84f1000feff32006055b8000807780052
:100450000e003700fab79f008bbf9f00e0392100e4
:1004600000425200c4ef9f006149b9000a00be007b
:10047000ee1407004fea97000401fb00cf91de0065
:1004800000054100818549000804e8001800fb00d0
:10049000400107008000780009017800e039210060
:1004a00052020700000278000000e000e9ff3a0075
:1004b0005fb09700880f500005003a000c00e00084
:1004c000010032000d0e78006000b80027003700f0
:1004d0008e005400303c2100694078000000fb0091
:1004e00000805000170033004240a9000f003c007c
:1004f0004fe997000200fb00cf80de0000005500ae
:1005000081805d00800f5500818f5d0007003900fc
:100510006149b900f11007007fb197008fb99700ca
:10052000820f5000838f5800060032002002200006
:10053000f0ab88000085eb008085eb00b3c2b30010
:10054000d3ef9f00d0c2b3005fea9700804f520004
:1005500002003a0060051500e0851d000c00e00077
:1005600001003200080e78000a00be004f07780034
:100570004f06be004f05be004f04be00af00b100e5
:1005800000000600f8874700889fbe008a9fbe00d3
:100590008c9fbe008e1f7800c0b79f0001047800ba
:1005a0000206be0000057800788057001802070098
:1005b000680760000030a100e10f500043003a00de
:1005c000cfb0970024002000c3fd2f008f81410091
:1005d000080178000a0078008f0207008005780083
:1005e0000000e00007003a006000b8006011b800a9
:1005f000d0b79f00e1b79f00f2b79f0083bf9f0075
:100600002d0037006400b800c2fd2f000f0141002b
:10061000000041001000be0087100700d0b79f0007
:10062000e1b79f00f2b79f0083bf9f000b05e90071
:100630004240a900200034006450b800c2fd2f00e1
:100640000f014100000041001000be00e00f50000b
:10065000e08f5800150032000a8455006844b80045
:10066000e24e210002044400731007000002be00a5
:100670000203be003800be002801be00400f070084
:100680000002be000203be005fb09700efb097000b
:100690007fb197008fb99700080e0700d0b79f0071
:1006a000e1b79f00f2b79f0083bf9f000a05e900f2
:1006b0004240a900e0ff3c006fa89700ffa8970008
:1006c0000c0240008d82480045003700e20f5000c8
:1006d00049003a00cfb0970000027800c3fd2f0018
:1006e0008f814100080178000a007800300307007c
:1006f000800578000000e00007003a006000b800c4
:100700006011b800d0b79f00e1b79f00f2b79f001b
:1007100083bf9f002d0037006400b800c2fd2f008a
:100720000f014100000041001000be004210070010
:10073000d0b79f00e1b79f00f2b79f0083bf9f0033
:100740000b05e9004240a900200034006450b800c5
:10075000c2fd2f000f014100000041001000be004b
:10076000e00f5000e08f5800150032000a84550059
:100770006844b800e24f2100020444002e10070034
:100780000002be000203be003800be002801be0009
:10079000fb0e07000002be000203be005fb0970020
:1007a000efb097007fb197008fb99700c30d070096
:1007b000d0b79f00e1b79f00f2b79f0083bf9f00b3
:1007c0000a05e9004240a900e0ff3c006fa997003c
:1007d000ffa9970076805700ed0307000c02be00ca
:1007e0005fb09700efb097007fb197008fb9970087
:1007f0007704070013003700e30f500004003a00ad
:100800006000b8000200200003ff27000600370048
:10081000e40f500009003a00f0ff2f00f1ff2f0015
:10082000f2ff2f00f3ff2700d0b79f00e1b79f0032
:10083000f2b79f0083bf9f00060037006000b8003a
:100840006011b800d0b79f00e1b79f00f2b79f00da
:1008500083bf9f005fb09700efb097007fb1970014
:100860008fb997000e00e0000100320003f0a200f3
:100870004f0778004f06be004f05be004f04be0074
:100880008f01b10000000600800178000200e00046
:10089000070032001104e00005003200b159780071
:1008a0000201e900020032001104e000fbff3a00ff
:1008b0000200e000030032008059eb000201e90071
:1008c000fdff3a00000006001004e0000a003200bc
:1008d000010178001104e000050032009041780029
:1008e00092cf5100050032005204e000fbff3a00b5
:1008f0005004e000f6ff3a000000eb0000000600a4
:10090000800178000200e000030032008159780085
:100910000201e900fdff3a000000060080007800b7
:100920001004e000020032005104e000feff3a0033
:1009300000805000000006000400fa00889fbe00fe
:100940008a9fbe008c9fbe0080bf9f0091bf9f000a
:100950000206be00bb1307000001be000004be007b
:100960000c00be00b11307000fb997009fb99700a4
:1009700000055100818559000800be000a01be0033
:100980004f06be004f05be004f04be000080fa00b7
:1009900000000600800078001104b100030035005b
:1009a0009101b10001003c000050a00000000600d1
:1009b00080027800800178001004e0000b00320013
:1009c0000101780012427800058051000404e00023
:1009d00007003200934f1200020032000201e800cb
:1009e000f8ff37005304e000f5ff3a00058051009e
:1009f00000000600800178001004e0000a003200c8
:100a0000010178001104e000050032001042780076
:100a1000924f5200040032005204e000fbff3a0003
:100a20005004e000f6ff3a0003005000000006000a
:100a3000800178000200e00003003200b159780024
:100a40000201e900fdff3a00000006000001780005
:100a5000314978003204e000fdff3a000000060052
:100a6000800078001106b100030035009101b1004b
:100a700001003c000050a100000006000200fa0046
:100a8000889fbe008a9fbe008c1f780000057800fa
:100a900081047800020678000100e00001003a00bd
:100aa000ec8457000a047800010037000804e800cd
:100ab0001800fb00c50007000000e000fbff3a0043
:100ac00098407800d0c2b30080cf500003003200bd
:100ad000bbc2b3008bcf500002003a0081457800c2
:100ae0000804e8000c0178000800be0012fe0700b0
:100af0000001be00990f540001003a008a0c7800f2
:100b0000990f550003003a00e00f5100e08f5900a3
:100b10000e003a00b0c2b30080cf550003003a0087
:100b2000e00f5100e08f590008003500d0c2b3003b
:100b300080cf55000f003a0000002000010028007f
:100b4000800f5100818f59000a00360020022000da
:100b5000f0ab880002002000030028006b4040003a
:100b600080cf550008003200f2ff2f00f3ff27006e
:100b700005003700d0c2b30080cf550002003a0014
:100b800060011100e08119000200be004f067800ec
:100b90004f05be004f04be000080fa0000000600b2
:100ba0000200e0000b003200104278009141780012
:100bb000834f5200030032000080eb000600390032
:100bc000100005000000e8008100e8000201e900d3
:100bd000f5ff3a000000eb00000006000003b10042
:100be000030035009000b10001003c00100005003a
:100bf0000000050010417800914f510006003a00b6
:100c00008001eb000204e0000a003200504178004d
:100c1000d14f5100faff320010407800914f500040
:100c2000020031000080eb000100370010002000be
:100c30008001780003007800000006008002780040
:100c40000200e0000e003200954178001142780069
:100c500084cf5100030032000080eb00090039000e
:100c6000100005000000eb000304e0000500320066
:100c70008502e8008100e8000201e900f2ff3a0085
:100c80000000eb000000060090cf100005003200cd
:100c90001004e00001003a0000000500d0cf100071
:100ca000fbff3a0000000600881f7800020478006d
:100cb0005fff0700080040004f04780000000600b6
:100cc0000000fa00881f7800000478003fb9970000
:100cd000ea8157008000780040652000eb030700a0
:100ce000800078000000e000020035000040eb00ca
:100cf00000f47800010078004f0478000080fa00ca
:100d000000000600889fbe0000047800820478007e
:100d100010019000890f5100010031008204780019
:100d2000180078000901780041ff0700188c440082
:100d30001800900009005000100498000800780086
:100d40004f04be00000006000400fa000100e000ad
:100d500004003a000f80e900e0bf9f000008eb00ac
:100d600003003700e0bf9f008100e900f1bf9f0052
:100d7000e480570020682000c4030700efb8970004
:100d80008048eb000080fa00000006008001780037
:100d9000000178001004e000020032005204e0007c
:100da000feff3a0011407800004978000004e0009e
:100db0000400320051407800006978000004e0002f
:100dc000fcff3a0003007800000006006900e10023
:100dd000040035006d00e100030034000002b100a2
:100de0000100320000000500100005000200e000d4
:100df0000500320090cf1000040032000000e8002f
:100e00000201e900fbff3a000000eb0000000600d1
:100e1000889fbe008a9fbe008c1f78000006780065
:100e200081057800100478000005eb000100370010
:100e30000804e8001800fb00e4ff07000000e000e1
:100e4000fbff3a0098407800d0c2b30080cf50003a
:100e500002003a008a00200003003700b0c2b3004d
:100e600080cf500001003a000804e8009840780064
:100e7000e2c6b30082cf500003003200e3c4b300e7
:100e800083cf50001f003a00d840780010c6b3004e
:100e900080cf50000300320010c4b30080cf500058
:100ea0002a003a00d840780082cf50000300320078
:100eb000e0c4b30080cf500024003a000804e800ea
:100ec000880478004a00200080c2b300984f1000c8
:100ed00007003a005900fb00210407000000e00071
:100ee000fcff3a00f0c5b300994f1000f9ff320043
:100ef00090c2b300994f10003c003a000904e8008a
:100f00003a00370090c6b30080cf50000300320093
:100f100090c4b30080cf500038003a0058407800a9
:100f2000824f500002003200834f500007003a0009
:100f3000d840780060c6b30080cf50000600320071
:100f400060c4b30080cf5000030032001c0478005e
:100f50000005eb00250037003a00b300d8407800c8
:100f600093c6b30083cf50000300320090c4b30097
:100f700080cf50001d003a008800e8001141780041
:100f8000e0c6b300804f510003003200e0c4b3005c
:100f9000804f510015003a0051417800834f5100b5
:100fa0000300320090c4b300804f51000f003a009c
:100fb0005141780040c7b300804f51000300320018
:100fc00040c5b300804f510008003a0051417800fd
:100fd00090c7b300804f51000300320090c5b300aa
:100fe000804f510001003a000104e8000b00e000ce
:100ff00003003200880d7800010037000a00a000cd
:10100000080e78000a0078004f0678004f05be00f1
:101010004f04be0000000600e6874700889fbe0020
:101020008a9fbe008c9fbe008e1f7800f0b79f0085
:101030000105780082bf9f000306780083047800d2
:101040006920b900000478008006eb0000c3b300fb
:101050009a4f100003003a001d002000da4f1000e4
:10106000fdff32008005eb00000eeb003c1678001f
:1010700028003700888f550016003d0092002000a0
:10108000110009008205d800010078000000e0008e
:1010900003003a00e4844400800ceb00b9147800ab
:1010a0001900be00a200200003002000df1107008d
:1010b0001a4178000201fb00cf91de0000004100e0
:1010c000818049000003b1000180b100808cbe0026
:1010d0000d00370010002000010020001c0e400011
:1010e0005c964800888f550008003a0040c3b30062
:1010f0009a4f100005003400120020000300200069
:10110000990c4100d99449008b05e8000a05e800d4
:101110001d0020001a00fb00b0fe07000000e000e8
:10112000d4ff3a008b0f540001003d008805780081
:10113000e0c2b3009a4f100001003a000a05e8002f
:101140000b00e00029003a0000c3b3009a4f1000e2
:1011500026003a000081eb008081eb001c0e41006c
:101160005c9649001d002000da4f1000f9ff3200a4
:101170001e003700888f55001a003d0092002000a5
:10118000110009008205d800010078000000e0008d
:1011900003003a00e4844400800ceb00b9147800aa
:1011a0001900be00a2002000030020009f110700cc
:1011b0001a4178000201fb00cf91de0000004100df
:1011c000818049000003b1000180b100808cbe0025
:1011d0008b05e8000080eb008080eb001c0e4000d7
:1011e0005c9648000a05e8001d0020001a00fb007c
:1011f0007afe07000000e000deff3a0092002000c7
:10120000110009008205d800010478000800e00000
:1012100010003200690414001902be00e00f5200f1
:10122000e08f5a00070032006440b80022512100cc
:10123000020040001001be000400be007b11070048
:10124000808cbe00888545006140b9001c1e1000de
:101250001c961800e88f5500100034001900be00dd
:10126000e00f5000e08f58000c003a00e98555006f
:1012700090002000010020001c0e40005c964800f9
:10128000e4845400e88f5500040034001900be00c7
:10129000e00f5000e08f5800f4ff32000d00e00036
:1012a000310032009a40780050c6b30080cf500021
:1012b0000300320050c4b30080cf50002a003a002f
:1012c000da407800b0c2b30080cf50000400320092
:1012d0000047780000c0e80080cf500002003a00cc
:1012e000014778000a05e8006044b8008006eb007a
:1012f00012003700f00f2e00515f2000800f5400c5
:10130000818f5c000b003c00a20020000300200045
:101310000800be00451107001a4178000201fb00d9
:10132000cf91de0000044100818449000803b10030
:101330000980b1000a05e8001d0020001a00fb002a
:1013400026fe07000000e000eaff3a00d0c2b3002a
:10135000804f570002003a0060041400e0841c0033
:101360001c0e44005c964c008fb897000100e00012
:1013700006003200ffb097000d00e00001003200cf
:101380008a0078000fb997000109780092002000c8
:10139000110009008205d8004f0778004f06be00f3
:1013a0004f05be004f04be006f00b10000000600f4
:1013b000e6874700889fbe008a9fbe008c9fbe00c4
:1013c0008e1f7800f0b79f000105780082bf9f0054
:1013d00083057800030478006720b9008004780052
:1013e0008006eb0000c3b3009a4f100003003a00e0
:1013f0001d002000da4f1000fdff32000006eb0058
:10140000800deb00bb1578002e003700890f5600c9
:1014100019003d0072002000811f780011000900b2
:101420000206d80001007800cf0078000000e0003c
:1014300003003a0064044400000ceb003814780008
:101440001801be004418dd00cc11de0083017000dd
:101450004411dd00a0472100008050001149210007
:1014600060c078000000fb00cf80de00001c41005f
:1014700001944900100037001200200003002000f2
:101480009b0d4100db954900890f56000b003a0087
:10149000a0472100008050001149210060c0780061
:1014a000e74f50000500340010002000010020002c
:1014b000180c4000589448000c06e8000a05e800a3
:1014c0001d0020009a00fb0062012000a0472100bf
:1014d00046fe0700800078000000e000cbff3a00e5
:1014e0008c8f540001003d0009067800e0c2b30073
:1014f0009a4f100001003a000a05e8000c00e000d5
:101500002c003a0000c3b3009a4f100029003a00a3
:101510000081eb008081eb009b0d4100db954900d1
:101520001d002000da4f1000f9ff320021003700c3
:10153000890f56001d003d0072002000811f7800b9
:10154000110009000206d80001007800cf007800e1
:101550000000e00003003a0064044400000ceb00cb
:10156000381478001801be004418dd00cc11de00ec
:10157000830170004411dd00a0472100008050006d
:101580001149210060c078000000fb00cf80de0020
:10159000001c4100019449000c06e8000081eb00aa
:1015a0008081eb009b0d4100db9549000a05e800b6
:1015b0001d0020009a00fb0062012000a0472100ce
:1015c0000afe0700800078000000e000d8ff3a0023
:1015d00072002000110009000206d8000100780006
:1015e0000000e0000d003200670010006402b90046
:1015f0001801be000402e9000300330002014100ab
:1016000083814900fbff3700028cbe0000064600c4
:10161000cf80de009b1d10009b951800e60f560042
:10162000100034001800be00e00f5000e08f58009a
:101630000c003a00670656007000200001002000f0
:101640009b0d4000db95480064045400e60f5600f3
:10165000040034001800be00e00f5000e08f580076
:10166000f4ff32001b00be004209dd00ce00de00a8
:10167000810071004200dd00808dbe000d00e000a1
:10168000310032009a40780000c7b30080cf50008c
:101690000300320000c5b30080cf50002a003a009a
:1016a000da407800b0c2b30080cf500004003200ae
:1016b0000047780000c0e80080cf500002003a00e8
:1016c000014778000a05e8006044b8008006eb0096
:1016d00012003700f00f2e00515f2000800f5400e1
:1016e000818f5c000b003c00a20020000300200062
:1016f0000800be004d1007001a4178000201fb00ef
:10170000cf91de0000044100818449000803b1004c
:101710000980b1000a05e8001d0020001a00fb0046
:101720002efd07000000e000eaff3a00d0c2b3003f
:10173000804f570002003a0060041400e0841c004f
:101740009b0d4400db954c008fb997000300e0002f
:1017500006003200ffb097000d00e00001003200eb
:101760008a0078000fb89700010878007200200006
:10177000110009000206d8004f0778004f06be008e
:101780004f05be004f04be006f00b1000000060010
:10179000881f78008a9fbe00000478000205be0002
:1017a000300190000200d000c500de00f07f200074
:1017b000808f50000c003a006f00610008003a0072
:1017c000280090000000e00005003a00180090009a
:1017d0000000e00002003a001800e0001c003200a7
:1017e000200020005d0037000100e00006003a0004
:1017f00008007800e8010700800078000000eb0096
:101800000100e00055003c006108b9000a054000f5
:101810008b854800e07f2000800f5500e08f5d0041
:101820000d003400380090006022b800060020004f
:1018300007ff2f000000e000030035006022b80021
:101840000600200007ff2700049cbe000694be008f
:101850001000200041003700b8009000e00f550054
:10186000e08f5d0005003400f0002800008060007b
:10187000c450dd0001007000360037000000280071
:10188000808260006f8060000040a00030049800fb
:1018900061055500e0855d00c0fc2f00f1ff2f00c1
:1018a000800f5500818f5d0006003d0035049800d3
:1018b0000000eb002004980010049800000ceb00de
:1018c000260037000a027800f00f45000b003c00ac
:1018d00018009000000c7800280090001004980078
:1018e00038009000200498000000eb0030049800bd
:1018f00070024200f00f4200f5ff34000402ea00db
:1019000012003200180178000411de00f00112000c
:10191000180090008300dd00010c71000400de005f
:10192000280190008310dd00010070001004980071
:101930000411de00380090008301dd000301710016
:10194000220498000400de00300498003800900063
:1019500005007000300498000080eb004f05be00c9
:101960004f047800000006000200fa00889fbe00c5
:101970008a9fbe008c1f7800000678000404be0019
:101980000605be00800078006c805700d501070076
:101990003c00be002c01be000802be000a03be00cf
:1019a000770a0700009ebe000296be002fb997007e
:1019b000cf91de000c00780075ff07004f0678001d
:1019c0004f05be004f04be000080fa000000060074
:1019d0001800fa00889fbe008a1f780090b79f0009
:1019e000a1b79f00b2b79f00c3b79f000404be0019
:1019f000e00f5200e08f5a009c0032006022b800d5
:101a00006033b800c90807000000e000970032000a
:101a10006000b8000200200003ff2300d0b79f0041
:101a2000e1b79f00f2b79f0083bf9f00e00f540013
:101a3000e08f5c0048003d0060041400e0841c005e
:101a40000005eb001a0032000808a3001000320065
:101a50006850b800823e2100020040003002be0003
:101a60002003be005fb09700efb097007fb19700f2
:101a70008fb99700420a07000002be000203be00b1
:101a8000d4b79f00e5b79f00f6b79f0087bf9f00c0
:101a90008904d1000884d3000a05e800e00f54004f
:101aa000e08f5c0002003200e70f5500e6ff3600d1
:101ab0005fb29700efb297007fb397008fbb97009c
:101ac0006000b8000200200003ff2300a108070007
:101ad0000002be000203be007e805700a2ff070086
:101ae000000578000000e00059003d00e00f5400c0
:101af000e08f5c0056003200834221003302be00ba
:101b00002303be006000b8000200200003ff230092
:101b10009008070090bf9f00a1bf9f00b2bf9f0029
:101b2000c3bf9f001fba9700afba97003fbb970093
:101b3000cfbb97007e8057008bff07000005780021
:101b40000000e00042003d0061045400e0845c00bd
:101b5000f4ff3a003e003700e00f5400e08f5c00d5
:101b60003b0034000005eb000808a3001000320021
:101b70006850b800823e2100020040003002be00e2
:101b80002003be005fb09700efb097007fb19700d1
:101b90008fb99700fa0907000002be000203be00d9
:101ba000d4b79f00e5b79f00f6b79f0087bf9f009f
:101bb0008984d1000884d3000a05e800e00f5400ae
:101bc000e08f5c0002003400e70f5500e6ff3600ae
:101bd0005fb29700efb297007fb397008fbb97007b
:101be0007e80570060ff0700000578000000e000dd
:101bf00017003d00e00f5400e08f5c00140034003b
:101c0000814221005101be004100be00d0b79f00bb
:101c1000e1b79f00f2b79f0083bf9f005fb29700bc
:101c2000efb297007fb397008fbb97007e8057007d
:101c30004dff0700000578000000e00004003d00b3
:101c400061045400e0845c004240a900f3ff3c00c2
:101c5000000120000a00e00003003200e10f5500ff
:101c600002003a00800020004c0107001fb09700de
:101c7000afb097003fb19700cfb197004f05780004
:101c80004f04be000080fa00000006006200fa0067
:101c9000889fbe008a9fbe000004be000205780037
:101ca000830078006a80570047010700f88f9f0083
:101cb00089979f000000eb00909f9f001a80fb0017
:101cc0008005fb000000ea00cf04de000904780074
:101cd00050022000808f550001003a000904e900fd
:101ce0000800e0000c0034000f9097000801780015
:101cf0008a007800ff8997000300010080979f0009
:101d00008080eb000000e000900032001f989700f8
:101d100008004000909f9f000905450050022000e8
:101d2000808f5500040032000b00e000e3ff3a0012
:101d30009f989700850037000000eb00f0979f0008
:101d4000e0979f00d0979f00c0979f00b0979f009b
:101d5000a0979f00b09f9f0009003700c05421004a
:101d6000008050000000d0002155210001004000fb
:101d7000bf98970090807000b19f9f000a05e8000f
:101d80009a00fb00c0542100bffb070080007800d0
:101d90000000e000f1ff3a00a0c2b3009a4f10002b
:101da0000e003a003fb897000080e900b0bf9f00e6
:101db00010007800a09f9f000000e00005003d009b
:101dc0000000ea00a09f9f003f9897000020a0001d
:101dd000b09f9f000a05e80011003700a19f9f00f7
:101de0000b003700af989700f0ff2700808f50005e
:101df000060032006a09b9001a00fb000200400028
:101e000001fd2f0001004000a09f9f000a05e8008f
:101e10001a00fb0071fb07000000e000f1ff3a0030
:101e2000e0c2b3009a4f1000030032000080eb00c4
:101e3000809f9f001c003700a0c2b300da4f100043
:101e400007003a003fb897000080e900b0bf9f004c
:101e500010007800809f9f000a05e80012003700fc
:101e60000000eb00809f9f000b0037008f989700c9
:101e7000f0ff2700808f5000060032006a09b90089
:101e80001a00fb000200400001fd2f00010040008d
:101e9000809f9f000a05e8001a00fb004ffb070027
:101ea0000000e000f1ff3a009a00fb0020ee210064
:101eb00075fb07008040eb000000e00001003200ed
:101ec000ba407800817f9f0080c6b30080cf500069
:101ed00004003a009acf100002003a006640500019
:101ee000070037008f789700c0c6b30080cf50003e
:101ef00005003a009acf100003003a006540400008
:101f0000807f9f000a05e800a0fb2f0000844700a7
:101f10003a01fb0088017800ea80570060f92f0041
:101f20000f004000780107000000e00006003a00c2
:101f30008800780060f92f000f004000a40007001f
:101f40000000e0005dff3d008080eb0001007800b4
:101f50004f05be004f04be000080fa0000000600de
:101f60000003b1000b0035009000b1000800340000
:101f70008000b100070035009001b100040034007a
:101f80007000b100030035009001b10001003c0079
:101f900010000500000005000002780030009000ed
:101fa0000100280001036000150020006f006000a0
:101fb0003002980008003a00240090000000e00081
:101fc00005003a00140090000000e00002003a0012
:101fd0001400e0003e003200340090000000e000f9
:101fe0000b003a002400900030029800140090008a
:101ff000200298001400780010029800000aeb00fc
:10200000f0825200340090000000e000f5ff320042
:1020100034009000ef0f500014003e008001d0000b
:10202000a40090004f08de00808171003302980008
:102030008100d000140190004f10de0080807000fd
:10204000210298000201d000940078004f08de00c1
:102050000001710012029800010ad0008502e90017
:1020600003007800ef8f5100ecff3600b4019000c0
:10207000ff8f5100130036001401d10014009000ae
:10208000cf00dd00010a71000000d100a400900023
:102090004f09dd0002007000100298008100d1009d
:1020a0004f18dd0080807000210298000300d100ed
:1020b000300298008502e80080017800ff0f500090
:1020c000edff3e00340090006f0060003002980089
:1020d000340090000600700030029800050078007f
:1020e00000000600889fbe0080047800010478008c
:1020f000310090000000d0004501de00f07f20009c
:10210000800f510010003a00800ceb00310090006d
:102110006f00600008003a00210090000000e0001d
:1021200005003a00110090000000e00002003a00b3
:102130001100e000020032002000200015003700ee
:1021400010002000130037000200e00005003c00f2
:102150000100780090ff0700000178000000e00017
:102160000a003c0038009000f100280001006000e7
:1021700001fe2300010070003004980020c02f00f1
:10218000800c41000080eb0002003700800ceb0067
:102190000000eb004f04be00000006008000780045
:1021a000650060000300320010022000f0ab8800e0
:1021b000000006007880600002003200200220004b
:1021c000f0ab88000000060001087800000006005f
:1021d0000400fa00889fbe008a9fbe008c1f780012
:1021e000000478000106780070089000f800900064
:1021f00001005000880890000100500098089000ed
:1022000001005000a808900001005000b80890009c
:1022100001005000c8089000810550000002220013
:1022200090bf9f0000032300a0bf9f0008109000f4
:102230000028a30018003a000b00e000160034004c
:102240000b0578008a047800e20f55000100360083
:10225000290020000900e0000c0034005800900024
:10226000c801900009017800ee80570003000100ca
:10227000500498008080eb000000e0009c003200d9
:102280006808900009004000600c9800090555009e
:102290004240a900ebff3c00780190000200e00002
:1022a0000c00340058009000c80190008c007800a9
:1022b00003000100500498008080eb000000e00063
:1022c0008b00320068089000f80090000100400088
:1022d000600c9800080890000000e0001600340030
:1022e000000578008a047800e20f550001003600ee
:1022f000290020000900e0000c0034005800900084
:10230000c801900009017800ec805700030001002b
:10231000500498008080eb000000e0007400320060
:102320006808900009004000600c980009055500fd
:102330004240a900ebff3c00180990000200e000b9
:102340000c003400e800900058009000c801900094
:1023500003000100500498008080eb000000e000c2
:102360006300320068089000980890000100400067
:10237000600c9800280890000000e000160034006f
:10238000000578008a047800e20f5500010036004d
:10239000290020000900e0000c00340058009000e3
:1023a000c801900009017800ec805700030001008b
:1023b000500498008080eb000000e0004c003200e8
:1023c0006808900009004000600c9800090555005d
:1023d0004240a900ebff3c00380990000200e000f9
:1023e0000e003400e8009000180890008080400043
:1023f00058009000c80190000300010050049800ac
:102400008080eb000000e000390032006808900096
:10241000b808900001004000600c98004808900047
:102420000000e00016003400000578008a047800ff
:10243000e20f550001003600290020000900e000ed
:102440000c00340058009000c80190000901780089
:10245000ec80570003000100500498008080eb00de
:102460000000e000220032006808900009004000ef
:10247000600c9800090555004240a900ebff3c00a4
:10248000081090000028a300180032000b00e000a4
:10249000160034000b0578008a047800e20f55001e
:1024a00001003600290020000900e0000c00340083
:1024b00058009000c801900009017800ee80570094
:1024c00003000100500498008080eb000000e00051
:1024d000070032006808900009004000600c980076
:1024e000090555004240a900ebff3c008000eb00cd
:1024f000010078004f0678004f05be004f04be0073
:102500000080fa0000000600889fbe008a1f780045
:102510000004780001027800024578008304780006
:102520000200fb00cf80de005002b1000180b1004c
:1025300032052000820f5000e08f58008c013e00d1
:1025400000600100840137008901370088013700ed
:102550008701370086013700850137008401370085
:102560008301370082013700810137008001370085
:102570007f0137007e0137007d0137007c01370085
:102580007b0137007a013700790137007801370085
:102590007701370076013700750137007401370085
:1025a0007301370072013700710137007001370085
:1025b0006f013700ed0037006d0137006c01370007
:1025c0006b013700e9003700e8003700e70037000b
:1025d0006701370066013700650137006401370085
:1025e0006301370062013700610137006001370085
:1025f0005f0137005e0137005d013700420137009f
:102600005b0137005a013700590137005801370084
:10261000800037005601370055013700540137005c
:102620005301370052013700510137005001370084
:102630004f013700cd0037004d013700150037003e
:102640001c003700c9003700c8003700c70037003a
:1026500047013700170037004501370044013700b4
:102660004301370042013700e300370069003700bb
:10267000160137003e0137003d01370022013700c7
:102680003b0137006300370039013700380137005c
:10269000600037006e014400120078008081410024
:1026a0009480e900010a78000009e8009149780067
:1026b00038013700a8609000c0c6b30080cf50003a
:1026c0000a003a009400780064805000000a780004
:1026d0001000be004f89de00cf91de000002be0078
:1026e00002037800820378001500370010c7b3009a
:1026f00080cf500002003a00140178000400370037
:1027000014017800a0c6b30080cf500005003a0045
:1027100068005100000a78003002be002003be00ad
:10272000070037000280e900000a780010007800f6
:1027300000027800cfa2de0005037800860378004f
:10274000049cbe000694be00a860900080c6b30042
:1027500080cf50000f00320020c6b30080cf500061
:1027600006003a00184078000000fb00cf80de0031
:1027700001017800820178000a00370040c7b300e9
:1027800080cf5000030032006640400080cf5000f0
:1027900006003a0018007800cf80de0001017800c2
:1027a00082017800009cbe000294be003800be008a
:1027b0002801be00e00f5000e08f5800e00f5900e4
:1027c000e08f590004003d006e0144009200780043
:1027d000d0c2b3000c003700081090000018a3000e
:1027e000040032006e01440092007800b0c2b300d1
:1027f000050037000008a300570032006e014400b6
:102800009200780000c2b30080f478000109e8006b
:1028100051003700a8609000c0c6b30080cf5000c0
:1028200006003a009400780064805000000a7800a6
:102830001002be006033b8001500370010c7b300a7
:1028400080cf500002003a001401780004003700e5
:1028500014017800a0c6b30080cf500005003a00f4
:1028600068005100000a78003002be002003be005c
:10287000070037000280e900000a780010007800a5
:10288000000278000500200006002000070020005c
:10289000049cbe000694be00a860900080c6b300f1
:1028a00080cf50000f00320020c6b30080cf500010
:1028b00006003a00184078000080fb00010020006c
:1028c00002002000030020000a00370040c7b300c8
:1028d00080cf5000030032006640400080cf50009f
:1028e00006003a00180078000100200002002000d5
:1028f00003002000009cbe000294be00081090005f
:102900000038a300140032003800be002801be00c9
:10291000e00f5000e08f5800e00f5900e08f5900a1
:102920000d00320080c7b300804f55000300320015
:1029300080c5b300804f550007003a006e00440088
:102940009000780002c3b30082f478008100e800b0
:102950008af478000108e8007800900000804400c4
:10296000600498008a407800640037001401780001
:1029700068005100000a78005001be004000be000f
:10298000009cbe000294be00380090000000e000f1
:1029900004003d006e01440092007800d0c2b300f4
:1029a0000c003700081090000018a300040032004b
:1029b0006e01440092007800b0c2b30005003700f9
:1029c0000008a300050032006e0144009200780068
:1029d00000c2b30080f478000109e800780090009c
:1029e00000804400600498008a4078000800780065
:1029f0001e01070067003700286090008000fb0080
:102a0000c0062000808f5000230032000a003c00e6
:102a100064005000808f50002600320004003c000b
:102a200066005000808f50000b00320021003700fc
:102a3000a00620000500370040072000808f5000ce
:102a40001c0032001b003c0063005000808f5000cf
:102a500007003200170037001480e900000a7800f0
:102a600010007800485c9000084878004900370062
:102a70001480e900000a78001002780068089000cd
:102a8000cf80de000101780082017800009abe004c
:102a90000292be003f0037001480e900000a78006f
:102aa0001001780068089000cf80de000089be0029
:102ab000380037001480e900000a78001000780020
:102ac000680c900008087800320037001480e90094
:102ad000000a780010007800cf80de000101780045
:102ae00082017800009cbe000294be007800900035
:102af000008044006004980081c7b300080078009b
:102b000028000700230037001480e900000a78003d
:102b10001000780060049800580990000200e0005e
:102b200002003d007df70700090037008000eb0040
:102b3000aef80700800078000000e00003003200db
:102b40006800900000805000010037005808900095
:102b5000100c98000f0037006e01440092007800be
:102b600050c2b30080f178000109e8000900370085
:102b7000ee00440011007800808144000a42780091
:102b80008008e8000a04e00001003a0054c2b300e3
:102b9000844978000000eb004f0578004f04be0028
:102ba000000006006f02b000889fbe008a9fbe0032
:102bb0008c9fbe008e1f780080067800504e21004a
:102bc000b0b79f0080c5b30080cf50000200320034
:102bd000424d2100b2b79f0083002000c3b79f0081
:102be000f0c6b30080cf50000a00320069404000b8
:102bf00080cf500005003200a4002000c4b79f0021
:102c000080c5b30080cf500002003a0000012000d0
:102c1000c0b79f008e0120003d04be002d05be0000
:102c200040c6b30080cf5000030032006540400032
:102c300080cf50000a003a00e00f5400e08f5c00a3
:102c4000e00f5d00e08f5d0005003d000800be0064
:102c50000a01be000a0b07000205be000004be0008
:102c6000e00f5400e08f5c00e00f5d00e08f5d003e
:102c700003003a005d0890000000e0000c00320004
:102c80007e012000cfb0970001027800cfa2de00c5
:102c900005037800860378000800be000a01be0024
:102ca0008d0b07003fb2970064407800d0e79f008b
:102cb0004fb09700cf80de000101780082017800dc
:102cc000d0b79f00e1b79f00f2b79f0083bf9f007e
:102cd0000203be000002be000800be000a01be00e2
:102ce000760b0700809ebe008296be00e00f50006b
:102cf000e08f5800e00f5900e08f590022003400a7
:102d00000e00e000200034003d00be002d01be009a
:102d10005fb29700efb297007fb397008fbb970029
:102d2000710b07000205be000004be000e07e9009b
:102d3000e1fc2f008f804000010647005fb2970042
:102d4000efb297007fb397008fbb97000800be00db
:102d50000a01be00010c07001d0010003fb19700e2
:102d6000624e7800889ebe008a96be00e00f540036
:102d7000e08f5c00e00f5d00e08f5d00020034003a
:102d80000e00e000e0ff3c00cfb19700e88f51005b
:102d900010003a000d1090000038a3000d00320022
:102da000f70f570006003e00e4fc2f000e02420021
:102db000e4c07f0000c3b30080cf500005003200a4
:102dc0000e07e90000c3b300e1fc2f008e80400035
:102dd00080f07f0078011700920e98006d0090003f
:102de000e3fc2f008f8141008e80410010f7070027
:102df0001d0e90005d089000800f560006003d00fb
:102e00000c005000800e98000d1090000040a100b2
:102e1000801698000f0037000000e0000d003d0014
:102e20000d10900074006000f00f500009003a008f
:102e30007d089000fd009000010050008d0890007a
:102e4000010050000c0750004240a900010034006e
:102e50008e0e98004f0778004f06be004f05be004b
:102e60004f04be006f02b10000000600ef04b00086
:102e7000889fbe008a9fbe008c9fbe008e1f780078
:102e8000c0af9f00a1df9f0060fa2f000f0040003d
:102e9000e0af9f00cfaa97005503be004502be00d9
:102ea00084af9f0095af9f00a6af9f00b7af9f0074
:102eb00010c6b30080cf50001600320010c4b3001b
:102ec00080cf5000130032004fab9700560890009f
:102ed0000000e00003003d0060002000500b98005f
:102ee0000c0037000000e0000a003a0070c6b30092
:102ef000afdb970080cf53000300320070c4b300f3
:102f000080cf530003003a0010002000cfa89700a4
:102f1000d0089800cfa89700e2fc2f00028047005d
:102f200070fc070080017800e20f500014003a00a6
:102f3000cfa99700e300900030002000900998008e
:102f400010c6b3002fda9700804f52000a003200fb
:102f500064404000804f5200070032000040e8000b
:102f6000804f52000400320002eb21000040e800d4
:102f7000804f520017003a0042eb21001500370045
:102f80000000e00018003400cfaa9700e500900090
:102f900030002000900a980010c6b3002fdb970085
:102fa000804f53000a00320064404000804f5300bd
:102fb000070032000040e800804f53000400320058
:102fc00082eb21000040e800804f530001003a00ee
:102fd000c2eb2100b258780002007800b0587800a7
:102fe00090487800f201370014c6b300afdb9700b9
:102ff00084cf53000300320010c4b30080cf5300cd
:1030000010003a004fa89700ec0040001101780032
:1030100000c3b300005978008208e80080c7b300fd
:10302000afd8970084cf50000100320080c5b300b4
:10303000004978004fa99700720090000080e800d6
:10304000700198000300e00003003a008006eb00e6
:10305000fda79f00d001370011c6b300afd997007c
:1030600081cf51000300320010c4b30080cf510063
:10307000ad003a000eec21002fda9700814f52008c
:10308000010032001eed2100cfaa970055089000e4
:103090008006e8000000e00001003d001d02200065
:1030a0000d06e8004fab97003604be002605be00b3
:1030b0006022b8006033b8000fa897009fa897005f
:1030c0002fa99700bfa99700180307000000e00090
:1030d00001003d000bf0a20088af9f0099af9f0058
:1030e000aaaf9f00bbaf9f007fa097006400500075
:1030f000f0a79f00efab9700805beb00e7af9f006e
:103100003f003700c20120000300200001fd2f0016
:10311000018047009ef907000faa97009faa970019
:103120002fab9700bfab9700f4af9f0085b79f0010
:1031300096b79f00a7b79f000400be000601be001f
:10314000f90507000004be000005be006706560032
:103150004240a9000c003400b70507000002be0081
:103160000203be007fa897008fb097001fb19700a1
:10317000afb19700ae05070080af9f0091af9f00f1
:10318000a2af9f00b3af9f00efaa9700e782420073
:10319000e5af9f0070002000e00f5400e08f5c005e
:1031a0000d003400600020006fab97006f63650076
:1031b000e6af9f00cc5bdd004455de000a8573005e
:1031c000c4ddde00e00f5500e08f5d00020034003a
:1031d0000000e900f4ff3b000000e90005003300b7
:1031e000efa897008060eb00e1af9f000000e900ce
:1031f000fbff3b006fa9970067014100e2af9f0012
:103200000c00e000090034006022b8006033b80010
:103210000fa897009fa897002fa99700bfa9970014
:10322000c70207000000e000b6ff3c00efa99700ce
:1032300064fa2f000f024200048051000006e900ea
:1032400075fa2f0085824700e5af9f008d0f56006d
:1032500001003d008c0678000d00e0002b003500d9
:103260008c8f560005003d006fab970066c07e0056
:10327000f2c0b300e74f500001003c000041eb00fa
:103280008d00e900efab970067c07800824f5000d7
:1032900006003a008d06e9008100e900efa99700d9
:1032a00063c07800824f5000faff3200ef4f5100a8
:1032b00004003a006faa970064c078000040e8005c
:1032c00000f278000100e00007003d00efaa97003f
:1032d0008502e900e5af9f008d06e8007fa097001a
:1032e00064004000f0a79f008d00e9000700330054
:1032f0006fab970066c078000000fb006e4078005e
:1033000000f378008100e900f9ff3b00cfab9700a4
:10331000570890000000e0001f013d000d00e9008b
:10332000d00b98001c0137000fac97009fac9700a2
:103330002fad9700bfad97006022b8006033b80092
:103340000800be000a01be00780207000000e0008d
:1033500005003d000bf0a20088af9f0099af9f00d1
:10336000aaaf9f00bbaf9f007fa0970072592700b4
:103370000280b900026a280013002000310907000a
:10338000e4005000f1a79f001d003b006380100087
:10339000c1ff2f00010460000800ea00f0a79f00b1
:1033a0008004eb000800e000470034000808a30098
:1033b0000e0032006848b80022432100020040009d
:1033c0003002be002003be000fa897009fa8970000
:1033d0002fa99700bfa99700e903070080af9f00be
:1033e00091af9f00a2af9f00b3af9f000884d100b0
:1033f0008904e8000800e000ecff3c0032003700e0
:103400000100e000300034006022b8000600200017
:1034100007ff2300b4b79f00c5b79f00d6b79f0032
:10342000e7b79f00c0ff2f0000806000f0a79f005b
:10343000000478008004eb00160034000808a300a4
:10344000100032006848b800254321000500400004
:103450003002be002003be003fb09700cfb09700ff
:103460005fb19700efb19700c50307000002be00ef
:103470000203be00b4b79f00c5b79f00d6b79f0038
:10348000e7b79f000884d1008904e8000800e00045
:10349000eaff3c003fb29700cfb297005fb39700be
:1034a000efb397000fa897009fa897002fa9970048
:1034b000bfa997002702070080af9f0091af9f0030
:1034c000a2af9f00b3af9f004fab9700d60890000c
:1034d00060c6b300afdb970080cf5300040032001a
:1034e0006687400060c4b30080cf530003003a00f9
:1034f0007fa09700008040006a074000f30f57004c
:10350000010034003e01200000c3b300efa8970083
:1035100080587800e1af9f003a0037000800be00f5
:103520000a01be00000507000006be00f0b79f00bc
:1035300081bf9f00680757004240a9000e00340079
:10354000bd0407000002be000203be000800be006a
:103550000a01be00b60407006022b80046782d00bc
:10356000771924008603070080af9f0091af9f006a
:10357000a2af9f00b3af9f00efa99700e881410081
:10358000e3af9f0088002000e00f5600e08f5e0050
:103590001100340078002000a20020000300200069
:1035a0007fb097008fb89700e3f407006faa9700e9
:1035b00005c3b30005624100e4af9f00f0b79f0070
:1035c00081bf9f00e00f5000e08f580002003400e0
:1035d0000804e900f0ff3b000804e900060033009e
:1035e00000c3b300efab970080637800e7af9f00a4
:1035f0000804e900faff3b006fa89700680040004c
:10360000e0af9f000e00e0000b0034000fac97000d
:103610009fac97002fad9700bfad97006022b80018
:103620006033b8000800be000a01be00c4010700f4
:103630000000e000b9ff3c00efa8970062fa2f00fd
:103640000f014100028050000007e90073fa2f00cb
:1036500083814700e3af9f007fa097006700400091
:10366000f0a79f0001c3b30093cf10000a003a00f7
:103670000e07e9007fa097000000e900f0a79f0077
:103680006faa97000402e800e4af9f00144278009c
:10369000814f5200f6ff3200cfaa9700d508900064
:1036a00060c6b3002fdb9700804f53000300320049
:1036b00060c4b300804f530004003a007fa097001d
:1036c000008040008006e8000a0037008001eb001f
:1036d00050c6b300afdb970080cf53000300320029
:1036e00050c4b30080cf530001003a001300200003
:1036f000838640008d0f570001003d008e06780044
:103700000d00e000240035008e8f560006003d00bd
:103710006fa89700e0c07e0092c3b30040c3b3001f
:1037200080cf500001003c0002c3b3008d00e900cf
:10373000efa9970063c07800824f500006003a005e
:103740008d06e9008100e9006faa970064c0780047
:10375000824f5000faff320090c3b300804f5100f7
:1037600004003a00efaa970065c078000040e80026
:1037700080f278000100e00007003d006fab970089
:103780000603e900e6af9f008d06e8007fa09700e2
:103790000000e800f0a79f007fa297008d0178004d
:1037a0006fa99700afd897004fa8970006000700b1
:1037b0004f0778004f06be004f05be004f04be0005
:1037c000ef04b100000006000a00fa00889fbe0066
:1037d0008a9fbe008c9fbe000004780001457800df
:1037e0008205780083047800040678000300e00076
:1037f00002003c0019002000abee210060c6b300bf
:10380000804f55000e00320060c4b300804f550059
:103810000b00320070c6b300804f55000300320029
:1038200070c4b300804f550083003a00e40f460097
:103830008100350058089000800f56007e003d0042
:103840000c06e80060c6b300804f5500100032003f
:1038500060c4b300804f55000d0032000810900086
:103860000038a30004003a0058089000808f5400ec
:1038700001003d00590c9800580890000c005000c1
:10388000500c980002003b000000eb00500c980028
:103890000c00e00027003c00f20144001301780016
:1038a0006800900001c3b300017079000201e800d4
:1038b00082097800580890000000e00003003c00f6
:1038c000081090000038a30004003200e8009000c7
:1038d000e0c2b300807079008209e8000c00ea00c1
:1038e000d8089000808f500001003d000106ea00da
:1038f0000c00ea00200c98000c804000500c98004e
:10390000890f500001003d0080047800680090009d
:103910009808900001004000390c980009017800d7
:103920008b00780042f4070058089000090050000e
:103930001a003700e8009000180890008c8f54009f
:1039400018003d0000804000090178008b007800dd
:1039500037f407001808900009014000120c980085
:1039600009005600200c9800580890000000e00064
:1039700003003c00081090000038a300060032004d
:10398000e8009000e0c2b300807079003808900031
:103990000000e800300c980058089000400c980097
:1039a000a3003700008040000c0178008b007800f5
:1039b0001ff40700180890000c004000100c98003d
:1039c0008c845400580890000000e00003003c0084
:1039d000081090000038a30006003200f2014400f5
:1039e0009300780068019000e0c2b30000f1780015
:1039f0008109e80058089000890f500001003d003f
:103a00008004780068009000980890000100400051
:103a10008c8045000901780005f407001808900023
:103a200009004000100c9800580890000900500050
:103a3000200c98007e00370070c6b300804f550000
:103a40000300320070c4b300804f550014003a00e8
:103a500058089000808f540004003d00081090002a
:103a60000038a30001003a00590c98005808900053
:103a70000000e900500c980002003b000000eb0041
:103a8000500c980051c6b30070c6b300804f55006b
:103a90000100320051c4b30001457800090037002d
:103aa00010c6b300804f550002003a000ac7b300a9
:103ab0000400370010c4b300804f550001003a00e5
:103ac0000ac5b300f20144001301780068009000b9
:103ad0003b7079000201e8008209780058089000e4
:103ae0000000e00003003c00081090000038a30034
:103af00004003200e8009000e0c2b300807079005a
:103b00008209e800580890000000e000100034002e
:103b10008904e900890f500001003d00800478000d
:103b200068009000980890000100400009017800aa
:103b30008b007800bef307001808900009004000d1
:103b4000100c98005808900009005000200c9800b4
:103b5000e800900018089000808540008a5d780099
:103b60008b06e8000c00e00004003500b0c2b30092
:103b7000804d78008d05780004003700d0c2b30076
:103b8000804d78008d0578000c06ea008004eb007b
:103b90000c00e00009003400a10020000c007800b7
:103ba0003a0007007681540001f17f00000678009a
:103bb0008904e8000000e000f7ff3c00e18f5400ba
:103bc00009003c0050c6b300804f5500030032008e
:103bd00050c4b300804f550003003a0000c3b30047
:103be000805e78008d0578000900e00002003a0050
:103bf00000c3b300805d78000900e00007003400d6
:103c00008904e900f680540061c07f0002c3b3005c
:103c1000825d40000900e000f9ff3c006800900070
:103c2000980890000100400000805500300c98007a
:103c30000810900074006000f00f50000e003a0071
:103c4000780090009808900001004000a8089000bb
:103c500001004000b808900001004000c808900032
:103c60008100400078089000808f500002003d00e5
:103c700001005000000c98004f06be004f05be002a
:103c80004f04be000080fa00000006000101780029
:103c900000027800110009000200d8000002fd00b7
:103ca0000491b900820250000400be00000006002a
:103cb00081037800b40307000001be006000b80073
:103cc0000478a30013003a006220e10015003e00d2
:103cd0000d0039008301d1000281d3008180d3001f
:103ce0008301d1000281d3008180d3008301d10000
:103cf0000281d3008180d3000538b000c42add00e2
:103d0000f300b2008381720007f0a70003f0a00067
:103d100000000600f3ff2700f2ff2f006110b9003a
:103d2000fbff370003ff2700f7ff37008f1fd1008d
:103d3000aa0307008f87e9000000e00000000600ea
:103d4000809feb00a50307008f87e9000000e000db
:103d5000000006002800fa00889fbe008a9fbe006f
:103d60008c9fbe0003866b00c50307006400e10062
:103d7000440032006408e1004a0032006100e100c2
:103d8000460032006108e10049003200ec064700bd
:103d90006000b8003d02be003d03be00f48657003f
:103da0006011b8003d04be003d05be007d0320004b
:103db0000b0037000000a0008d06e9001300320060
:103dc0000402420085824a0006034b0087834b00b1
:103dd00000004000818048000201490083814900c1
:103de0000802520089825a000a035b008b835b0041
:103df000f0ff3b000802420089824a000a034b00a0
:103e00008b834b008d06e900edff3a00848272003f
:103e100086827200f707b2008782720001003200ca
:103e2000150020001e0490003e0b90000603540075
:103e3000e63fb0000368a300070032000000a700bf
:103e40000500a0008301d1000281d3008180d3004e
:103e50000080d3000603e8008301d1000281d30073
:103e60008180d3000080d3000002eb000482d200e6
:103e70009c03070003f0a1000cf0a70003f0a000d2
:103e800093033700640247006408e1008d033200a9
:103e90003400be003401be00f6ff37006108e100c7
:103ea000880332006011b8006000b800f1ff3700ed
:103eb00003ff270002002000fbff37002800fa0064
:103ec000889fbe008a9fbe008c9fbe0007067800b8
:103ed000878669000c003b000304780087047800a3
:103ee00008f0a10009f0a100840f5000858f580050
:103ef000860f5900890f5c00030033000cf0a2000c
:103f000001003a000cf0a1005d0307006400e1002d
:103f10005f003200780147006408e1006100320070
:103f20006c014700748557003200be001201be00cc
:103f30003a04be001a05be001e039000be0a90009f
:103f40008503530006003d000004fd008104fd00d0
:103f50000205fd008305fd008703ea0005037800e4
:103f60000df8a3000400320060041400e0841c007b
:103f700060051d00e0851d006022b8007d03200063
:103f80000d38e1008006eb000b0039004433dd0002
:103f9000f300b2008301730039003700848272009d
:103fa0000d027800e10664008b85d1000a85d300fc
:103fb0008984d3000884d3008703e900f7ff3b001e
:103fc00008004000898048000a0149008b814900af
:103fd00004003b0060001000e08018006001190040
:103fe000e08119000358a300090032008d8272009d
:103ff00084827200610260008301d1000281d300db
:104000008180d3000080d3000603e8001b00370046
:104010000348a30017003a000600e0001700340030
:104020000603e9000d00a30000004800818048005d
:1040300002014900838149000348a3000f003a00b0
:104040000600e000090034000603e900000040001b
:1040500081804800020149008381490001003a0043
:104060000003eb000348a300f5ff32006022b80014
:104070000200370084827200618266001903070023
:1040800003f0a1000cf0a70003f0a000100337001c
:10409000640147006408e10002003a000df8a30043
:1040a00008033a003200be001201be0008033700c8
:1040b0001400fa00889fbe008a9fbe008c9fbe003d
:1040c0000005be000206be00680047000c90be005e
:1040d0000a90be002f0307006400e1001a003200be
:1040e00016003e006100e1001a0032006e049000ec
:1040f000fe0490000e0b90009e0b90006011b80023
:104100009e0590000b38b100d5012000828171001e
:10411000610164008703d1000683d3008984d30042
:104120000884d3008502e900f8ff3a004003070045
:104130000df0a70001f0a000e5023700f1ff270015
:10414000f0ff2f00e202370001f8270000002000f6
:10415000f7ff37006000b800f5ff370003f0a2005a
:10416000889fbe008a9fbe008c1f78005603070000
:104170005d0333006450e1004f0032006420e10031
:104180005200320003826c0007003b000905d0009a
:104190000306d000820f54000c065d0002003900b7
:1041a00002003200890178000306780085825500fc
:1041b00004003d000003fd008103fd008502ea00cc
:1041c0008b854200840f720002003b0060001000eb
:1041d000e08018006011b8000005eb007a28e100cb
:1041e0000a00390006007800c75ddd00f707b2005d
:1041f000878075002d003700828171000a017800e8
:10420000610560008180d1000080d3008502e90053
:10421000f9ff3b00060440008784480002003b0091
:1042200060041400e0841c000988a3000700320029
:104230008a81710082817100610164008904d1006a
:104240000884d3008b05e800170037000978a30025
:1042500013003a000b00e000130034008b05e90066
:104260000804440089844c000a4474000978a300bf
:104270000d003a000b00e000070034008b05e90058
:104280000804440089844c0001003a000b0020001f
:104290000978a300f7ff32000001eb0002003700ad
:1042a000828171000a017800e10207000cf0a7008a
:1042b00001f0a000150337006420e10002003a007d
:1042c000838f6c00150333000801be000200be009e
:1042d0000e033700889fbe008a9fbe00010578004c
:1042e0000100e0000400350008003c000000e00090
:1042f000200032000500370060001000e080180048
:1043000002003b0001f02c001a0037000004be0040
:104310006011b8006b0920000982cf00020039004b
:104320000882cf000441b000694252000e00320002
:1043300008003b0082817100610164008904d100a2
:104340000884d3008b05e8000442e800f9ff3a0036
:10435000050037000804440089844c008b05e900ff
:104360000442e900fbff3a00b10207000af0a7008f
:1043700001f0a0004f05be004f04be000000060083
:104380002800fa00889fbe008a9fbe008c9fbe0056
:1043900003866b003a0207000028a30064003a007d
:1043a0000128a30067003a000008a30062003a0059
:1043b0000108a30065003a001e009000be089000ae
:1043c00081064000ed3fb100f4805700ee019000ff
:1043d000111ab8008e099000311bb8009e09900098
:1043e000311cb800511db800f48557004600070085
:1043f000fe0190003a0007008b85e8003e000700b0
:104400008e09900040000700ee0190003400070084
:104410008b85e800380007008e09900040000700f7
:104420009e0990001b18b800890440000a854800c6
:10443000fe019000340007008b85e800380007007b
:10444000ee019000300007008e0990001b18b800a4
:10445000890440000a8548000a98a30008003a0031
:104460000402420085824a0006034b0087834b000a
:1044700008044c0089844c000a054d008d06e900b3
:1044800084827200850273004c3add00850272005e
:104490000100320015002000443ade001400b20092
:1044a0004538de00cb45dd000b007000c540de0066
:1044b000cb4ddd008b8070004549de00cb55dd0023
:1044c0000b017100c551de000d03780005020700e5
:1044d00003f0a1000cf0a70003f0a000fc013700de
:1044e0001b18b8008502400006834800e0834b009b
:1044f00060044c00070037001b18b800060340009a
:1045000087834800faff37001b18b8008703400074
:1045100008844800e0844c0060054d00000006005f
:104520001b18b8000804400089844800faff3700cf
:104530000108a300e3013a005800be005801be0084
:10454000e3ff37000008a300de013a000904780009
:10455000f9ff37000002eb0073023700889fbe00ae
:104560008a9fbe008c1f7800570207005e0233004e
:1045700003866c006450e100240032006420e100f6
:10458000270032006150e100220032006120e1008a
:10459000210032008b854200eb07b1000134b800e6
:1045a000003ab8000804420089844a00013ab80081
:1045b0000030b8008880400009014a000400330040
:1045c0000000400081804800020149008b05e9009d
:1045d000c909dd00830170000100320013002000d2
:1045e000c814de004814dd004709de001200b200e6
:1045f000c808de00088470000d02070001f0a10069
:104600000cf0a70001f0a000400237006120e1009b
:10461000420232000801be000200be00f7ff370070
:104620006150e100fcff3a003c0237001400fa0040
:10463000889fbe008a9fbe008c9fbe000004be0003
:104640000205be00680047000a90be000890be0048
:10465000d00107000078a3003d003a006100e100ae
:104660003c0032000bf8a3003d003a006400e1007a
:10467000380032006c0347001e009000f03fb1008c
:104680003602be001603be000008a300040032007c
:104690000402420085824a0006034b0087834b00d8
:1046a000100798008e1f78006000b8006011b800f5
:1046b0005c0020006d0120006e0020000200370029
:1046c0008d86e900fc0020000402420085824a0039
:1046d00006034b0087834b000004400081844800a0
:1046e00002054900838549006060e1001d60ad005e
:1046f0000804520089845a000a055b008b855b0020
:10470000030039001e60ad000802be000a03be00af
:104710000c06e900ecff3b000e87e900e8ff3b00d8
:104720004f07780061026000840278008301d100a5
:104730000281d3008180d3000080d3001e0390004b
:1047400041b3de00f63fb0006601070060013700ac
:104750000b30a0000800be000a01be005c0137005b
:1047600012022000f2ab8800560137000000fa0068
:10477000889fbe008a9fbe008c9fbe000404be00be
:104780000605be0095020700040678000c78a30019
:1047900020003a000800fd008900fd000a01fd002c
:1047a0008b01fd008d020700840678000d78a300c0
:1047b00018003a000d0666006460e100190032003e
:1047c0006160e100170032000002be000203be007b
:1047d0000a01be000800be00070478005dfd070066
:1047e00003f0a1008f02070008f0a60006003700c2
:1047f00003f0a20097002400b61f220045442500c4
:1048000084d12200adfd07000bf0a70003f0a20049
:104810002f01370018022000f8ab88000330a000f9
:104820002b01370018022000f8ab88002501370063
:1048300007f0a200a1fd37004f89de008201780059
:104840002e0337001400fa00889fbe008a9fbe0026
:104850008c9fbe000004be000205be006800470039
:104860000a90be000890be004a0107000070a70031
:104870000bf0a1000bf8a30016003a009e02900076
:104880003043200080825200b0fe2f000028e1005b
:104890000d003c00b0fc2f000028e1000d003400aa
:1048a0001e0990008e0890007e0090000501b00067
:1048b0000201d1008180d3000080d3008502e8008e
:1048c000fbff3a0002013700010028000000200031
:1048d000ff0037006000b800fd0037006022b8001c
:1048e000060220000000d0008180d2000482d200a5
:1048f0008582d2000000a0000202520083825a008a
:1049000003003b000202420083824a000000a10033
:104910000603e900f3ff3a0000000600efff07007e
:104920000400be00000006001400fa00889fbe00cc
:104930008a9fbe008c9fbe000004be000205be0020
:10494000680047000a90be000890be0011010700f1
:104950000070a7000bf0a100304320009e029000e1
:1049600080825200b0fe2f000028e10011003d00bf
:10497000b0fc2f000028e100150034001e09900053
:104980008e0890007e0090000501b0000201d10069
:104990008180d3000080d3008502e800fbff3a004d
:1049a0000b00e000ca003b0060001000e08018002f
:1049b000c7003700f0ff2f00f1ff27000b00e000d9
:1049c000c3003b000100280000002000c0003700a9
:1049d0006000b800be00370014002000fe0237005f
:1049e000889fbe008a9fbe008c1f7800360107009a
:1049f0003d01330003866c006450e1002e0032005c
:104a00006420e100330032006150e1002f003200e9
:104a10006120e1003100320085855500eb07b000d0
:104a200009002000080420000500370008044400a5
:104a300089844c000a0031000603430087834b0041
:104a40000001530081815b00f8ff33000203be00c8
:104a50000800a0000804440089844c00f6ff3900d7
:104a6000c639dd008301730001003200130020000d
:104a70008904d1000884d3000998a30005003200fe
:104a80000800a7000300a0008904d1000884d30017
:104a90008b05e8008904d1000884d3000001eb00f5
:104aa0000281d200e200070001f0a1000cf0a70093
:104ab00001f0a000150137006420e1001701320069
:104ac0000801be000200be00f7ff37006120e100d0
:104ad000120132006000b800f3ff37000000200030
:104ae00001f82700f0ff3700f4ff2f00ba0237006b
:104af000801feb00390007008f87e9000000e0000d
:104b0000000006000001be001f0007000470a7009f
:104b100003f0a1006509b100160032000d00350058
:104b20006828e10006003500f0ff2f00f1ff2700a4
:104b30000300e00013003b00010028000000050016
:104b400000004000818048008502e900fcff3a0037
:104b500008003700f88f420002003c008000eb00a4
:104b6000000005008100d1000080d3008502e8002c
:104b7000fcff3a000300e00002003b006000100070
:104b8000e080180000000600c70ade00f107b2004e
:104b9000f50fb20008003200e1cf420002003200ff
:104ba0000170a00024000500810f70000100320098
:104bb0000408050044000500810f700002003a005f
:104bc000140005008502e9000000400081c0480093
:104bd000fcff3b000170a00024000500889fbe0080
:104be0008a9fbe008c9fbe000404be000605be0066
:104bf000809fbe00829fbe007801070004067800f7
:104c00000800be000a01be00740107008406780097
:104c10004f03be004f02be008d4f76007fb097005d
:104c200013003300f0ff2f008b8f6b0006003b005a
:104c30000d0666000c00a7000a00370007f0a6006a
:104c4000100020000a003700880f5200898f5a0098
:104c50008a0f5b008b8f5b0003003900100020007f
:104c600001003e000000200007f0a7000000ea005d
:104c70004f06be004f05be004f04be0000000600f8
:104c8000680447000294be000094be00fc04470084
:104c90008694be008494be00090078003d000700a1
:104ca000080078003b00070099007800814f7000f1
:104cb0000b003b000800be00620207004f00b1007d
:104cc00003003700f3ff2700f2ff2f006110b90047
:104cd0004f06be004f05be004f04be000080fa0024
:104ce00000000600180020005700200008045300b0
:104cf0000d003d000600200097fc2f000740e1005a
:104d00001e00340084827200610260008301d100c1
:104d10000281d3008180d3000080d3000804e80022
:104d2000f8ff3a00470020006104600005047400a9
:104d3000040464000d00320061004000e08048007f
:104d400060014900e081490003b8a5000700320076
:104d50000603e8006538e10004003a008301d10051
:104d60000281d3008180d3000080d300f87f20002f
:104d70000830e10003003500080378006000b80047
:104d80006011b8004433dd00f300b200830173000a
:104d900000000600800078005002be005003be00f4
:104da0004439de00f700b200f37f20000301610008
:104db000090032000218e10016003a008501720075
:104dc00083017300838173000008200015003a00fe
:104dd000400020001300370085017200830173003a
:104de0008381730005003a0004a8be0006a8be0037
:104df000100020000b0037000201e900040242000d
:104e000085824a0006034b0087834b000748a300b6
:104e1000f9ff32000740a00004a8be0006a8be00ab
:104e200020002000800098009200980000000600fa
:104e300081002000618055000b003d000b00200028
:104e400061fe2f000100e1001d003400828171002d
:104e5000610164008904d1000884d3000000e800e7
:104e6000faff3a0071002000610064000300700046
:104e7000020060000900320061044400e0844c003c
:104e80000988a500050032008b05e8006808e100ec
:104e900002003a008904d1000884d300f20f2000f8
:104ea0000258e10005003d00c75ddd00f907b200d2
:104eb0008980750008007800000006000bf82700c4
:104ec0008b007800000005000004be002eff0700e4
:104ed0000003be000405be000200be002aff07005a
:104ee000844f7500000006000200be006450e1001f
:104ef000050036006420e100020036000968a300c6
:104f000001003a000800be000160a0004f067800d2
:104f10004f05be004f04be0000000600f0ff2f004a
:104f2000f1ff2700f9ff37000800fa00889fbe0054
:104f30008a9fbe008c9fbe00040678000004be005d
:104f40000205be00a50007006420e1009f003e00ae
:104f50009b0032006120e1009600320003f0a100c6
:104f6000171b240036582c0005a021000400200047
:104f70006efb07000800be000a01be0007003500f6
:104f800097012400b61f22004544250084d1220049
:104f9000ba0107000004be000205be008006eb0057
:104fa0000c00a700cf1ede0003f0a1000bf0a10053
:104fb00047fd230006f3250095dc260034882c00ed
:104fc000effc07006022b8000003eb0007fe23009f
:104fd0000c00a60007ff2300b8fb070052fe0700e5
:104fe0000000a7000d00a20013fe07000c00e00067
:104ff00004003a0007fe2300060020006022b800eb
:105000000bfe070003f0a200009fbe000297be0047
:1050100097002400060022006022b800d8fc070098
:105020000802be000a03be00a4fb0700809fbe006a
:10503000829fbe003e00be002e01be00f7f423009a
:1050400046542b00152d2400a4462800ccfc070054
:105050004f03be004f02be0098fb07000004be00d5
:105060000205be0003f0a10067e42300e6092a0060
:10507000f5672600d4bc23002cfb07000800be0007
:105080000a01be00480035000002be000203be0057
:10509000bbfc0700009fbe000297be0087ce230026
:1050a000f60f28003599260054f92d00b4fc0700ae
:1050b000a7d62b0006422e0085c02d00c4992400df
:1050c0007efb07003e02be002e03be00acfc0700c4
:1050d00067de2300c6232100a586260004432d0099
:1050e00076fb07003e02be002e03be00a4fc0700b4
:1050f000a7e52b0056642e00d5b52400b40a2c0079
:105100006efb07003e02be002e03be009cfc0700a3
:1051100077ec230036de210045522a0034062f00aa
:1051200066fb07003e02be002e03be0094fc070093
:10513000a7f22b00061a200015a02100a4e12300ed
:105140005efb07003e02be002e03be008cfc070083
:1051500017f823001611210015112100040b21005e
:1051600056fb07003e02be002e03be0084fc070073
:1051700057fc2b0056552500555525005455250044
:105180004efb07003e02be002e03be007cfc070063
:105190000802be000a03be0079fc07000802be0038
:1051a0000a03be0045fb07000d00a70003f0a200a4
:1051b000c7fe37000c00a60003ff2300c4fe370023
:1051c000f3ff2700f2ff2f006110b9000330a000a9
:1051d00014022000f4ab8800bdfe370005ff270055
:1051e00005826100070032000428e100010032005e
:1051f000240005000600070001003a0044000500f5
:105200000408050002000700f9ff3a001400050039
:105210006f82610081027000850271008502720058
:10522000000006000800fa00889fbe008a9fbe00aa
:105230008c9fbe000004be000205be0083067800fd
:10524000e6ff07006420e100a3003e00a600320054
:105250000006eb000bf0a10003ff2300020020007a
:105260006000b8000802be000a03be00b4fa0700de
:1052700009003d0003ff2300020020006000b80089
:105280000802be000a03be00b2fa07000004be0016
:105290000205be002c00200013fd23004261220005
:1052a000e1e9250060d52c000802be000a03be001b
:1052b000a3fa07001d003d00b3ff2300a2672b00e7
:1052c00081852e00a0ca24000802be000a03be0089
:1052d000fafa0700009fbe000297be0073fe23008b
:1052e00052cf2600010b2d00509529000802be0068
:1052f0000a03be0022fc070007ff2300060020006f
:105300006022b8004afd07000802be000a03be0082
:10531000eafa07003e02be002e03be008dfa070027
:105320000004be000205be000c06e8000800be0036
:105330000a01be0003f0a10067e42300e6092a0089
:10534000f5672600d4bc230078fa07000800be00e9
:105350000a01be004c0035000802be000a03be0070
:1053600007fc0700009fbe000297be00e702240072
:1053700096c42000a5142e0004712c00cffa07005b
:105380003e02be002e03be00fdfb0700d704240032
:10539000a6a02c00d5202300743d2a00c7fa0700e0
:1053a0003e02be002e03be00f5fb07005705240099
:1053b00026a12800b540200054da2600bffa0700d5
:1053c0003e02be002e03be00edfb07004704240092
:1053d000c687280045cc2b00945a2900b7fa07004d
:1053e000809fbe00829fbe003e00be002e01be0018
:1053f000a7fe2b00a6d72c00159b2d00d47b2800e0
:10540000dffb070007022c00f6d32f00d5c82500cc
:1054100034a62600a9fa07003e02be002e03be00f5
:10542000d7fb070047032c00f6172800259e2b000a
:10543000b4cc2b00a1fa07003e02be002e03be0032
:10544000cffb0700b7022c00660a26006510250076
:1054500024ce210099fa07003e02be002e03be00b2
:10546000c7fb07004f03be004f02be0039fa07001a
:105470000802be000a03be00c1fb07000802be000e
:105480000a03be008dfa07000c00e0000f00320096
:105490000c10a70003f0a20084d12200454425008f
:1054a000b61f220097ff23006260e1000600320071
:1054b00064362700d582230026152c0007fe230022
:1054c0000c10a70007ff23007cfa07000df0a700cf
:1054d00003f0a200fefd37000330a00014022000fc
:1054e000f4ab8800fafd370093ff2300b21f2200bf
:1054f0004144250080d12200f4ff3700889fbe0080
:10550000830478000300e0002c00350003003c0019
:105510000082700004027100260032003643200031
:10552000c50020008383cf000a0039000541b10087
:105530008283cf00070039000541b1008183cf008d
:10554000040039000541b1008083cf00010039001b
:105550000541b10085c353006022b800120032003b
:105560000a003b0084827200610260008301d10066
:105570000281d3008180d3000080d3000603e800bd
:105580008743e800f7ff3a000700370000004000bb
:105590008180480002014900838149000603e90037
:1055a0008743e900f9ff3a00cefd070009f0a700a4
:1055b00003f0a0004f04be000000060060001000d1
:1055c000e080180060011900e0811900d3ff3b0062
:1055d000033e2c00f7ff3700889fbe008a9fbe0065
:1055e000841f780038fe07004f0078001100330058
:1055f000f0ff2f00838f6c0006003b000405650060
:105600000a00a7000800370009f0a60010002000db
:1056100008003700820f5400838f5c0003003900bc
:105620001000200001003e000000200009f0a7004b
:105630000000ea004f05be004f04be000000e0007d
:1056400000000600e48240001078a300070032004a
:10565000640240001178a3003400be001401be00b3
:10566000040032000330a700000006003500be0031
:105670001501be000330a00000000600801feb00f3
:10568000020007008f87e900000006002800fa00ea
:10569000889fbe008a9fbe008c9fbe000efe9700b2
:1056a00077fd07006108e1005c0032006200e10064
:1056b0005a003e00540039006408e10052003200f4
:1056c0006c014700748557003200be001201be0015
:1056d0003a04be001a05be009e029000be0e900065
:1056e0000d82520017003b000402e80046003a0019
:1056f000880f5000898f58008a0f59008b8f5900ee
:105700004100340064014700780347003200be00c6
:105710001201be003602be001603be0007f0a10053
:1057200003f0a60007f0a0000c70a700e3f9070043
:1057300067fd3700000040008180480002014900f9
:10574000838149000c00a0000800500089805800a7
:105750000a0159008b81590005003b0008004000f8
:10576000898048000a0149008b8149000c00a10092
:105770000402e900efff3b00000240008182480084
:1057800002034900838349001b00320008025200d3
:1057900089825a000a035b008b835b004200f80099
:1057a00005003700000040008180480002014900e8
:1057b000838149008d06e9000340a600f9ff370008
:1057c0006022b8000d03780046fd0700780347000b
:1057d0004200f9000800350002003c000c08a3005c
:1057e000050032003602be001603be0007f0a0001e
:1057f0000c70a700b1f907005e02900004f0a7004a
:1058000003f0a20032fd37002e009000be00900091
:105810004e019000de0190002dfd370010022000a7
:105820000c70a600f0ab880026fd3700020ab90014
:10583000001bb9000200b800810042008100430053
:1058400000000600839f68000100e00002003d00a8
:1058500060001000e08018000300e00002003d003e
:1058600060011100e08119001cfc07004f00e000fe
:1058700002003b0060001000e080180000000600fd
:1058800060001000e080180060011900e08119003c
:1058900000000600881f7800000478005001be0058
:1058a0004000be000000420081804a0002014b001f
:1058b00083814b00009cbe000294be00dc00070008
:1058c00003003100480090000000e8004004980008
:1058d0004f04780000000600889fbe000004780096
:1058e0008004eb005001be004000be00d000070065
:1058f000010031001900200004005000858058008c
:105900000601590087815900009cbe000294be0028
:105910004800900009005000400498004f04be0069
:10592000000006001200fa00889fbe008a9fbe0099
:105930008c1f78000205be000004be00f4b79f0073
:1059400085bf9f0096bf9f00a7bf9f000000eb0090
:10595000e0b79f00d0b79f00c0b79f00b0b79f00cf
:10596000a0b79f000006eb005fb197006fb09700f3
:105970008000d0000000e00015003d00e1b79f006e
:10598000010078000200e00001003d000000a000de
:10599000ac00070001003d000000a000af000700c0
:1059a00001003d000000a000b200070001003d0022
:1059b0000000a0008100070001003d000000a000e1
:1059c000b20007007c805700b2ff070014003700c8
:1059d000e1b79f00010078000200e00001003d00f7
:1059e0000000a0009700070001003d000000a0009b
:1059f0009a00070001003d000000a0009d00070084
:105a000001003d000000a0006c00070001003d0007
:105a10000000a0009d0007007c805700aeff07003b
:105a20006fb097000000e000070035001000200074
:105a3000010020006011b800080470008984700023
:105a40000a0571008b8571000c06e800f003200048
:105a5000800f5600c4ff34006fb097000000e000d4
:105a600006003d007fb297008fba97001fbb9700da
:105a7000afbb97007c80570086ff07000802be007e
:105a80000a03be006fa897000000e00004003a007f
:105a90002fb29700bfb297004fb39700dfb39700c4
:105aa0000400be000601be004f0678004f05be0090
:105ab0004f04be000080fa0000000600881f780036
:105ac00018002000881f780096ff07008f87e900e4
:105ad0004f04780000000600801feb0091ff0700d4
:105ae0008f87e900000006000800fa00889fbe00ca
:105af0008a9fbe008c1f78006e00070005003d00e5
:105b000043000700300007000c003d003300070091
:105b10000b003700e00f5200e08f5a00e00f5b00ef
:105b2000e08f5b0006003d000400be000601be00e1
:105b300053ff07000205be000004be001c00200049
:105b40002c000700ddff07000c00e0000100320020
:105b50004bff07004f0678004f05be004f04be0004
:105b60000080fa00000006000800fa00889fbe00ce
:105b70008a9fbe008c1f78004e00070002003d0087
:105b80001c002000220007000f00070001003d005c
:105b90001200070017000700cfff07000c00e0000d
:105ba0000100320036ff07004f0678004f05be00a7
:105bb0004f04be000080fa000000060090b79f006e
:105bc0000100d00080b79f00e00f5400e08f5c0020
:105bd000e00f5d00e08f5d00000006000800be00e1
:105be0000a01be0026ff07000205be000004be0039
:105bf000000006000802be000a03be005fb0970066
:105c0000efb097007fb197008fb9970000000600b2
:105c10001bff07000100070000000600b0b79f004f
:105c2000c1b79f00d2b79f00e3b79f0000000600f6
:105c30000400e1000588e1000690e1000798e1001a
:105c400000000600c0b79f000200d000b0b79f0060
:105c5000afb097000100e00000000600b0b79f0061
:105c60000100d000a0b79f009fb097000100e000a6
:105c700000000600a0b79f000100d00090b79f0071
:105c80008fb097000100e0000000060080b79f0081
:105c90000804d0008984d2000a85d2008b85d20006
:105ca0005fb29700efb297007fb397008fbb97006a
:105cb00000000600d9ff07000605be000404be0070
:105cc0000006eb00e00f5000e08f5800e00f590095
:105cd000e08f590000000600889fbe008a9fbe002a
:105ce0008c9fbe000404b8000506b8008904460075
:105cf00060854e000606b8000a054600e0854e00a5
:105d00000706b8008b054600040eb800890446005b
:105d10000a854e00050eb8000a0546008b854e0028
:105d2000060eb8008b0546000416b8000a054600aa
:105d30008b854e000516b8008b054600041eb80082
:105d40008b0546000800be000a01be004f06be00db
:105d50004f05be004f04be00000006000800fa0018
:105d6000889fbe008a9fbe00170007000605be0080
:105d70000404be00e00f5200e08f5a00e00f5b0009
:105d8000e08f5b0008003d000400be000601be007d
:105d9000bbfe07000205be000004be000f000700a6
:105da000b7fe0700080007000802be000a03be0095
:105db0000a000700c8ff07004f05be004f04be00e1
:105dc0000080fa0000000600e0b79f00f1b79f00d6
:105dd00082bf9f0093bf9f00000006006fb0970036
:105de000ffb097000fb997009fb997000000060019
:105df000ef02b000889fbe008a9fbe008c9fbe004d
:105e00008e1f7800000478000000e00003003200dc
:105e1000104078000004e00011003a00881f78006c
:105e200040dc2800801f780010072000fc7c020066
:105e3000000000000003eb00e50420001407200030
:105e40005305200072df2800c102200000e0280076
:105e5000967c020000000000e4875700184078009c
:105e60008000eb00d1af9f008005eb006066b800ba
:105e70000005eb000007eb00880478000004e00058
:105e80001300320098407800d0c2b30080cf500099
:105e900096023200a0c3b30080cf500091023200be
:105ea000e0c2b30080cf50008c0232000100fb0042
:105eb00088010200000000000000e0000100320044
:105ec0008b05e800d94078000104e000eeff3a00bd
:105ed000e10f55007c023c000c00e000340232006f
:105ee000e20f56002e023a00e18f560028023c00d5
:105ef0000b00e00022023a006055b8008ab79f000c
:105f00009bb79f00eaaf9f00fbaf9f008000eb00b4
:105f1000c1b79f00b1b79f00a1b79f0008027800ea
:105f200088047800184078000004e0000e00320079
:105f3000ea4f50000c0032000c00e0000201320079
:105f4000a0c3b300994f1000cf0032008900e800d1
:105f500081047800114078000004e0000200320063
:105f6000ea4f5000f4ff3a00890f5200bb003a009c
:105f70000a00be00581e020000000000d0b79f00bb
:105f8000e1b79f00f2b79f0083bf9f006022b80077
:105f900006002000e7042c00961e0200000000000e
:105fa0000000e0000b0034006022b8000600200072
:105fb000e70424005fb09700efb097007fb197002f
:105fc0008fb99700a01e0200000000000000e00052
:105fd000140035005fb09700efb097007fb19700d5
:105fe0008fb99700809fbe00829fbe0081e028008d
:105ff000811f780030082000fc7c020000000000b7
:10600000f0ff2f00f1f72700ea8757004f077800cd
:106010004f06be004f05be004f04be00ef02b100a8
:10602000000006000fb097009fb09700581e0200b6
:10603000000000000004be000205be006022b8009f
:1060400006002000e7042c00961e0200000000005d
:106050000000e000090034006022b80006002000c3
:10606000e70424000800be000a01be00a01e0200d2
:10607000000000000000e00006003500889fbe0020
:106080008a9fbe00a2e42800821f780040082000fa
:10609000d9ff3700dfa997000300e00005003200b8
:1060a0006fa89700ffa8970001f0a200e0af9f0043
:1060b000f1af9f006fa89700ffa89700581e02003d
:1060c000000000006022b8006033b800961e020095
:1060d000000000000000e00040003d006022b80029
:1060e00006002000e70424000800be000a01be00ec
:1060f000aa1e0200000000000004be000205be004f
:106100006022b80006002200c70a24005fb0970092
:10611000efb097007fb197008fb99700aa1e0200d9
:10612000000000000002be000203be000800be0026
:106130000a01be005e1f020000000000582002009d
:10614000000000000001be006fa89700ffa89700a4
:10615000ae20020000000000e0af9f00f1af9f0002
:106160006fa89700ffa89700581e020000000000cb
:106170000004be000205be006022b8000600280030
:1061800067072c00961e0200000000000000e000df
:10619000090035006022b8000600280067072400c7
:1061a0000800be000a01be00a01e020000000000a0
:1061b0000000e00006003400889fbe008a9fbe00f9
:1061c000c1e82800811f7800500820008aff3700ae
:1061d0006fa89700ffa897008cff37006022b800d7
:1061e00006002000e70424000800be000a01be00eb
:1061f000aa1e0200000000000004be000205be004e
:106200006022b80006002200c70a24005fb0970091
:10621000efb097007fb197008fb99700aa1e0200d8
:10622000000000000002be000203be000800be0025
:106230000a01be005e1f020000000000582002009c
:10624000000000000001be006fa89700ffa89700a3
:10625000b020020000000000bfff3700891f780057
:10626000841f7800a2eb2800821f780020082000fd
:10627000fc7c020000000000f0ff2f00f1f7270077
:10628000e687570061ff3700e20f56000e003a0024
:10629000a20020008000eb00040078009c010200b6
:1062a00000000000cf80de006a2102000000000034
:1062b000e0af9f00f1af9f000902e8008400780082
:1062c0001c00200022ff3700e10f560015003a00a5
:1062d000a20020008000eb00040078009c01020076
:1062e00000000000cf80de006a21020000000000f4
:1062f00080b79f0091b79f000902e8006011b800c5
:106300008000eb0004007800c202020000000000e0
:1063100058200200000000000005be0009027800bd
:1063200011ff370062ef2800821f7800b0072000bd
:10633000fc7c020000000000f0ff2f00f1f72700b6
:106340008f87e90031ff37000e00e000e3003200e4
:10635000194178000200fb00cf80de006900500088
:10636000e0805800e3062000830f5000e08f5800c3
:10637000ce003e0000600100f4fe3700cb00370085
:10638000ca003700c9003700c8003700c70037000f
:10639000c6003700c5003700c4003700c30037000f
:1063a000c2003700c1003700c0003700bf0037000f
:1063b000be003700bd003700bc003700bb0037000f
:1063c000ba003700b9003700b8003700b70037000f
:1063d000b6003700ddfe3700b4003700b3003700e9
:1063e000b2003700b1003700b0003700af0037000f
:1063f000ae003700ad003700ac003700ab0037000f
:10640000d2fe3700a9003700d0fe3700cffe37009c
:10641000a6003700a5003700a4003700a30037000e
:10642000a2003700a1003700a00037009f0037000e
:106430009e0037009d0037009c0037009b0037000e
:106440009a0037009900370098003700970037000e
:10645000960037009500370094003700930037000e
:10646000370037004f003700320037008f00370009
:106470008e0037008d0037008c0037008b0037000e
:106480008a003700890037006d0037002900370087
:10649000860037008500370084003700830037000e
:1064a0002400370081003700800037007f0037006c
:1064b000200037007d0037007c0037007b0037006c
:1064c0007a0037007900370078003700770037000e
:1064d000760037007500370074003700730037000e
:1064e000170037002f003700120037006f00370009
:1064f0006e0037006d0037006c0037006b0037000e
:106500006a003700690037004d0037000900370086
:10651000660037006500370064003700630037000d
:106520000400370061003700600037005f0037006b
:10653000000037000902e8008400780084fe37007c
:10654000cfb097000100e0000d003a006011b800e4
:106550008000eb0004007800c2020200000000008e
:1065600058200200000000000005be000902e800fb
:106570008400780012002000c2b79f0074fe37002c
:106580000a00be00581e020000000000809fbe00ee
:10659000829fbe00e0f12800801f7800e007200005
:1065a00095fe37002fb097000000e0001a003a0077
:1065b00004845400080178008400780060fc2f00f7
:1065c0000f004000440402000000000061fc2f00a6
:1065d0008f80400001044400004ceb006011b800c3
:1065e0008000eb0060fc2f000f004000c2020200a0
:1065f000000000005820020000000000e0af9f00f3
:10660000f1af9f000902e80084007800120020002a
:10661000a2b79f004efe37006fa89700ffa8970013
:10662000581e020000000000809fbe00829fbe0036
:1066300062f52800821f7800c00720006efe370038
:10664000bfb197000300e0000e003a006011b800ef
:106650008000eb0004007800c2020200000000008d
:10666000582002000000000080b79f0091b79f00f3
:106670000902e8008400780010002000b0b79f00f5
:1066800033fe37000fb097009fb09700581e0200ee
:1066900000000000809fbe00829fbe00e3f828003b
:1066a000831f7800d007200053fe370000cdb300d1
:1066b000004041008900e800e94f500024fe360008
:1066c0000200fb00801f7800801f780063fc280018
:1066d000831f7800f0072000e5fe37000d00e00082
:1066e00023003200e0c2b300994f100017fe3a00b9
:1066f000e28f56000e003a00a20020008000eb005e
:10670000040078009c01020000000000cf80de0041
:106710006a21020000000000e0af9f00f1af9f007f
:106720000902e800840078001d00200008fe370000
:10673000e18f56000a003a006011b8008000eb00bb
:1067400004007800c202020000000000582002008d
:106750000000000080b79f0091b79f00effe370058
:10676000e0ff2800801f780000082000f0fe3700be
:1067700071022900811f780010082000ecfe37000c
:10678000d1052900811f780050072000e8fe37005e
:10679000700a2900801f780040072000e4fe3700bf
:1067a000d30e2900831f780030072000e0fe370059
:1067b0000b00e0000c003a000d00e0000600320083
:1067c000e28f5600ccfd320053132900831f78005e
:1067d00070072000d6fe3700a21b2900821f780018
:1067e00060072000d2fe3700512029000800780001
:1067f00064040200000000000000e0002e003200ef
:10680000c120290008007800640402000000000094
:106810008004780011212900080078006404020037
:1068200000000000d0af9f000a00e000140032001a
:106830000900e00002003a000000e0001000320011
:106840000900e0000b0032001900fb00801f7800f7
:1068500063212900831f780090072000fc7c020040
:1068600000000000f0ff2f00f1f72700e487570039
:10687000e6fd37005fa997001200fb00f3ff370029
:106880000900e000020032000000e00002003a00cf
:106890001e00200098fd37001000fb00801f7800cc
:1068a0001900fb00801f7800d0262900801f780087
:1068b000a00720006efe3700e02b2900801f780023
:1068c000800720009afe37008a1f78007234290062
:1068d000821f780020072000e0ff37008d06e800c7
:1068e00078fd37000c06e80076fd37000a05e80061
:1068f00074fd37004f05b000889fbe008a9fbe0020
:106900008c9fbe008e1f78000004be000206780037
:106910000305780084057800a15621009140780095
:1069200070c4b30080cf500095003200a156210002
:10693000914078006340500080cf500090003200ba
:106940000102200010002000984b0200000000000f
:106950000000e0008a0032000a00e000cb003200b4
:106960000c00e000b90032000800e00095003a0099
:106970000900e0008a0032008a1f78008a1f780030
:106980008c1f78001904e00083003a00903e290033
:10699000801f7800891f7800a53e2900851f780098
:1069a000b67d020000000000ec87570001c2b30072
:1069b000b1c79f00c1c79f00c0c7b300d0df9f0011
:1069c000e1df9f000007eb006044b800f5fd2f00f9
:1069d000858647006f006400320032008a0f540041
:1069e0003000320024002000e78f540001003c00fa
:1069f0000002eb006348b8000000420005fa2f00d7
:106a00008f82420005004000ec407c000181fb00c9
:106a1000c411de00953d2900e3c17a003348980097
:106a20006f01610062c17a004248980002c2b3005f
:106a30005248980002c15000e0c5b300804f510099
:106a400015003e0081f67c000804e8008904e80097
:106a50008a0f5400dfff3a00f08f5400ddff320050
:106a6000708014006300b900040050000081e80049
:106a70006348b90003fa2f008f8141000080410074
:106a8000040040006b00400001022000800402006e
:106a900000000000cfff3700e0c2b30080f67c00aa
:106aa000e9ff37000800e00012003400a0c0b30086
:106ab00080f67c0001fe2f000180470009004000a5
:106ac0000048eb0000fa2f000f0040008e04020087
:106ad000000000000001780001fa2f008f804000c4
:106ae0001000200080430200000000000e07e800b4
:106af0008004eb008a0f5400210031000b00e000fd
:106b00000f003200110009000b87d8008000fd0043
:106b10000000e0000a003a000800e0001200320025
:106b2000703829008e040200000000000001780087
:106b3000713829001000200080430200000000008e
:106b4000881f7800881f7800c3412900831f7800c0
:106b5000a0f92f000f0040006006020000000000b6
:106b6000e68757009fff3700803829008e04020017
:106b7000000000000001780081382900edff370097
:106b80004f0778004f06be004f05be004f04be0001
:106b90004f05b10000000600704229007cff37005d
:106ba0008a1f78008a1f78008c1f7800a342290072
:106bb000831f7800b67d020000000000e8875700c0
:106bc0007aff37000808a300190032000900e0002e
:106bd0000f0032008a1f78008a1f78001904e00035
:106be00009003a00903e2900801f7800891f780034
:106bf00081452900811f7800b67d02000000000059
:106c0000ea87570069ff370070422900f6ff370016
:106c10008a1f78008a1f7800f0462900801f7800bc
:106c2000b67d020000000000e68757005fff3700d6
:106c30000818a3005dff32008a1f78008a1f7800c1
:106c4000b3482900831f7800f5ff3700e149290088
:106c5000811f7800b0082000fc7c020000000000ca
:106c60000003eb00e5042000b408200053052000d9
:106c7000b24b29006119200000e02800967c020038
:106c8000000000008f87e90037ff3700304c2900f3
:106c9000801f7800b67d0200000000008f87e900a9
:106ca000b7ff3700889fbe008a9fbe000004be0069
:106cb00082057800030578000000e00079003200ca
:106cc0000900e000670032000b00e00054003200d1
:106cd000c0ff2f000000650040003a000800780067
:106ce0008e04020000000000800178000b00e90023
:106cf000808f51002f003e00090078000a08a30091
:106d00000d0032000001eb000300e0000a00340037
:106d100004c2b3009840780084cf500002003200d3
:106d2000e9cf500005003a000201e8000804e8003d
:106d3000830f5100f7ff3500984078000001eb0009
:106d40000104e00004003200185878000201e80055
:106d50005804e000fcff3a000048eb000a18a300ca
:106d600010003200028044000000e900890f50004a
:106d70000c00390003c2b3009040780083cf50006c
:106d800004003200e9cf500002003200eacf500088
:106d900004003a000050eb000201e900890f5000a6
:106da000f5ff3100020078004f05be004f04be0021
:106db00000000600831fe8008b1f7800a04d29000b
:106dc000801f780020092000fc7c020000000000e9
:106dd0000080eb00e6875700f3ff37008a1f78003a
:106de000b0512900801f780020092000fc7c02009f
:106df000000000000003eb00d5042000240920005f
:106e000053052000325429000123200000e028000f
:106e1000967c020000000000e4875700afff3700b7
:106e2000801feb00b0542900801f7800100920005b
:106e3000fc7c0200000000000003eb006505200060
:106e4000140920005305200032542900b1222000eb
:106e500000e02800967c020000000000e487570054
:106e60009bff3700d0562900801f780000092000c2
:106e7000fc7c0200000000000003eb00e5042000a1
:106e800004092000530520003254290071222000fb
:106e900000e02800967c0200000000008f87e900d7
:106ea00089ff370010592900801f7800f008200062
:106eb000fc7c0200000000000003eb00e504200061
:106ec000f40820005305200032542900312220000c
:106ed00000e02800967c0200000000008f87e90097
:106ee00077ff3700889fbe008a1f780080047800f3
:106ef000010478000000e000610032000800e000ba
:106f00004e0034000800e0004a003200994078004a
:106f100000c2b30080cf50003d003200e9cf5000e6
:106f20003b0032001a002000d0c2b30080cf5000d6
:106f300035003200b0c2b30080cf50002f003200c5
:106f40000800e000060032001940780001c2b300da
:106f5000814f500020003200e94f50001e003200e7
:106f60006033b8000804e900e10f4400110032006a
:106f700005cdb3001942780005404200e94f5000aa
:106f80000c003e006a31b8006a38b90080814100c7
:106f90000400fb000003b100cf80de0002034000cc
:106fa000838348008904e8000804e900e10f4400f5
:106fb000f0ff3a006151b9000230b80003b2b900e5
:106fc000048240000791b900820042004f0578001a
:106fd0004f04be00000006008904e8000804e90030
:106fe000dfff320019407800814f5000faff320075
:106ff000e94f5000f8ff3200d9ff37008904e8005c
:107000000804e900ceff37000085eb00fbff3700e6
:107010008904e8000804e90006003200994078007d
:1070200080cf5000faff3200e9cf5000f8ff320065
:10703000bcff370099407800baff3700881f7800fe
:10704000515b2900811f780070082000fc7c020041
:107050000000000008037800650520007408200087
:1070600053052000425d29007129200000e028001e
:10707000967c020000000000e4875700a1ff370063
:10708000a05d2900801f780060082000fc7c0200c1
:10709000000000000003eb00e5042000640820006d
:1070a00053052000425d29003129200000e028001e
:1070b000967c0200000000008f87e9008fff3700f8
:1070c000f6874700889fbe008a9fbe008c9fbe0047
:1070d0008e1f7800d0b79f00e1b79f0002067800ae
:1070e000f3b79f00840578000400e000a50032009b
:1070f0000c00e00004003200eb0f460002003500f7
:10710000eb0f5600100034008c1f7800c15f29007f
:10711000811f780090082000fc7c02000000000025
:107120000c0378002505200094082000530520005a
:10713000926129008136200000e02800967c020040
:1071400000000000e48757008c0678000c00e00087
:107150008a0035005fb09700efb09700e00f500055
:10716000e08f58007e0035008000eb0081bf9f005b
:107170005fb49700efb497000c00e00038003500d2
:107180000d05e900090033000a00e00022003a0082
:107190000fb997000200e0001f003200d0c2b30018
:1071a000804d78000a05e900f7ff3b00e00f54002e
:1071b000e08f5c000c003a007fb197000200e00015
:1071c000020032000040eb0080f57e000b007800ea
:1071d0004f0778004f06be004f05be004f04be00ab
:1071e0006f01b100000006008c1f78004fb09700bf
:1071f000dfb09700809fbe00f1612900811f7800f9
:10720000a0082000fc7c0200000000000000eb0051
:10721000e8875700eeff3700e00f5400e08f5c0076
:1072200003003a0000c3b30080757d00ddff370026
:10723000a2002000030020000800be009c04020001
:10724000000000000203be000002be0001c3b30044
:107250000140430080757d000404be00d1ff37006b
:107260000007eb000fb9970002855600e00f1500ec
:1072700013003d00a2002000030020000800be0013
:107280009c040200000000000203be000002be00d9
:1072900001c3b30001404300e2fd2f000e01410095
:1072a00000f17f000404be00e00f5200e08f5a009e
:1072b000030032000e07e8008a0f5700edff35008b
:1072c000e00f5400e08f5c00c7ff3a000005eb00c0
:1072d0000d00e0000f003400d3c2b300e2fd2f0028
:1072e0000f0141000fba97008400410002c2b300b1
:1072f0000a00e0000d003a000fb897000000e0001f
:107300000a003200834d78000a05e8008d0f550011
:10731000f7ff3500ffb097000100e000abff32003f
:107320000040eb0080757d00a8ff37000fba970082
:10733000040055008e0f500004003c000a00570066
:107340006140780080757d00efff37007fb09700c7
:107350000000e000efff3a0082757d00eaff370091
:107360001100200081bf9f005fb09700efb0970031
:1073700060041000e08418007fff37008c06ea00ec
:1073800074ff370040652900801f780080082000c6
:10739000fc7c0200000000000003eb00e50420007c
:1073a0008408200053052000926129004136200006
:1073b00000e02800967c0200000000008f87e900b2
:1073c0004bff3700e8874700889fbe008a9fbe00ba
:1073d0008c9fbe008e1f780000077800e1b79f00e9
:1073e000f2b79f0083bf9f000404be000606be00e4
:1073f0000000e000840032006fb097000000e00061
:10740000710032000801be001fb09700afb09700b6
:10741000ae200200000000000004be007fb1970013
:107420008fb997000c00be00b020020000000000e1
:10743000581e02000000000014d12d0025252a004e
:1074400066f42d0017f82300c021020000000000a0
:10745000aa220200000000005820020000000000e4
:107460000001be000800be00ae22020000000000c5
:1074700092872100a3282400ae2202000000000011
:107480000005be007fb197008fb997000c00be00c9
:10749000ae2002000000000092872100a3282400f3
:1074a000ae220200000000000006be000a01be007d
:1074b0000a00be00ae220200000000000004be0070
:1074c0000c01be000c00be00ae2202000000000055
:1074d0000001be000800be00b02002000000000055
:1074e000581e0200000000001623020000000000e9
:1074f0005820020000000000008fbe000a00be00fd
:10750000581e0200000000000004be000205be007c
:107510000c00be00581e0200000000000802be0061
:107520000a03be00b623020000000000b47c26005f
:1075300095e72100c65d2a00c7042400c02102008f
:10754000000000000002be000203be006000b800a0
:107550000200280063052400182402000000000037
:1075600058200200000000000004be00581e020067
:10757000000000006022b8006033b800961e0200d0
:10758000000000000000e00006003d0002002000b6
:10759000433b24000800be00b020020000000000b1
:1075a0000004be006fb097000888be000000eb002a
:1075b0004f0778004f06be004f05be004f04be00c7
:1075c0008f00b1000000060010672900801f7800be
:1075d000e0082000fc7c0200000000000003eb003b
:1075e000e5042000e408200053052000c2692900ba
:1075f0001115200000e02800967c02000000000029
:107600008f87e9007fff3700a06a2900801f78007c
:10761000d0082000fc7c0200000000000003eb000a
:10762000e5042000d408200053052000c269290089
:10763000d114200000e02800967c02000000000029
:107640008f87e9006cff3700e4874700889fbe0002
:107650008a9fbe008c9fbe008e1f780000067800b7
:10766000810578000205e9000200e00007003a0009
:107670000000eb004f0778004f06be004f05be002c
:107680004f04be004f00b100000006009c46780089
:107690001b84fb000d80fb0080bf9f00ca0402001a
:1076a00000000000800478000807780008007800d7
:1076b000ca04020000000000808f54000a003a0053
:1076c0000000eb000d04e000eaff32000c06e800c9
:1076d0008b05e8000a0078000a05e9000000e000d8
:1076e000eaff3a00e2ff37000fb89700ca04020031
:1076f00000000000000478000e007800ca040200b8
:107700000000000000005400daff3700889fbe0030
:107710008a9fbe008c9fbe008e1f78008005780077
:10772000010578001b4678001a84fb000c87fb00db
:107730000e007800ca0402000000000080047800f7
:107740008806780008007800ca04020000000000e3
:10775000808f54000b003a000000eb000c04e000a6
:10776000030032008b05e8000a05e800edff370052
:107770004f0778004f06be004f05be004f04be0005
:10778000000006000e007800ca040200000000009d
:10779000000478000d007800ca0402000000000018
:1077a00000005400f2ff3700889fbe008a9fbe0091
:1077b00000047800810578008204780003057800d1
:1077c0000000e000020032001004e00006003a0071
:1077d000004deb00800ceb000000eb004f05be00fd
:1077e0004f04be0000000600d804020000000000a4
:1077f000000444001804e000f5ff32008b0078001c
:1078000008007800fa0402000000000000004400b4
:10781000800c7800104d7800190078001004e0000a
:10782000020032000048eb00990ce80008007800e4
:10783000eaff37001600fa00889fbe008a9fbe004c
:107840008c1f78006e3f02000000000080992d0020
:10785000801f7800818d2900811f7800b67d02008d
:1078600000000000d197290000242100863b02007f
:1078700000000000e48757000000e0008e013200a5
:107880005212e2008401320040012000801f780083
:1078900041982900811f780080918000919180009b
:1078a000809fbe0081982900811f7800b67d02006c
:1078b00000000000ea87570020c0b300c0e79f0027
:1078c00000e224000100200080b79f0091b79f00d4
:1078d00002fe2f000f014100fc8057001000200025
:1078e000903f020000000000000478000000e0006b
:1078f0005f013500e10f540026013200d0c4b3000f
:107900006af5b700a0918000b1918000809fbe0011
:10791000619e2900811f7800b67d020000000000f2
:10792000e68757000cdb21007635ef007835ef0055
:10793000007d20000100200080b79f0091b79f00cc
:10794000b2a98000c3a98000c00320000014b800c1
:107950000098b900808444000800be001c24020086
:1079600000000000b0b79f00c1b79f00d2b79f00d2
:10797000e3b79f00e00f5400e08f5c00fb00350090
:107980007a55e200f6003a00a156210091407800b5
:1079900080c4b30080cf5000f10032000040eb0003
:1079a000c0e79f00a15621009140780070c4b30049
:1079b00080cf5000b3003200a156210091407800e2
:1079c000d0c4b30080cf5000aa00320001042000d0
:1079d00020002000984b0200000000000000e000a2
:1079e000830032005612e20049003a004fe097004f
:1079f0000024a000c0e79f0002fe2f000f014100fd
:107a0000fc80570030002000903f02000000000082
:107a1000000478000000e000330035000800e000ba
:107a20000f0032004fe097000028a3002a003a0020
:107a30000018a3000a003200a156210091407800ee
:107a400070c4b30080cf50001b003200a15621004b
:107a500091407800d0c4b30080cf500007003200be
:107a6000b0ab8000c1ab800061004000e080480006
:107a7000b0ab8800c1ab8800c1ff37008001eb00cc
:107a80001200200001db210002007800dc4102002e
:107a90000000000030c0b3009c4f1000f0ff3a001f
:107aa000200020002a4802000000000080c4b3002b
:107ab0006af5b700eaff3700e04c02000000000062
:107ac000e10f5000e1ff3a0001042000ae4802003f
:107ad00000000000ddff3700605d020000000000d4
:107ae0004fe09700d2ff37000003eb008002eb006d
:107af00000027800d304200082a32900910e200008
:107b0000d0a32900967c020000000000c3ff3700cc
:107b1000c850020000000000f0b79f0081bf9f0026
:107b200092bf9f00a3bf9f00f8aa800009ab80000e
:107b30000800be001c24020000000000e00f5400fa
:107b4000e08f5c00240035000002be000203be008e
:107b50007fb097008fb897001fb99700afb9970013
:107b6000aa1e020000000000222402000000000003
:107b70000005be00429a8000539a80000201500026
:107b800083815800b092800001002000800f5100d6
:107b9000818f590095ff3900004b2100a48a020013
:107ba000000000000000e00003003a004a9a88004c
:107bb0005b9a88008dff3700801f780048a4290059
:107bc000881f780090322000fc7c0200000000003a
:107bd000e4875700f5ff37006022b8000600200058
:107be000071f24005e1f020000000000d6ff3700c0
:107bf00008102000881f78004798210006202000e8
:107c0000455821005400200041002000a29180002e
:107c1000b391800020002000104502000000000009
:107c20008f87e9000000e0006eff32002000200096
:107c3000801f7800e1a62900811f780050042000f1
:107c4000fc7c02000000000026002000d50420007b
:107c5000540420008501780082a32900510c2000e3
:107c6000d0a32900967c020000000000e4875700a2
:107c70005cff37004fe097000014a000c0e79f00b2
:107c800052ff37000104200010002000984b020032
:107c9000000000000000e000040032004fe0970008
:107ca0000014a000c0e79f0043ff37003fb29700d9
:107cb000cfb297005fb39700efb39700884a2100d7
:107cc0003800be002801be005e1f02000000000058
:107cd0000004be000205be00c85002000000000003
:107ce0000002be000203be000800be000a01be0082
:107cf000961e0200000000000000e0002eff3d0084
:107d00000104200010002000404702000000000095
:107d10000000e000e1ff320010002000801f78002a
:107d200071a92900811f780070192000fc7c0200d5
:107d30000000000016002000d50420007419200067
:107d40008501780082a32900c10a2000d0a3290060
:107d5000967c020000000000e4875700cfff370048
:107d6000765102000000000005ff37006022b800d5
:107d700006002000071f24005e1f02000000000014
:107d8000b0b79f00c1b79f00d2b79f00e3b79f0075
:107d9000fbfe3700800c20000100200080b79f0010
:107da00091b79f0003fe2f008f81410008017800ea
:107db00001db210008007800dc4102000000000027
:107dc000e10f500010003200f8ac2900881f780045
:107dd00000192000fc7c0200000000000003eb0002
:107de00005192000d40420008401780082a3290012
:107df00011082000d0a32900967c0200000000009a
:107e00008f87e900c7fe370078a688005212e2008b
:107e10000f0032000cdb210031c0b3009ccf1000fa
:107e20000300320070c4b3006af5b700befe37002d
:107e300080c4b3006af5b7001202200021b0290007
:107e4000080078008043020000000000b6fe370002
:107e500080c4b3006af5b7002202200041b22900b5
:107e6000080078008043020000000000adfe3700eb
:107e70000003eb0080027800d40420008401780025
:107e800082a3290051062000d0a32900967c02007d
:107e90000000000097fe370048012000881f78008e
:107ea00070b42900801f7800b67d02000000000039
:107eb000e487570080fe370038b62900881f780015
:107ec000b67d02000000000080c4b3006af5b70070
:107ed00010c0b3007af5b700c9ff3700e0c4b300a3
:107ee0006af5b700f07c020000000000425002007a
:107ef000000000007c7f0200000000009c7a02006d
:107f000000000000944c020000000000e64d02005a
:107f1000000000000e5002000000000000000500fc
:107f2000889fbe008a9fbe008c9fbe008e1f780077
:107f30008001780001047800820478000000e900e4
:107f4000e70f500058003e00114178000204e000a5
:107f50004d0032000047eb000006eb007bc5b3008c
:107f60000900e000060032001900be00e9c5550016
:107f7000e00f5000e08f580001003200e6c54500d8
:107f80001dc0b3000045eb000218a30031003a0009
:107f90000228a30023003a000c00e0001e003a0073
:107fa0000a04e00011003a0070c5b30080cf55000c
:107fb0001500320040c5b30080cf55000b003a00d9
:107fc0000d01fb001900be00f84d0200000000008a
:107fd00039011000a98118004240a90003003400b3
:107fe0008046eb0018417800e7ff37000e4c780020
:107ff0000c0078004f0778004f06be004f05be000a
:108000004f04be0000000600d4e2a8000140fe00bc
:10801000d4e2a900f3ff3700fc4f0200000000008b
:10802000f2ff37000104200020002000c0050700f7
:108030000000e000050032002c13e200d6ff320001
:108040000e24a0000c06e800d3ff37000a45e80024
:10805000d1ff37000104200010002000b405070004
:108060000000e00006003200f412e20002003200dc
:108070000e14a0000c06e80018417800c4ff370079
:108080000a45e800fcff370042ba2900821f780049
:10809000c0032000fc7c0200000000000080eb0018
:1080a0008f87e900d3ff3700831f780030bc290099
:1080b000801f7800b0032000fc7c0200000000005c
:1080c0000080eb00e4875700caff3700889fbe009e
:1080d0008a9fbe008c9fbe008e1f7800000478002f
:1080e0008105780002057800830678000000e90029
:1080f000e10f50009d003e000b00e0008b003200bd
:10810000e10f5500780036000104200008007800d7
:10811000870507000000e000620032007ec5b30062
:108120000d00e000060032001d00be006947570048
:10813000e00f5000e08f5800010032006647470012
:10814000800320000040b800232b2100830440005e
:108150000a04e9000006eb000045eb0012c0b30082
:108160004240a9002a00340059009000880078009d
:10817000800f540001003400800078000100e0000e
:1081800034003400ee8144009300780031457800db
:1081900081097800090a900049009000000042001f
:1081a000808f500001003900840978008a5d7800d2
:1081b0000c06e8000804e900210420009140780042
:1081c0008180fb00c508de00010078006ff5b70074
:1081d00000ceb3004260b700590090000000e900f3
:1081e000d0049800c508dd0042c0bf007f40600099
:1081f0000140700042e0b700ea4f55001300320022
:108200000800e000110034000800e000d6ff3c0048
:108210003ed5bf000018a30009003a000c0078000a
:10822000ea4f5500010032000c00ea004f077800c9
:108230004f06be004f05be004f04be000000060002
:10824000fc4f020000000000f4ff3700804deb00ff
:10825000efff3700e0c4b300804f5700ecff32005f
:1082600069404000804f57000a0032000201fb00c5
:108270001d00be00f84d0200000000003d0110008e
:10828000ad8118004240a900e1ff34000041eb003d
:10829000ddff3700d4e2a8000140fe00d4e2a900cf
:1082a000d9ff3700881f7800e2bf2900821f7800bd
:1082b00000042000fc7c020000000000080378009d
:1082c000d5042000040420003305200012c3290037
:1082d000710e2000b0c32900967c0200000000004f
:1082e000e48757008dff37008a1f780040c42900bb
:1082f000801f7800f0032000fc7c020000000000da
:108300000a03780065052000f403200033052000ef
:1083100012c32900210e2000b0c32900967c020060
:1083200000000000e487570077ff370003c72900eb
:10833000831f7800e0032000fc7c020000000000a6
:108340000003eb00e5042000e403200033052000d7
:1083500012c32900e10d2000b0c32900967c020061
:10836000000000008f87e90065ff3700881f780054
:1083700020002000801f7800f2c92900821f7800a9
:10838000d0032000fc7c02000000000008037800fd
:1083900025052000d40320003305200012c3290046
:1083a000a10d2000b0c32900967c0200000000004f
:1083b000e687570050ff3700e4874700889fbe00dc
:1083c0008a9fbe008c9fbe008e1f7800000478003c
:1083d0000106780082047800030778000000e900b5
:1083e000e10f5000b3003e000c00e000a10032009d
:1083f0000900e0008e00320001042000080078002f
:10840000cb0407000000e0007800320071c5b30023
:1084100081f79f000e00e000080032001e00be0041
:10842000e2c4b30082f79f00e00f5000e08f5800d5
:108430000200320043c5b30083f79f008003200091
:108440000040b800222b2100020540008905780079
:108450008006eb0013c0b30093f79f000900e00013
:10846000300034005a0090000b047800808f5500d3
:1084700001003400000478000800e00044003400eb
:108480000a089000ca00900001004000fa00900025
:1084900081045000890f54002f0034000901780036
:1084a0000c007800180502000000000009004600da
:1084b000090154008a08900018050200000000001d
:1084c0000a0890000800400009005000700598005c
:1084d000080646008886460088855500210420004d
:1084e000914078008180fb00c508de000100780023
:1084f0006ff5b70000ceb3004260b7005a0090009d
:108500000800500050059800c508dd0042c0bf00bb
:108510007f4060000140700042e0b7000b00e000c7
:10852000d0ff3c003ed5bf000018a30007003a0072
:108530000d0078004f0778004f06be004f05be00c3
:108540004f04be004f00b10000000600fc4f0200c7
:1085500000000000f6ff3700080178000c007800ea
:108560001805020000000000fa009000888040001a
:10857000710598000a0990004a009000000041002f
:10858000808f5000d2ff390072059800d0ff37006d
:10859000e0c4b3008ff0970080cf5000e1ff3200bd
:1085a0006940400080cf50000c0032009ff19700de
:1085b0000301fb001e00be00f84d02000000000099
:1085c0003e011000ae8118004240a900d5ff3400e2
:1085d0008041eb0093f79f00d0ff3700d4e2a80062
:1085e0000140fe00d4e2a900ccff3700881f7800cc
:1085f000e0cd2900801f780040042000fc7c0200b0
:108600000000000008037800d50420004404200086
:108610003305200012d1290081152000b0c32900a4
:10862000967c020000000000e487570077ff3700c7
:10863000801feb00b3d12900831f78003004200095
:10864000fc7c0200000000000003eb006505200038
:10865000340420003305200012d1290031152000f8
:10866000b0c32900967c020000000000e487570098
:1086700061ff370072d42900821f78002004200097
:10868000fc7c0200000000000003eb00e504200079
:10869000240420003305200012d12900f114200009
:1086a000b0c32900967c0200000000008f87e9001b
:1086b0004fff3700881f780020002000801f7800bf
:1086c00061d72900811f780010042000fc7c020083
:1086d0000000000008037800250520001404200095
:1086e0003305200012d12900b1142000b0c32900a5
:1086f000967c020000000000e68757003aff370032
:10870000889fbe008a9fbe008c9fbe008e1f78008f
:108710000006be00820578005812e2000b0032000d
:10872000a15621009140780040c4b30080cf500092
:10873000060032000102200010002000fc030700a8
:1087400018c0b3000000e00001003a000044eb0054
:108750000c00e900e10f50000b0036000804e000b7
:10876000a5003a000c037800250520001404200021
:108770003305200052db2900911c2000b0c32900e2
:10878000967c0200000000000d00e000870032002f
:108790000b00e0000b003a000804e0007b003a0008
:1087a0000003eb00650520003404200033052000a1
:1087b00052db2900511d2000b0c32900967c020025
:1087c00000000000010220000c007800d803070020
:1087d0000000e0000b003a000804e00063003a00eb
:1087e0000c037800650520004404200033052000b8
:1087f00052db2900c11d2000b0c32900967c020075
:1088000000000000800320000060b800422c21001e
:10881000020540000007eb000b00e00036003200cc
:10882000ca0090005a009000008050004240a90009
:108830004a0034000b047800808f55000100360098
:10884000000478000a08900001004000ea0190004e
:1088500083045000890f540031003400090178006e
:108860008d00780003007800180502000000000069
:108870000a0890000901540089804600180502008a
:10888000000000000a0890000800400009005000a5
:1088900060059800888646008885550008074700cf
:1088a00021042000914078008180fb00c508de0093
:1088b000010078006ff5b70000ceb3004260b7004a
:1088c0005a0090000800400050059800c508dd00df
:1088d00042c0bf007f4060000140700042e0b7002e
:1088e000e10f56000c003200e20f56000800320083
:1088f0000b00e000caff3a000e0078004f07780036
:108900004f06be004f05be004f04be00000006002b
:108910008720a800f6ff37008540a800f4ff370045
:10892000080178008d007800030078001805020027
:1089300000000000ea009000888040006105980077
:108940000a0990004a00900000004100808f50000a
:10895000d0ff390062059800ceff3700d4e2a800ae
:108960000140fe00d4e2a900e1ff37008c1f78002f
:1089700000dc2900801f780040042000fc7c0200fd
:1089800000000000e487570095ff3700801feb00d0
:1089900042df2900821f780030042000fc7c0200a6
:1089a00000000000e48757007dff37000804e00066
:1089b0000a003a000003eb00e50420002404200034
:1089c0003305200052db2900f11c2000b0c3290030
:1089d000967c0200000000006dff370000e22900d5
:1089e000801f780020042000fc7c020000000000b2
:1089f0008f87e900efff37008c1f780020002000f0
:108a0000801f780002e52900821f780010042000f2
:108a1000fc7c020000000000e687570051ff370091
:108a2000e6874700889fbe008a9fbe008c9fbe00dd
:108a30008e1f7800800478000205be00f1b79f0009
:108a4000040778000506780086bf9f008706780037
:108a50000000e900e10f5000f6003e000a01be00f0
:108a6000e206b1000380b10020192c0011002000a3
:108a7000800f5100818f5900dd003e00ffb097004c
:108a80000100e900e60f5000c8003e000e00e900ba
:108a9000e60f5000b4003e000c00e000a2003200df
:108aa0000fb997000200e0008e0032000d00e000d8
:108ab0007c0032003fb197000200e0006800320005
:108ac000800320000048b800e22921000204400091
:108ad000180890000006b2005d003a000800780017
:108ae0001b0009000018eb000a01be000900780015
:108af00020030700e1ff2f000000e0002a003a00f9
:108b00002c1498001c1498000c1498003d1c98001c
:108b10002d1c98001d1c98008fb89700610c9800c0
:108b20003fb1970072149800e18f54002e0032007c
:108b3000e28f540023003a001622ef008f00a900b4
:108b40008f20a9008700a9008720a900674167003e
:108b5000a0c0bf0081cfb3000140600002407000a0
:108b6000a0e0b700efe8970067c160004411dd00a6
:108b7000a0c0bf00f1c8b300014060000240700017
:108b8000a0e0b70000002800b010880000402800d6
:108b9000c01088008f00a8008f20a80010062000b9
:108ba000100c98008000eb00010078004f0778005f
:108bb0004f06be004f05be004f04be006f00b1005f
:108bc00000000600891f780002e92900821f780052
:108bd00000042000fc7c0200000000008080eb000c
:108be000e4875700f0ff37000c22ef008d20a9002a
:108bf0008d40a9008520a9008540a9006741670034
:108c00004411dd0098c0bf00f1c8b300014060000e
:108c10000240700098e0b7006fe89700674160007d
:108c200099c0bf0081cfb3000140600002407000d6
:108c300099e0b7000000280060108800004028007c
:108c4000701088008d20a8008d40a800d3ff370049
:108c5000891f780050ec2900801f7800dcff370066
:108c6000801feb0000ef2900801f78002004200007
:108c7000fc7c0200000000000003eb006505200002
:108c80002404200033052000f2f1290031242000c3
:108c9000b0c32900967c020000000000e487570062
:108ca00087ff370091f22900811f780020042000ff
:108cb000fc7c0200000000000003eb00e504200043
:108cc0002404200033052000f2f12900f1232000c4
:108cd000b0c32900967c0200000000008f87e900e5
:108ce00074ff3700801feb0050f52900801f7800cb
:108cf00020042000fc7c0200000000000003eb00c8
:108d0000650520002404200033052000f2f129002d
:108d1000b1232000b0c32900967c020000000000af
:108d2000e487570061ff370041f82900811f780070
:108d300020042000fc7c0200000000000003eb0087
:108d4000e50420002404200033052000f2f129006e
:108d500071232000b0c32900967c020000000000af
:108d60008f87e9004eff37008e1f780000fb290037
:108d7000801f780020042000fc7c0200000000001e
:108d80000e03780025052000240420003305200070
:108d9000f2f1290031232000b0c32900967c0200a3
:108da00000000000e48757003bff3700811f780078
:108db000d2ff2900821f780020042000fc7c0200e2
:108dc000000000005fb39700250520002404200068
:108dd00033052000f2f12900f1222000b0c3290060
:108de000967c020000000000e487570027ff370050
:108df0008a9fbe00b2042a00821f7800200420004f
:108e0000fc7c0200000000000a0378002505200019
:108e10002404200033052000f2f12900b1222000b3
:108e2000b0c32900967c020000000000e6875700ce
:108e300012ff3700891f780020002000801f780073
:108e4000a1082a00811f780010042000fc7c020089
:108e5000000000000903780025052000140420000c
:108e600033052000f2f1290071222000b0c329004f
:108e7000967c020000000000e6875700f7fe3700ee
:108e8000889fbe0080047800010478000000e9009b
:108e9000e10f50005c003e0000022000800f5400f3
:108ea0001300320000042000800f54001000320034
:108eb000881f7800900c2a00801f78002004200072
:108ec000fc7c02000000000008037800250520005b
:108ed000240420003305200032102a00b12d200088
:108ee000b0c32900967c020000000000e487570010
:108ef000800320000048b800022b2100020040003f
:108f00001008a3003d003200880078000102b20082
:108f100010006400880f50002a003200e18f5400d6
:108f20001d003200e28f540012003a000100e00000
:108f30000c0032008720a9001942a80019e2a800fd
:108f40008f20a800800320000048b800022b2100d9
:108f500002004000100874000000eb004f04be0047
:108f6000000006008700a9001822a9008f00a800b1
:108f7000f4ff3700891f780020112a00801f780035
:108f800000042000fc7c0200000000000080eb00d8
:108f9000e4875700f1ff37000100e00005003200d0
:108fa0008540a9000f42a8000fe2a8008d40a8004c
:108fb000e4ff37008520a9000e22a9008d20a8001b
:108fc000e0ff3700c0142a000100e00001003a0071
:108fd00050152a00801f7800891f7800d2152a00ba
:108fe000821f780000042000fc7c020000000000ca
:108ff0000080eb00e6875700d8ff3700891f780014
:1090000050192a00ddff3700891f7800200020005a
:10901000801f7800021d2a00821f780010042000a3
:10902000fc7c0200000000000903780025052000f8
:10903000140420003305200032102a00712d200076
:10904000b0c32900967c020000000000e6875700ac
:1090500091ff3700881f7800000478000000e900c5
:10906000e10f50002a003e00e10f54001d003200c5
:10907000e20f540012003a001622ef008f00a90000
:109080008f20a9008700a9008720a90080cfb30006
:10909000a060b600f0c8b300a060b6001822ef00d0
:1090a000800320000040b800022b21000200400095
:1090b0000008eb000000eb004f0478000000060001
:1090c000881f780040212a00801f780000042000bb
:1090d000fc7c0200000000000080eb00e4875700e9
:1090e000f5ff37000c22ef008d20a9008d40a9006c
:1090f0008520a9008540a900f0c8b3009860b6009b
:1091000080cfb3009960b6000e22ef00e4ff370075
:10911000881f780020002000801f7800a2242a00e9
:10912000821f780010042000fc7c02000000000078
:1091300008037800250520001404200033052000d2
:10914000a2282a00c1342000b0c32900967c020066
:1091500000000000e6875700c3ff3700889fbe006d
:1091600080047800010478000000e900e10f50005d
:109170003f003e0000022000800f54001300320028
:1091800000042000800f540010003200881f780077
:1091900050292a00801f780020042000fc7c020057
:1091a00000000000080378002505200024042000aa
:1091b00033052000022d2a0011392000b0c32900f8
:1091c000967c020000000000e4875700e18f540005
:1091d0001d003200e28f540012003a000858a3002c
:1091e0000d0032008f20a9008720a9001942a90094
:1091f00019e2a900800320000048b800022b2100da
:10920000020040000881ea00100861000000eb0045
:109210004f04be00000006008f00a9008700a900cf
:10922000f4ff3700891f7800022e2a00821f780081
:1092300000042000fc7c0200000000000080eb0025
:10924000e4875700f2ff37000858a30005003200fa
:109250008d40a9008540a9000f42a9000fe2a90096
:10926000e4ff37008d20a9008520a900e1ff370029
:10927000891f780020002000801f7800b2312a006a
:10928000821f780010042000fc7c02000000000017
:109290000903780025052000140420003305200070
:1092a000022d2a00d1382000b0c32900967c02008c
:1092b00000000000e6875700aeff3700809fbe0029
:1092c000829fbe00849fbe00869fbe00881f7800dc
:1092d000d4c2bf000080fb004700de008083fb009b
:1092e000d4e2a9008540a900e0978000f1978000b2
:1092f00061004000e0804800e0978800f197880016
:109300000613e20030003200422d210012417800a5
:10931000d5002000639880002498800005437800e1
:109320000f22ab0014003a00ea4f51002100320036
:109330005898800038407800d4f2b70058988800d8
:10934000004178008080fb0081108800848041000b
:10935000810f540001003900539888000633ed0056
:10936000009880001198800061004000e080480073
:1093700000988800119888000613e200e8ff3a0080
:10938000ea4f5100e6ff3200c738dd00d4c2bf000b
:109390000074a10001407000d4e2b7004f047800cf
:1093a0004f03be004f02be004f01be004f00be0083
:1093b0000040060006007800d4f2b700851088004f
:1093c00005417800e6ff3700422d21001241780068
:1093d000ea4f5100ecff3a00cdff3700809fbe00fe
:1093e000829fbe00d4c2bf000080fb004700de00a9
:1093f0008081fb00d4e2a900d4c2a8008520a90086
:10940000509780006197800061004000e080480034
:1094100050978800619788000e22ab000700320049
:10942000b0968000c196800061004000e080480056
:10943000b0968800c1968800e832a8000e02ab0002
:109440000c0032000e42ab0017003200e852a800b8
:10945000d0968000e196800061004000e0804800e6
:10946000d0968800e1968800901080000e02ab0034
:10947000f4ff3a000e22ab00020032000e22a900d7
:10948000e832a900d4c2a900c718dd00d4c2bf00c9
:109490000074a10001407000d4e2b7004f01be008b
:1094a0004f00be0000400600e852a900a1978000ce
:1094b00090978000808f500013003100e892a9003f
:1094c000b19780009010800080587800b197880094
:1094d000d29780009097800000004100808f50005c
:1094e00001003900b2978800709780008197800052
:1094f00061004000e08048007097880081978800f4
:10950000f432ec00d9ff3700f0968000019780001c
:1095100061004000e0804800f096880001978800d4
:10952000e892a800d3ff3700809fbe00829fbe0054
:10953000841f7800d4c2bf000080fb004700de001b
:109540000082fb00d4e2a9008720a900a099800036
:10955000b199800061004000e0804800a099880037
:10956000b19988003e13e20015003200e3998000b3
:10957000229a80001922ab000f003a00109a800056
:10958000b080fb00d1108800109a88008300410051
:10959000810f500001003900129a8800c0998000a4
:1095a000d199800061004000e0804800c0998800a7
:1095b000d19988003e33ed003e13e200edff3a0002
:1095c000c720dd00d4c2bf000074a10001407000bc
:1095d000d4e2b7004f0278004f01be004f00be003a
:1095e00000400600809fbe00829fbe00d482a8007b
:1095f000d4c2bf000080fb004700de008081fb007a
:10960000d4e2a9008700a900109980002199800068
:1096100061004000e080480010998800219988008e
:109620001822ab00070032007098800081988000fb
:1096300061004000e08048007098880081988800b0
:109640002033a8001802ab000c0032001842ab0017
:10965000170032002053a80090988000a198800045
:1096600061004000e080480090988800a198880040
:10967000e01080001802ab00f4ff3a001822ab00a3
:10968000020032001822a9002033a900c718dd000b
:10969000d4c2bf000074a10001407000d4e2b70042
:1096a000d482a9004f01be004f00be00004006005a
:1096b0002053a9006199800050998000808f50004c
:1096c000130031002093a90071998000e010800000
:1096d0008058780071998800929980005099800094
:1096e00000004100808f500001003900729988000d
:1096f000309980004199800061004000e08048007e
:1097000030998800419988002c33ec00d9ff37004c
:10971000b0988000c198800061004000e08048005f
:10972000b0988800c19888002093a800d3ff370024
:109730000001be000000e900e10f50000a003e00f9
:10974000800320000010b800022b2100020040001e
:10975000030178000200a000100061001100200049
:10976000820f5000010032008000eb000100780001
:1097700000000600889fbe008a9fbe008c9fbe002e
:10978000000678000205be000000e900e10f50006d
:1097900052003e000a01be00e206b1000380b100a3
:1097a00020192c0011002000800f5100818f5900da
:1097b00039003e00f2aa800003ab80006a10b800b6
:1097c0006a19b900828040007051b800705ab9001f
:1097d000848141006e240200000000000004be00ed
:1097e000a2002000030020008e24020000000000e0
:1097f0001dc0b300e40f5000e08f580001003e0090
:109800008046eb00a2002000030020000800be00fc
:109810006e240200000000000d81fb0000014100e9
:109820008201e900800320000060b800a42a210022
:10983000040140000a89be00e22a21000200400023
:1098400003087800e10f560011003200e20f5600c5
:1098500006003a00f31088000000eb004f06be003f
:109860004f05be004f04be00000006008c1f7800ac
:1098700004362a00841f780000042000fc7c0200cb
:10988000000000000080eb00e4875700f3ff370082
:10989000a3108800f0ff37008a9fbe0094392a0089
:1098a000841f780020042000fc7c020000000000df
:1098b0000a03780025052000240420003305200039
:1098c000c23d2a0091532000b0c32900967c0200bb
:1098d00000000000e6875700b6ff37008c1f7800b5
:1098e00020002000801f7800a23e2a00821f7800fe
:1098f00010042000fc7c0200000000000c03780033
:10990000250520001404200033052000c23d2a0054
:1099100051532000b0c32900967c020000000000d3
:10992000e68757009bff37005212e2002100320009
:109930008291800093918000c0122000801f7800e7
:1099400047a821000620200045782100640020005f
:10995000310020001000200031fc07008f87e90053
:109960000000e00001003a000000060010002000a6
:10997000801f7800d0422a00801f78005004200009
:10998000fc7c02000000000016002000d50420002e
:109990005404200033052000b2452a005152200013
:1099a000b0c32900967c020000000000e487570045
:1099b000edff37006291800073918000deff370079
:1099c0000c00fa00889fbe008a1f7800d4a2a8006d
:1099d0008025200001002000f0b79f0081bf9f007c
:1099e00071a680000810200001005400e10f500013
:1099f0006d0034000005eb000101540003db210081
:109a000083804000f2815700100020006640020071
:109a1000000000000000e00010003c000c003500d9
:109a200064462a00841f780000322000fc7c02007b
:109a3000000000008f87e900d4a2a9000a00780086
:109a40004f0578004f04be000080fa0000000600b9
:109a5000ce34b5000085eb00f7ff3700ce34b400fc
:109a60001a002000c85002000000000090bf9f00b4
:109a7000a1bf9f00b2bf9f00c3bf9f00844a2100c7
:109a8000009abe000292be00b8a98000c9a9800059
:109a90000800be001c24020000000000e00f54007b
:109aa000e08f5c003a0035000002be000203be00f9
:109ab0001fb89700afb897003fb99700cfb997008c
:109ac000aa1e020000000000942402000000000012
:109ad00080a6880091a6880070a68000d2da2100b6
:109ae00082004000ce34ef008001eb0001007800de
:109af00004db2100848f50000600390042c2b3000d
:109b0000904f1100200032000000e900840f500047
:109b1000fbff31000300e00013003200838050009f
:109b20008100e800024b2100030078005885020004
:109b300000000000000478000000e000beff3200da
:109b4000e30f40000600320014482a00841f78000a
:109b5000f0322000fc7c0200000000008f87e9004a
:109b60000885e900b4ff3700a34a2a00831f780064
:109b7000e0322000fc7c020000000000ce34ef0048
:109b8000eaff2f00abff370080017800e1ff3700cc
:109b90006022b80006002000071f24005e1f02009c
:109ba00000000000c0ff3700004e2a00801f780030
:109bb00040332000fc7c0200000000008000eb002d
:109bc000ce34ef008f87e9008aff3700c091800014
:109bd000d191800080a5880091a58800e091800047
:109be000f1918000a0a58800b1a5880000000600c2
:109bf0000800fa00889fbe008a1f78000004be009b
:109c0000020578003e55e2004e0032000a00e000f6
:109c100032003a0011c1bf000078a30003003200f7
:109c2000d4e2a8000140fe00d4e2a900c85002001e
:109c300000000000485421003802be002803be0086
:109c400018240200000000006022b8000600240072
:109c5000f7082400c02102000000000090bf9f0010
:109c6000a1bf9f00b2bf9f00c3bf9f00b8a98000e3
:109c7000c9a980000800be001c24020000000000ea
:109c8000e00f5400e08f5c000e0035000002be00c3
:109c90000203be001fb89700afb897003fb9970006
:109ca000cfb99700aa1e0200000000009424020011
:109cb000000000004f0578004f04be000080fa004d
:109cc000000006006022b80006002000071f2400e4
:109cd0005e1f020000000000ecff37000800be001d
:109ce000280007000000e00006003a00c85002000b
:109cf0000000000048542100009cbe000294be00f9
:109d0000caff3700a4502a00841f78006019200081
:109d1000fc7c0200000000000003eb00d5042000e2
:109d2000641920003304200042522a00a1042000bc
:109d300090522a00967c0200000000008f87e90004
:109d4000eaff370010532a00801f780050192000c6
:109d5000fc7c0200000000000003eb00d5042000a2
:109d6000541920003304200042522a00e10320004d
:109d700090522a00967c0200000000008f87e900c4
:109d8000a2ff3700889fbe000004be003e55e200df
:109d900039003200e00f5400e08f5c0026003400f0
:109da00011c1bf000078a30003003a003ed5bf00f8
:109db0000018a3000f00320080552a00801f780091
:109dc000a0192000fc7c0200000000000003eb0052
:109dd000d5042000a41920003304200042582a0092
:109de0006109200090522a00967c020000000000c9
:109df0008f87e9000821ef000621ef00d4a9800039
:109e0000e5a980000821b80009a0b9000080410040
:109e100005c2b90084014000620888007308880008
:109e200011e1a80030c0b3003ef5b7000000eb0020
:109e30004f04be0000000600e0582a00801f780092
:109e400050192000fc7c0200000000000003eb0021
:109e500065052000941920003304200042582a0090
:109e60000109200090522a00967c020000000000a8
:109e70008f87e900caff3700705b2a00801f7800d7
:109e800090192000fc7c0200000000000003eb00a1
:109e9000d5042000941920003304200042582a00e1
:109ea000b108200090522a00967c020000000000b9
:109eb0008f87e900b7ff3700809fbe00829fbe00fa
:109ec00011e1a900d4c2bf000080fb004700de0002
:109ed000d4e2a90084e0a90002aa800013aa8000ad
:109ee00061014100e081490002aa880013aa8800ac
:109ef00051c0b3008000fd003ef5b7008000fd00ba
:109f00004700dd00412d2000914078000174a10040
:109f100080c0700001007800d4e2b7004f01be009d
:109f20004f00be0000400600889fbe000004be0037
:109f30003e55e200200032000800be0091ff0700fd
:109f40000000e0000c003a0011c1bf000078a3003f
:109f500006003200d4e2a8000140fe00d4e2a900cd
:109f600011c1bf000078a300faff3a000000eb0027
:109f70004f04be0000000600305e2a00801f7800fb
:109f800080192000fc7c0200000000000003eb00b0
:109f9000d50420008419200033042000b2602a0078
:109fa0006107200090522a00967c02000000000009
:109fb0008f87e900e4ff370010612a00801f7800d6
:109fc00070192000fc7c0200000000000003eb0080
:109fd000d50420007419200033042000b2602a0048
:109fe000c106200090522a00967c0200000000006a
:109ff0008f87e900d0ff370011e1a9000821ef00a9
:10a000000621ef000e21ef00700880006008880034
:10a0100050c0b3003ef5b700000005001221ef006c
:10a0200090088000800888000821ef000621ef00da
:10a030000e21ef00700880006008880080cfb30018
:10a040009760b60097c0bf00f1c8b3000140600040
:10a050000054a00097e0b7008cc0a9008ce0a800d5
:10a0600084c0a90084e0a9001061a80011a1a90082
:10a07000f0ccb3001061b60050c0b3003ef5b7009d
:10a080000000060000002000211c2000f0aa88002b
:10a0900001ab8800b0a98800c1a98800303327002f
:10a0a0000100200010ab880021ab8800d0a98800f7
:10a0b000e1a98800000037002021ef00000980009e
:10a0c000f00888001621ef001421ef001c21ef009a
:10a0d000e0088000d0088800f0c8b3009e60b60099
:10a0e0009fc0bf0081cfb300014060000014a000fa
:10a0f0009fe0b7008ea0a9008ec0a80086a0a9008e
:10a1000086c0a9001e61a8001fa1a900f0ccb30061
:10a110001e61b6000080eb00d0088800e0088800cf
:10a120001fe1a80030c0b30068f5b70000000600ca
:10a1300086c0a9006635ec00004006006855e200c4
:10a1400009003200a008800001002000b208800051
:10a1500003002000c011dd0002002000020070009a
:10a1600083807000000006000003eb00d50420008f
:10a170003413200033042000a2632a009109200038
:10a1800010642a00967c020000000000edff3700fa
:10a190000800fa00889fbe008a1f78006855e20018
:10a1a0004800320042c0bf000080fb004505de00d1
:10a1b0000a0078006ff5b70000ceb3004260b70028
:10a1c000a808800009002000b008800001002000dd
:10a1d000c000dd00000020000004740081847400d1
:10a1e0000800be001c2402000000000090bf9f0079
:10a1f000a1bf9f00b2bf9f00c3bf9f00e00f5400ec
:10a20000e08f5c002500350038ab80006140b9006c
:10a210001c240200000000000800e00019003500c6
:10a220006022b80006002000071f2400c0210200a1
:10a23000000000000002be000203be001fb897002d
:10a24000afb897003fb99700cfb997005e1f0200e3
:10a2500000000000c552dd002404200014427800f4
:10a260007f426200054272000002fd0042e0b7003a
:10a270000002fd004f0578004f04be000080fa0088
:10a28000000006006022b80006002000070f24002e
:10a290005e1f020000000000e1ff37006022b800ee
:10a2a00006002000071f24005e1f020000000000bf
:10a2b00090bf9f00a1bf9f00b2bf9f00c3bf9f0080
:10a2c000d1ff37000003eb00d50420003413200039
:10a2d0003304200092642a00f10a200010642a004e
:10a2e000967c020000000000aeff37003800fa0044
:10a2f000889fbe008a9fbe008c9fbe005212e20063
:10a30000ec0532008091800091918000809fbe001a
:10a3100080a72b00801f7800b67d0200000000009f
:10a32000e687570071a82b0000242100863b02001d
:10a33000000000000000e000d6053200820020008e
:10a34000e1a82b0010002000804302000000000064
:10a350008001eb00220320008e0078001000200016
:10a360006640020000000000a0c0b3002077980003
:10a3700012002000210320008e804000020078009f
:10a380008043020000000000d2c0b3009e4f1100c5
:10a39000e4ff32008044eb000005eb0033032000b3
:10a3a0008e814100420320000e01410091382b00b4
:10a3b0000e007800d43b020000000000000478008a
:10a3c0000001eb00321f9800080078008e040200a4
:10a3d00000000000000178003e1a90006822b800da
:10a3e00003962b00030242008800780014007800d6
:10a3f000243b0200000000000000e000a3053a003a
:10a400008944e8003e1990006810b80003962b00bc
:10a41000030540000201e800321f980020022000de
:10a42000800f5100e8ff36000904e0009205320079
:10a43000e1cf54008b053c002e1c900008027800f0
:10a440003a4090000081fb000300200061022000e0
:10a45000810f5100e08f59007a043e000260010034
:10a4600078003700770437009e003700e30037009c
:10a470001c01370073043700530137001f003700f9
:10a4800070043700650137009a013700bd013700bd
:10a490000f0237003c023700690237009002370094
:10a4a0002a003700b2023700e60237001d033700ea
:10a4b0005203370085033700be033700e20337003d
:10a4c000e4033700e6033700ec033700f4033700fa
:10a4d0005c0437005b0437005a0437005904370026
:10a4e00024043700570437005a0437007f0437002c
:10a4f000dc0437000b05370028053700f201200087
:10a5000071a92b0010002000804302000000000011
:10a510006044b800f0aa800001ab8000120e200059
:10a52000030020006e24020000000000800f540091
:10a53000818f5c000300310061044400e0844c0022
:10a54000faff37000000fe002e1a900033032000af
:10a550008e814100420320000e01410091382b0002
:10a5600004007800d43b0200000000000000e0007e
:10a570002c0032009040780090c7b30080cf50008c
:10a580002300320090c5b30080cf5000200032007d
:10a5900010c3b30080cf50001d00320040c7b3008d
:10a5a00080cf50001a00320040c5b30080cf500069
:10a5b000170032007140400080cf5000140032007c
:10a5c00050c4b30080cf5000110032005a32ef0067
:10a5d0003200200071ab2b001000200080430200ed
:10a5e0000000000052012000b1ab2b001000200041
:10a5f000804302000000000022002000a12521006d
:10a60000605a2f00848002000000000045ff3700e0
:10a6100010002000d09288002200200011ad2b00f5
:10a62000eeff3700823e2b00821f780043ad2b00e7
:10a63000831f7800b67d020000000000e487570009
:10a6400038ff370040c4b3006af5b700f682020055
:10a650000000000080c4b3006af5b70021938000b9
:10a6600000408000808f500011003200801f780071
:10a67000811f7800c3af2b00831f7800d00e20000d
:10a68000fc7c020000000000064080006505200000
:10a69000d40e200023052000a2b42b00c10e200000
:10a6a00070b52b00967c020000000000e687570082
:10a6b000620a2000c122210080572f0084800200fe
:10a6c000000000007c7f0200000000008257200094
:10a6d0002180200000002f00bc7602000000000056
:10a6e00010ff3700330320008e8141004203200019
:10a6f0000e01410091382b0008007800d43b020085
:10a70000000000000000e00017003200a20020005e
:10a710008000eb009c010200000000000002be006f
:10a720000001be00e206b1000380b10020192c0038
:10a7300011002000800f5100818f59000300360066
:10a74000849fbe00e0b52b00f2fe370084918800a4
:10a75000959188004200200001232100c0572f005e
:10a760008480020000000000a2918000b39180006c
:10a77000829fbe008091800091918000809fbe00ea
:10a7800001b82b00811f7800b67d02000000000098
:10a79000829180009391800010002000ba4b02004b
:10a7a000000000006044b800ea875700f0aa80006b
:10a7b00001ab8000120e2000030020006e24020076
:10a7c00000000000800f5400818f5c000300310006
:10a7d00061044400e0844c00faff370070c4b30009
:10a7e0006af5b7000000eb004f06be004f05be0043
:10a7f0004f04be000080fa00000006003303200072
:10a800008e814100420320000e01410091382b004f
:10a8100008007800d43b0200000000000000e000c7
:10a8200019003200a20020008000eb009c01020011
:10a83000000000000002be000001be00e206b10000
:10a840000380b10020192c0011002000800f51005e
:10a85000818f5900baff3e00a4918800b59188000d
:10a86000420020004123210000582f008480020074
:10a8700000000000a2918000b39180002000200021
:10a88000ba4b020000000000a2918000b39180004a
:10a89000829fbe0003bd2b00831f7800b67d02009f
:10a8a000000000006044b800e6875700f0aa80006e
:10a8b00001ab8000321c2000030020006e24020047
:10a8c00000000000800f5400818f5c000300310005
:10a8d00061044400e0844c00faff3700d0c4b300a8
:10a8e000bfff3700330320008e8141004203200068
:10a8f0000e01410091382b0008007800d43b020083
:10a90000000000000000e00014003200a20020005f
:10a910008000eb009c010200000000000002be006d
:10a920000001be00e206b1000380b10020192c0036
:10a9300011002000800f5100818f590080ff3e00e0
:10a94000649188007591880042002000c122210096
:10a9500080572f0084800200000000006291800078
:10a9600073918000829fbe0063c02b00831f78001c
:10a97000b67d0200000000006044b800e687570082
:10a98000f0aa800001ab8000321c200003002000f0
:10a990006e24020000000000800f5400818f5c00d4
:10a9a0000300310061044400e0844c00faff3700ea
:10a9b000629180007391800010002000ba4b020069
:10a9c0000000000057fe3700a2918000b391800084
:10a9d000829fbe0003bd2b00831f7800b67d02005e
:10a9e000000000006044b800e6875700f0aa80002d
:10a9f00001ab8000120e2000030020006e24020034
:10aa000000000000800f5400818f5c00b3ff310014
:10aa100061044400e0844c00faff37003303200057
:10aa20008e814100420320000e01410091382b002d
:10aa300008007800d43b0200000000000004780009
:10aa40000000e000290032002e189000080050009d
:10aa50000001e900321f9800e60f51001f003c0082
:10aa6000820478000200e00011003d0088007800b8
:10aa700000242100260502000000000082002000c2
:10aa800001242100c0582f00848002000000000033
:10aa900001242100811f780052c22b00821f780000
:10aaa000b67d0200000000007a75ef00e3fe37007b
:10aab00068c07c000080fb00300502000000000040
:10aac00000f47c003e1890000001e900321f98005d
:10aad00082047800f6ff3b00e4ff3700881f78000f
:10aae00060c42b00801f7800d2fe370072c72b0095
:10aaf000cdfe3700330320008e8141004203200049
:10ab00000e01410091382b0008007800d43b020070
:10ab100000000000f14d2b000000e00015003200a5
:10ab20000001eb008000eb003e0502000000000089
:10ab3000ef0f5000e08f580004003600809fbe00e9
:10ab400013c82b00831f7800f3fd3700f00fb2000d
:10ab500040928800220020008124210040592f00cb
:10ab600084800200000000004812f80010cb2b0087
:10ab7000dcff3700811f780042ad2b00821f780078
:10ab8000acfe3700330320008e81410042032000d9
:10ab90000e01410091382b0008007800d43b0200e0
:10aba00000000000000478000000e00046003200d1
:10abb000f82e0200000000000005be00f2ff2f008a
:10abc000f3f72700ec240200000000000000e00082
:10abd00005003a00881f7800f37e2b00831f780061
:10abe00010cd2b00cbfd37002e1890003303200032
:10abf0008e814100420320000e01410091382b005c
:10ac0000d43b02000000000000047800e1802b002b
:10ac10000000e000d7ff3200f82e02000000000024
:10ac20000006be00f2ff2f00f3f72700ec2402001d
:10ac3000000000000000e00003003a00881f7800d8
:10ac4000e3802b00e5ff3700ca918800db91880084
:10ac5000ec918800fd9188004200200081232100b2
:10ac600040582f00848002000000000042002000b5
:10ac7000c123210080582f008480020000000000c2
:10ac8000e0918000f1918000581e02000000000059
:10ac9000809fbe00829fbe00c0918000d191800045
:10aca000581e020000000000809fbe00829fbe0070
:10acb00001cf2b00811f7800b67d0200000000004c
:10acc000f287570097fd3700c17a2b00a9ff3700a4
:10acd000330320008e814100420320000e01410019
:10ace00091382b0008007800d43b020000000000df
:10acf00000047800f27e2b000000e0004afe3200e3
:10ad0000f82e0200000000000005be00f2ff2f0038
:10ad1000f3f72700ec240200000000000000e00030
:10ad200006003a00881f7800f07e2b00801f780014
:10ad300011cd2b00811f780077fd3700ca91880064
:10ad4000db918800420020008123210040582f0021
:10ad50008480020000000000c0918000d19180003a
:10ad6000581e020000000000809fbe00829fbe00af
:10ad700082d12b00821f7800b67d02000000000007
:10ad8000ea87570067fd3700330320008e814100ba
:10ad9000420320000e01410091382b00080078008a
:10ada000d43b02000000000000047800e3802b0088
:10adb0000000e0001f003200f82e0200000000003a
:10adc0000005be00f2ff2f00f3f72700ec2402007d
:10add000000000000000e00006003a00881f780034
:10ade000e1802b00811f780012cd2b00821f78009c
:10adf00049fd3700ea918800fb918800420020005d
:10ae0000c123210080582f00848002000000000030
:10ae1000e0918000f1918000581e020000000000c7
:10ae2000809fbe00829fbe0043d32b00831f78000b
:10ae3000d1ff3700831f780040ad2b0029ff37007a
:10ae4000330320008e814100420320000e014100a7
:10ae500091382b0008007800d43b0200000000006d
:10ae600001d52b000000e00042ff3200a2002000cc
:10ae70008000eb009c010200000000006102b900ac
:10ae800061005200e0805a00e50f5000e08f58004a
:10ae900009003600849fbe0063002000831f7800f5
:10aea00020d52b00801f7800b67d02000000000036
:10aeb000e88757001bfd37005492880022002000cd
:10aec000a124210060592f008480020000000000ae
:10aed0004a12f800f1d72b00811f7800d5fd37000a
:10aee000330320008e814100420320000e01410007
:10aef00091382b0008007800d43b020000000000cd
:10af000002d52b000000e000c7fd3200a2002000a7
:10af10008000eb009c010200000000006102b9000b
:10af200061005200e0805a00e50f5000e08f5800a9
:10af300006003600849fbe0060002000801f78005d
:10af400021d52b00811f7800d7ff3700649288003d
:10af500022002000c124210080592f00848002009b
:10af6000000000004c12f80072d92b0003ff3700dc
:10af7000330320008e814100420320000e01410076
:10af800091382b0008007800d43b0200000000003c
:10af9000813e2b000000e000f6fe32009040780079
:10afa00090c7b30080cf50002100320090c5b3009d
:10afb00080cf50001e00320010c3b30080cf50007d
:10afc0001b00320040c7b30080cf50001800320091
:10afd00040c5b30080cf50001500320071404000e2
:10afe00080cf50001200320050c4b30080cf500018
:10aff0000f0032005c32ef003200200071ab2b00fa
:10b00000100020008043020000000000b201200078
:10b0100011db2b0010002000804302000000000024
:10b0200022002000c1252100805a2f0075fd370025
:10b0300013002000e39288002200200011ad2b00b5
:10b04000efff3700330320008e81410042032000d0
:10b050000e01410091382b0008007800d43b02001b
:10b06000000000000000e0002a003200904078005c
:10b0700090c7b30080cf50002100320090c5b300cc
:10b0800080cf50001e00320010c3b30080cf5000ac
:10b090001b00320040c7b30080cf500018003200c0
:10b0a00040c5b30080cf5000150032007140400011
:10b0b00080cf50001200320050c4b30080cf500047
:10b0c0000f0032005e32ef003200200071ab2b0027
:10b0d000100020008043020000000000a2012000b8
:10b0e000d1dc2b0010002000804302000000000093
:10b0f00022002000e1252100a05a2f0041fd370049
:10b1000012002000f29288002200200011ad2b00d6
:10b11000efff3700803e2b00801f780041ad2b00f1
:10b120006dff3700330320008e8141004203200071
:10b130000e01410091382b0008007800d43b02003a
:10b14000000000000000e0002a003200904078007b
:10b1500090c7b30080cf50002100320090c5b300eb
:10b1600080cf50001e00320010c3b30080cf5000cb
:10b170001b00320040c7b30080cf500018003200df
:10b1800040c5b30080cf5000150032007140400030
:10b1900080cf50001200320050c4b30080cf500066
:10b1a0000f0032004e32ef003200200071ab2b0056
:10b1b0001000200080430200000000002201200057
:10b1c00081de2b0010002000804302000000000000
:10b1d00022002000e1242100a0592f0009fd3700a2
:10b1e00011002000719288002200200011ad2b0078
:10b1f000efff3700833e2b000eff370033032000a4
:10b200008e814100420320000e01410091382b0045
:10b2100008007800d43b0200000000000000e000bd
:10b22000bcff32009040780090c7b30080cf500040
:10b230002100320090c5b30080cf50001e003200c4
:10b2400010c3b30080cf50001b00320040c7b300d2
:10b2500080cf50001800320040c5b30080cf5000ae
:10b26000150032007140400080cf500012003200c3
:10b2700050c4b30080cf50000f0032005032ef00b6
:10b280003200200071ab2b00100020008043020030
:10b290000000000092012000b1df2b001000200010
:10b2a0008043020000000000220020000125210050
:10b2b000c0592f00d3fc3700120020008292880072
:10b2c0002200200011ad2b00efff370033032000d8
:10b2d0008e814100420320000e01410091382b0075
:10b2e00008007800d43b0200000000000000e000ed
:10b2f000ccfc32009040780090c7b30080cf500063
:10b300002700320090c5b30080cf500024003200e7
:10b3100010c3b30080cf50002100320040c7b300fb
:10b3200080cf50001e00320040c5b30080cf5000d7
:10b330001b0032007140400080cf500018003200e6
:10b3400050c4b30080cf50001500320000c7b300d6
:10b3500080cf50001200320000c5b30080cf5000f3
:10b360000f0032006032ef003200200071ab2b0082
:10b370001000200080430200000000008203200033
:10b3800051e12b001000200080430200000000006b
:10b390002200200001262100c05a2f0099fc37000e
:10b3a00010002000009388002200200011ad2b0027
:10b3b000f0ff37000a962b00e3e42b00831f780090
:10b3c000a0e52b00801f7800f1e52b00811f78009d
:10b3d00072e62b00821f7800b67d0200000000009c
:10b3e0000001eb00321f9800e88757002802200078
:10b3f0002a4090000004e00007003a00680545007c
:10b400000200e800301f980000017800880f50000b
:10b41000f7ff3600c3fb3700ba019000831f7800a6
:10b420002a009000801f78009a1f780072e62b0097
:10b43000821f7800b67d020000000000e8875700f8
:10b440003e199000edff3700b481020000000000bb
:10b45000b4fb3700ec77020000000000b1fb3700be
:10b460006432ef00c205200081e72b0010002000ad
:10b470008043020000000000f6ff370000652a004c
:10b480008e040200000000000001780001652a001f
:10b49000100020008043020000000000a1fb3700e4
:10b4a000330320008e814100420320000e01410041
:10b4b00091382b0008007800d43b02000000000007
:10b4c000000478000000e00012ff320002022000b9
:10b4d00051ed2b001000200080430200000000000e
:10b4e0009840780090c7b30080cf50001c00320015
:10b4f00090c5b30080cf50001900320010c3b300d4
:10b5000080cf50001600320040c7b30080cf5000fb
:10b510001300320040c5b30080cf5000100032004d
:10b520007140400080cf50000d00320050c4b30085
:10b5300080cf50000a0032005232ef00120120008a
:10b5400061ef2b001000200080430200000000008b
:10b550002200200021252100e0592f0029fc37007e
:10b5600012002000929288004200200081f02b00ff
:10b57000f4ff3700330320008e8141004203200096
:10b580000e01410091382b0008007800d43b0200e6
:10b59000000000000000e00016ff3200904078003c
:10b5a00090c7b30080cf50002100320090c5b30097
:10b5b00080cf50001e00320010c3b30080cf500077
:10b5c0001b00320040c7b30080cf5000180032008b
:10b5d00040c5b30080cf50001500320071404000dc
:10b5e00080cf50001200320050c4b30080cf500012
:10b5f0000f0032005832ef003200200071ab2b00f8
:10b60000100020008043020000000000b201200072
:10b61000d1f02b0010002000804302000000000049
:10b620002200200081252100405a2f00f5fb370021
:10b6300011002000c19288002200200011ad2b00d3
:10b64000efff37000080fb00801f780093f22b0093
:10b65000f7fb3700330320008e81410042032000b6
:10b660000e01410091382b0008007800d43b020005
:10b67000000000000000e0001a0032000001eb00b2
:10b680008000eb003e050200000000000002be004a
:10b69000411f2000810f5200e08f5a000600360043
:10b6a000849fbe00421f2000821f7800d3f42b002d
:10b6b000831f7800fcfd3700a49288002200200040
:10b6c00041252100005a2f00848002000000000064
:10b6d0005412f80000f82b00801f7800a1f82b000e
:10b6e00094fd3700d3532b00d2fd370033032000e5
:10b6f0008e814100420320000e01410091382b0051
:10b7000008007800d43b020000000000000478002c
:10b71000d3fa2b000000e000c6fd320060262100b5
:10b720001f0009000018eb000001eb00321f980019
:10b730008000eb004e709000084050000040e9008f
:10b74000e84f50003c003e008084fb000905780073
:10b7500068c07c000080fb00300502000000000093
:10b7600000f47c008904e900f9ff3b003e199000d9
:10b770006810b80062262100020040000a0178002b
:10b780008800780044040200000000002e18900099
:10b79000330320008e814100420320000e0141004e
:10b7a00091382b00d43b0200000000000004780018
:10b7b000ee7490003e1890000001e800321f9800df
:10b7c00082007800e70f510002003c000800e00012
:10b7d000d8ff3a00e1cf44000c0032000940e800f5
:10b7e000d2f2b7000204200061262100205b2f0066
:10b7f0008480020000000000d2d2bf000080fb0065
:10b80000801f780070fb2b00b6fc3700e3fd2b0097
:10b81000831f7800b67d02000000000002042000b3
:10b82000215b2f00602621006a80020000000000da
:10b830008f87e900bbfa370082002000821f780062
:10b84000881f7800811fe80053002c00831f7800b8
:10b85000b67d02000000000080c4eb00e8875700be
:10b86000dcff3700330320008e81410042032000bb
:10b870000e01410091382b0008007800d43b0200f3
:10b8800000000000d2532b000000e00066fb3200f5
:10b890000001eb008000eb003e050200000000000c
:10b8a0000002be00e00f5000e08f5800050032009b
:10b8b0006a005000e0805800eb0f4000e08f580015
:10b8c00011003e00b4928800220020006125210072
:10b8d000205a2f008480020000000000b0928000f7
:10b8e0000000e00005003200801f780092032c0069
:10b8f000821f7800a3f82b0092fc37007201200011
:10b9000001042c00e2fe3700849fbe00809feb0004
:10b91000a0002000801f780081052c00811f780086
:10b9200015fd3700330320008e81410042032000c3
:10b930000e014100f1082c0008007800d43b020001
:10b9400000000000000478000000e0001100320058
:10b95000602a2100150009000018eb00b202200047
:10b9600088007800602a21004404020000000000e2
:10b97000c2022000612a2100205f2f008480020083
:10b9800000000000622a2100821f780023092c0099
:10b9900027fb3700500b2c00dffd3700330320005e
:10b9a0008e814100420320000e01410091382b009e
:10b9b00008007800d43b020000000000000478007a
:10b9c0000000e000250032009040780040c6b3003f
:10b9d00080cf50001a00320040c4b30080cf500026
:10b9e0001700320000c7b30080cf500006003200bd
:10b9f00000c5b30080cf500003003200881f7800dc
:10ba0000420c2c005dfc3700800020001093880061
:10ba100002072000321f9800e2012000910e2c0046
:10ba200010002000804302000000000022002000df
:10ba3000610320008e804000e05a2f00f1fa3700a9
:10ba4000400020001093880042062000321f98001a
:10ba5000e201200081102c00f1ff370070122c0051
:10ba6000adfd37008e1f780032132c00821f780046
:10ba7000d3132c0033fc37008e1f7800e0142c0009
:10ba8000801f7800d1132c00aafc37003e199000cb
:10ba900060fa370061152c00811f7800b67d020026
:10baa0000000000010c0b3007af5b7008f87e900ee
:10bab00022fa3700609180007191800013fa3700fc
:10bac0007a01fa00881f78000210200001bb2100d3
:10bad00020002000cc0207000000e00097003400a6
:10bae000a0ab8800c8500200000000002224020021
:10baf0000000000080ab880091ab8800a1ab800003
:10bb000042e82f000f01410000bb21007701070030
:10bb1000a12c2c00e30f50006f003a0040e82f00ea
:10bb20000f0040008c0507000000e00077003a009d
:10bb300040e82f000f004000127e020000000000cd
:10bb4000a12d2c00e10f50006300320040e82f00cf
:10bb50000f004000906a0200000000000000e000ba
:10bb6000020032006012e20066003200e4805700fa
:10bb700040e82f000f004000bc73020000000000ee
:10bb8000e40f50004700320016003c00e20f500066
:10bb900008003e00d12e2c0040e82f000f0040008e
:10bba000c80307000000eb004f0478000080fa0093
:10bbb00000000600801f780000312c00801f7800f4
:10bbc000b67d020000000000e1342c0000e82f00e8
:10bbd0000f004000570407000080eb00e487570087
:10bbe000f1ff3700e80f5000f2ff3a006fb89700fe
:10bbf000e10f400025003200801fe8007c00b80003
:10bc0000c2812000e01f790020372c00801f7800bf
:10bc1000b67d020000000000e6875700c1382c0006
:10bc200040e82f000f004000a6030700021020008c
:10bc300001cb210040e82f000f004000500007001a
:10bc4000000478000000e0000c00320000017800e1
:10bc500001cb21002000200022020700880f5000a5
:10bc6000d0ff3200801f7800d2382c00821f78006d
:10bc7000b67d020000000000d7ff3700801feb00f8
:10bc8000313a2c00811f7800f9ff3700213d2c004c
:10bc9000811f7800b67d0200000000008f87e90058
:10bca000deff37006fb89700e10f40000f00320051
:10bcb000801fe8007c00b800c2812000e01f7900ee
:10bcc000903e2c00801f7800b67d0200000000002e
:10bcd000e6875700c1382c0040e82f000f004000d5
:10bce000780307000080eb00afff370031402c00e5
:10bcf000811f7800b67d0200000000008f87e900f8
:10bd0000f4ff3700a1412c00f3ff37000000d00002
:10bd1000822b2c00e01f7900b0432c00801f78009c
:10bd2000b67d020000000000c1382c0000e82f00a2
:10bd30000f00400063030700a7ff37000000e0008a
:10bd400007003a0020452c00801f780000052000e5
:10bd5000fc7c0200000000008f87e900e1ff370053
:10bd6000801f780081462c00811f7800600420002d
:10bd7000fc7c020000000000e4875700d9ff370078
:10bd80001401fa00889fbe008a9fbe0080047800dc
:10bd900081057800020578000000e000c300320051
:10bda0000b00e000b100320010032000800f5500ae
:10bdb0009d00360046ee2f000f0343000004eb0009
:10bdc0008000eb000001eb0003c4b30002804400dc
:10bdd000004890000004e00001003a00110020003b
:10bde0000100e0008e003200034b78000201e80001
:10bdf0000603e8000804e800e50f5100f3ff3400f3
:10be000079489000005b78000804e8008000eb00af
:10be10000001eb0003c4b30062c07c000004e0003a
:10be200001003a00110020000100e0007a00320019
:10be3000034b78000201e8000603e8000804e8006c
:10be4000e50f5100f4ff340079409000004b78007a
:10be5000c9d092000104e00002003a001604a000dc
:10be6000c9d092000603e8000804e8008003eb0054
:10be70000104e000200032008000eb000001eb0034
:10be8000683ab80003c4b300040041000900400050
:10be9000405092000004e00001003a001100200030
:10bea0000100e0005a003200034b78000201e80074
:10beb0000603e8000804e800e50f5100f2ff340033
:10bec0000480440030589200004b7800c9d09200a2
:10bed0000180fb000000e900808f53004900320020
:10bee0008703e8000603e8000804e8000180fb007f
:10bef000808f5300e0ff350030c0b300005b780056
:10bf000000cfb300005b78000884e80009099000c6
:10bf1000020044000080e8008a0f50002f0031002a
:10bf2000f2804400060078001805020000000000be
:10bf300009089000000444000b03780001ccb30012
:10bf4000015b7800005beb000000eb000001eb0000
:10bf5000e00f140010003d0001427800fbc04000db
:10bf6000c5cdb300d7cdb30049ee2f008284440085
:10bf7000e9c17f0084cf51001400320081cf51000d
:10bf80000e003200034b78000201e8000603e800cf
:10bf9000880f5100f4ff35008000440000ccb3004e
:10bfa000005b7800004beb00638040004f05be0053
:10bfb0004f04be000080fa0000000600034b78002a
:10bfc0000000e800076b7800efff3700014b7800b6
:10bfd0000000e800056b7800ebff3700801f780059
:10bfe0008a1f7800e9472c00891f7800300520005f
:10bff000fc7c0200000000000080eb00e687570098
:10c00000eaff37001604a000c9d09200b4ff370041
:10c01000004bd000a5ff3700004bd00085ff370054
:10c02000004bd00071ff37008a1f7800004c2c00b5
:10c03000801f7800f0042000fc7c0200000000005b
:10c040000a03780065052000f40420004305200061
:10c05000024f2c005114200000502c00967c02004e
:10c0600000000000e487570052ff370060502c00aa
:10c07000801f7800e0042000fc7c0200000000002b
:10c080000003eb00e50420000502780043052000d2
:10c09000024f2c001114200000502c00967c02004e
:10c0a000000000008f87e9003fff370070532c002d
:10c0b000801f7800d0042000fc7c020000000000fb
:10c0c0000003eb00e5042000d40420004305200019
:10c0d000024f2c00d113200000502c00967c02004f
:10c0e000000000008f87e9002dff3700889fbe0009
:10c0f0008a9fbe008c9fbe008e1f780000047800cf
:10c1000001077800820478000000e000e5003200ba
:10c110000900e000d30032000e00e000c000320051
:10c1200022002000e88644000d0578000900780010
:10c13000bb0009000018eb000884e8008005eb0054
:10c140000006eb000e00e0001d003200e30f51007e
:10c15000970032004a003c00e10f510038003200e5
:10c16000e20f51002d003a008b05e800e68f5500e4
:10c1700020003400004deb0018407800f046980095
:10c180008005eb0089067800090578007940900069
:10c190000000d1006f00600010003a001200200083
:10c1a0000c06e8000804e8008e0f56000400310079
:10c1b000e70f510002003200e80f5100e3ff3a00a0
:10c1c00069f092000080fb004f0778004f06be0028
:10c1d0004f05be004f04be000000060080562c0034
:10c1e000801f7800b67d0200000000008f87e90004
:10c1f000eaff37009840780000c4b30080cf5000b9
:10c20000040032000180fb000000d100005d7800d6
:10c21000e3ff3700005deb00e1ff3700821f78008d
:10c2200070582c00801f7800d0052000fc7c020094
:10c230000000000010002000e4875700e2ff3700f4
:10c240008b05e800e68f5500eaff3400004deb0057
:10c2500018407800f04698008005eb001880fb003d
:10c26000420020000008a300cdff3a004d1120003d
:10c27000898646000d05780032002000c8ff37008f
:10c28000e50f510044003200e40f51002d0034004e
:10c29000e60f5100e1ff3a009841780000ccb3006e
:10c2a00080cf5100240032000e00e900800f5600bc
:10c2b0001600320089089000f00f2000808f500097
:10c2c00006003e00035d7800090890000000e800c9
:10c2d000800c98008b05e800b1ff3700811fe80053
:10c2e000d05b2c00801f780060062000fc7c0200e0
:10c2f00000000000004deb0080c0b300e0f49a00a5
:10c3000082002000e4875700a5ff370040602c0022
:10c31000801f780050062000fc7c02000000000016
:10c32000004deb0080c0b300e0f49a0082002000d2
:10c330008f87e9009aff3700004deb007200200064
:10c3400097ff370018407800c0f49a007200200070
:10c350001880fb00e10060000d0032000018a3000f
:10c3600009003200c00ab20004003a0030c0b30035
:10c37000e0f49a005200200089ff370020c0b3008b
:10c38000e0f49a0086ff370010c0b300fcff3700ce
:10c39000e1f49a0082ff370018407800d0f49a0048
:10c3a000728544008005eb00620020007cff3700ae
:10c3b0008b05e800e68f55008eff3400004deb0042
:10c3c00018407800f04698008005eb0049d09200b4
:10c3d0000040e800c0d49a00e74f500008003e003b
:10c3e0001880fb000008a300020032004200200079
:10c3f0006bff3700e88646000d05780068ff3700c0
:10c4000080002000801f780060642c00801f78006e
:10c4100090052000fc7c020000000000b6ff370001
:10c42000801feb0010692c00801f78008005200021
:10c43000fc7c0200000000000003eb00650520000a
:10c440008405200043052000926b2c00411f200032
:10c4500000502c00967c020000000000e48757008a
:10c460002fff3700806c2c00801f780070052000a3
:10c47000fc7c0200000000000003eb00e50420004b
:10c480007405200043052000926b2c00011f200042
:10c4900000502c00967c0200000000008f87e9000d
:10c4a0001dff3700506f2c00801f780060052000b2
:10c4b000fc7c0200000000000003eb00e50420000b
:10c4c0006405200043052000926b2c00c11e200053
:10c4d00000502c00967c0200000000008f87e900cd
:10c4e0000bff3700889fbe008a1f78008004780009
:10c4f00001057800020478000000e900e10f500017
:10c500002e003e000a00e0001c0032000800e0009f
:10c5100009003200080178008a00780009007800dc
:10c520008043020000000000080078004f057800fa
:10c530004f04be0000000600801feb0010722c00ac
:10c54000801f780000062000fc7c02000000000034
:10c550000003eb00650520000406200043052000d1
:10c5600052742c00312d200000502c00967c0200cb
:10c5700000000000e4875700e6ff370000752c003c
:10c58000801f7800f0052000fc7c02000000000005
:10c590000003eb00e5042000f40520004305200023
:10c5a00052742c00f12c200000502c00967c0200cc
:10c5b000000000008f87e900d4ff3700891f780052
:10c5c00020002000801f780070772c00801f7800ea
:10c5d000e0052000fc7c0200000000000003eb00ee
:10c5e00025052000e40520004305200052742c009e
:10c5f000b12c200000502c00967c020000000000ae
:10c60000e6875700bfff3700e4874700889fbe00da
:10c610008a9fbe008c9fbe008e1f78008005780028
:10c6200081067800020578000000e900e10f500063
:10c630007d003e000d00e0006b0032000a00e000cb
:10c64000580032006044b8001ec0b3000cccb300e8
:10c650008a8f54004e0031008001eb001200200050
:10c66000f08057000b007800dc4102000000000061
:10c67000e10f500041003a00e10f54002800320061
:10c680000800e00022003200e20f540017003a00d8
:10c690008ff09700d0cdb30080cf50001000320053
:10c6a000c0cdb30080cf50000a0032001800200037
:10c6b0000e04e000e6ff3a00090078004f0778001a
:10c6c0004f06be004f05be004f04be004f00b10034
:10c6d000000006008cf67c008904e800f3ff3700b8
:10c6e00000c0e90080f67c00fbff3700881f78005f
:10c6f000817a2c00811f780070062000fc7c0200eb
:10c70000000000000080eb00e4875700ebff3700db
:10c710008ff097008ccf5000e5ff3a00edff370017
:10c720008ff097008ccf500008003200b0cdb300de
:10c7300080cf50000300320081f67c008904e800bd
:10c74000dbff370028002000d9ff3700e18f5400bd
:10c75000d7ff36008cf67c008904e8000047eb0028
:10c760008a8f5400d2ff39008a1f7800707e2c0017
:10c77000801f780060062000e0ff3700801f7800ef
:10c7800001822c00811f780050062000dbff37005b
:10c790008a1f7800707e2c00801f780040062000e1
:10c7a000d6ff3700801feb0031852c00811f7800f9
:10c7b00030062000fc7c0200000000000003eb00bb
:10c7c00065052000340620004305200072872c00f8
:10c7d000f12f200000502c00967c02000000000089
:10c7e000e487570097ff370010882c00801f7800df
:10c7f00020062000fc7c0200000000000003eb008b
:10c80000e5042000240620004305200072872c0048
:10c81000b12f200000502c00967c02000000000088
:10c820008f87e90085ff37008b1f780020002000ec
:10c83000801f7800718a2c00811f7800100620006c
:10c84000fc7c0200000000000003eb002505200036
:10c85000140620004305200072872c00712f200051
:10c8600000502c00967c020000000000e687570074
:10c8700070ff37000200fa00889fbe008a9fbe004a
:10c88000800478000105780002047800a156210098
:10c890009140780070c4b30080cf50004100320056
:10c8a000a1562100914078006340500080cf500095
:10c8b0003c0032000102200010002000984b0200d2
:10c8c000000000000000e000360032000900e00037
:10c8d0006c0032000a00e00059003200a0c0b30032
:10c8e000e0f79f0012002000ea8057000200780065
:10c8f00080430200000000000800e0000200320057
:10c900001804e00045003a000004eb000a00e000d3
:10c910001d003200bb0d200069417c008280fb00bd
:10c920008b8f50003a0032002d003c00000c20009c
:10c93000808f5000270032000204e0001d00350007
:10c940000280fb000000d000a1ca2c0060807800ab
:10c950008e040200000000000001780069407c00a5
:10c960000080fb000000d000a1ca2c00e08078000d
:10c970001000200080430200000000000804e800ce
:10c980008a0f5400e4ff3900ea805700a0c0b300ca
:10c9900080687800120020000200780080430200c6
:10c9a000000000004f05be004f04be000080fa00ea
:10c9b000000006000280fb00801f7800708d2c00b4
:10c9c000801f7800b67d020000000000e487570059
:10c9d000eaff370042002000e18d2c00e4ff370021
:10c9e000c00d2000808f5000060032000000e800db
:10c9f000808f5000d0ff3a0042002000318e2c0082
:10ca0000dbff370042002000818e2c00d8ff37006a
:10ca100042002000d18e2c00d5ff3700080078009e
:10ca20008e040200000000000001780088007800f9
:10ca3000100020008043020000000000b2ff370019
:10ca4000801feb00218f2c00811f780090062000b2
:10ca5000fc7c0200000000000003eb0065052000e4
:10ca6000940620004305200032912c0061382000fc
:10ca700000502c00967c020000000000e487570064
:10ca800096ff3700e0912c00801f78008006200080
:10ca9000fc7c0200000000000003eb00e504200025
:10caa000840620004305200032912c00213820000c
:10cab00000502c00967c0200000000008f87e900e7
:10cac00084ff37000800fa00889fbe008a9fbe00de
:10cad0008c1f780080047800010578000000e000d9
:10cae00084003200794890000080fb000000d100f3
:10caf0000080fb00010020006f0060008000eb0060
:10cb00007282570013002000e2ff2f0060380200fd
:10cb1000000000006e845700794090000080fb0008
:10cb20000000d1000080fb00010020006f006000c9
:10cb30008000eb000802780013002000e2ff2f00c5
:10cb40006038020000000000f94890000100d100a8
:10cb50006f006000728157000000e00001003a00a1
:10cb6000c2382c00821f78000100d1006f006000e5
:10cb7000e1932c0001003a00c1382c00811f78009d
:10cb8000e89f4400f94090000100d1006f00600070
:10cb90000801780001003a00c2382c00821f78009a
:10cba0000100d1006f006000e1932c0001003a0009
:10cbb000c1382c00811f7800891f78008a00780016
:10cbc0000a00e00049003200811f780001942c0027
:10cbd000811f7800b67d0200000000000006eb0017
:10cbe000f087570049d092000004e0003200320084
:10cbf0006865b8000a844400385892000080fb0041
:10cc00000000d1000080fb00010020006f006000e8
:10cc10008000eb007282570013002000e2ff2f001b
:10cc200060380200000000003858920001952c0086
:10cc30000078a30001003a00c1382c00811f780061
:10cc40000a804400305892000000d1006f0060005c
:10cc5000f48057000000e00001003a00c1382c00c9
:10cc6000811f78000a804400305892000000d100f3
:10cc70006f006000e1932c0001003a00c1382c00e5
:10cc8000811f78000a80440041112000811f40006c
:10cc900020952c00801f7800b67d02000000000067
:10cca000ea8757000c06e80049d092000080fb009c
:10ccb000800f5600ceff3500f29f4400890c900093
:10ccc000891f7800c1952c00811f7800b67d020075
:10ccd00000000000e68757004f0678004f05be00b1
:10cce0004f04be000080fa0000000600c1382c008e
:10ccf000b5ff3700e0962c00801f7800a0062000ca
:10cd0000fc7c0200000000000003eb00e5042000b2
:10cd1000a40620004305200052992c00b13b2000be
:10cd200000502c00967c0200000000008f87e90074
:10cd30006cff3700889fbe000004be000000e000ca
:10cd40000b0032000800be0019000700880990009f
:10cd500072014400a4002000719a2c0010002000f1
:10cd60007a340200000000004f04be0000000600fc
:10cd7000c09a2c00801f7800a0062000fc7c0200d6
:10cd8000000000000003eb00e5042000a4062000e2
:10cd900043052000c29c2c00013f200000502c00c5
:10cda000967c0200000000008f87e900e5ff370055
:10cdb0000800fa00889fbe008a9fbe008c1f780082
:10cdc00080047800010578000000e000d200320005
:10cdd000794890000080fb000000d1000080fb003b
:10cde000010020006f0060008000eb00728257009d
:10cdf00013002000e2ff2f00603802000000000056
:10ce00006e845700794090000080fb000000d10044
:10ce10000080fb00010020006f0060008000eb003c
:10ce20000802780013002000e2ff2f0060380200a3
:10ce300000000000794190000280fb00c500de0088
:10ce4000e39f6000c700de00811f7800801f78002c
:10ce50000000d1006f0060008800780001003a00f7
:10ce6000719d2c00811f78000200d1006f006000ce
:10ce7000e1932c0001003a00a19d2c00811f780055
:10ce8000891f780061002000811f78007949900097
:10ce90000280fb00c500de00e39f6000c700de00eb
:10cea000811f7800801f78000000d1006f006000b3
:10ceb000a1fd2f008f8040000000e00001003a003b
:10cec000719d2c00811f78000200d1006f0060006e
:10ced000e1932c0001003a00a19d2c00811f7800f5
:10cee000e89f440060002000801f78008a007800de
:10cef0000a00e00086003200811f7800c19d2c00ee
:10cf0000811f7800b67d0200000000000006eb00e3
:10cf10000f02b10049d092000004e0003800320056
:10cf20006865b8000a844400385892000080fb000d
:10cf30000000d1000080fb00010020006f006000b5
:10cf40008000eb007282570013002000e2ff2f00e8
:10cf50006038020000000000385892004500de00f2
:10cf6000e31f6000385892004700de00e11f6000b8
:10cf7000385892000080fb00801f780038589200db
:10cf80000000d1006f006000f88057000000e00052
:10cf900001003a00719d2c00811f78000a80440036
:10cfa000305892000000d1006f006000e1932c0027
:10cfb00001003a00a19d2c00811f78000a804400e6
:10cfc00041112000811f400060002000801f780078
:10cfd0000c04e800881f7800b1a32c00811f7800a2
:10cfe000b67d020000000000f287570008067800b6
:10cff00049d092000080fb00800f5400c8ff35002c
:10d00000794890000080fb004701de0079409000e5
:10d010000080fb004700de0081a62c00800f51003d
:10d020000400320041a72c000200e00001003a0099
:10d0300041a82c00811f780059f092000080fb006d
:10d04000801f780049f092000080fb00801f78006c
:10d0500050a92c00801f7800b67d0200000000005f
:10d0600079f092000084fb00e88757000818a300bd
:10d070002200320009f092000080fb00801f78003f
:10d0800079e892000080fb00801f780069e8920038
:10d090000080fb00801f780059e892000080fb00b0
:10d0a000801f780059289100e9289100581e02003d
:10d0b00000000000809fbe00829fbe0039289100c2
:10d0c000c9289100581e020000000000809fbe0089
:10d0d000829fbe00f0ab2c000828a30001003a009c
:10d0e000c0382c00801f780071ac2c00811f7800a4
:10d0f000b67d020000000000fc8757004f06780054
:10d100004f05be004f04be000080fa00000006007c
:10d11000c1382c0078ff370070b02c00801f7800d9
:10d12000a0062000fc7c0200000000000003eb00d1
:10d13000e5042000a406200043052000b2b22c0024
:10d140005140200000502c00967c0200000000009e
:10d150008f87e9001eff3700e4874700889fbe00e5
:10d160008a9fbe008c9fbe008e1f780080057800cd
:10d170000000e000cc0032007bf092000068a300c9
:10d18000210032007b4990000200d1006f00600056
:10d190000004e0001c0032008080fb00130020002f
:10d1a00060928000808f50000e003e00230020001f
:10d1b00050928000808f50000a003e0010ceb300d5
:10d1c00000406100f04d980000017800120eb2009e
:10d1d0000100e9004240a90009003400f24d980026
:10d1e0008001eb00030078004f0778004f06be0077
:10d1f0004f05be004f04be004f00b1000000060006
:10d200000200a000f5ff37008046eb000047eb006e
:10d210009ef79f008ef79f000086eb0048112000cc
:10d220000b0444000005eb00cbd492000904e0009d
:10d230001800320042002000a1da2c00080078001b
:10d24000d0050200000000000000e00051003a009c
:10d25000c840900000c2b30080cf500002003200ee
:10d260000104e00036003a00784090000078a30006
:10d2700003003a008d46e800e10f46002e00320020
:10d280000a05e800680444000980fb00800f55008f
:10d29000e8ff350053002000e10f4600d1ff3200c7
:10d2a0000d81fb000e80fb000000410063002000a8
:10d2b00061928000810f5000caff3e0051928000b1
:10d2c00073002000810f5100c6ff3e001ff1970040
:10d2d0000280fb0083002000810f5000c1ff3e0050
:10d2e0006860b800808145000ff097000004e000fe
:10d2f0000f003200b35892000100d1006f006000af
:10d300000041e90010ceb30080c060000280fb0045
:10d310000000d00000c07000b0599a000204e00084
:10d32000afff3a000074a000b0599a00acff37007c
:10d3300033589200fbff37000a067800d0ff370011
:10d34000784090000080fb008000d1006fc1600039
:10d350004700de00caff3a00430020000204e0005c
:10d36000a0ff320002474700e10f460005003200ef
:10d370001ff09700804f5100c1ff360092f79f00c9
:10d38000bfff37000a06780010c0b30080f79f0087
:10d39000f7ff37000a00e00011003a0052002000b9
:10d3a000f1da2c0008007800d0050200000000002f
:10d3b0000000e0000a003a004e12e20006003a00c7
:10d3c000784090000078a300adff3a000074a00000
:10d3d0007044980082ff37003300200081ff37003f
:10d3e0005200200051db2c0008007800d00502001c
:10d3f000000000000000e00005003a0078409000c6
:10d400000074a00070449800cbd492009cff3700b9
:10d41000080078008e0402000000000000004400b4
:10d4200070f897000080fb00ee050200000000008d
:10d430000000e00015003200784090000080fb0002
:10d440008000d1006fc160004700de00eeff3a00af
:10d45000430020000204e00062ff32000247470060
:10d46000e10f4600050032001ff09700804f510089
:10d47000e5ff360092f79f00e3ff37000a067800c9
:10d4800010c0b30080f79f00f7ff37000124210090
:10d4900008007800fa050200000000000000e0002b
:10d4a000d6ff3200d8ff3700b0db2c00801f780099
:10d4b000a0062000fc7c0200000000000003eb003e
:10d4c000e5042000a406200043052000a2dd2c0076
:10d4d000b14b200000502c00967c020000000000a0
:10d4e0008f87e90024ff3700800178000001eb00fe
:10d4f0006410b800841d2c00840040001100fb0063
:10d50000808f5100040032000201e800e70f510053
:10d51000f7ff360000000500110090000000060033
:10d520004f03b000889fbe008a9fbe008c9fbe0044
:10d530008e1f7800000678000000e000ac01320089
:10d540008004eb00680546000904d000e2f62c00d8
:10d5500002044400180078008e040200000000005d
:10d56000000178008a007800180078001e0602008a
:10d57000000000000000e000990132008904e8008a
:10d58000f98f5400f0ff36006015200000004600bf
:10d5900080bf9f00720746000c0c9000d0c7b300fc
:10d5a0009e4f10007e0132007cf092000004a0002b
:10d5b00070f69a001e4078000080fb0001002000f9
:10d5c0007c005000e0805800f2052000820f5000df
:10d5d000e08f58006b003e00006001000a01370038
:10d5e0000901370067003700660037006500370023
:10d5f0006f003700630037006200370057003700c4
:10d60000600037005f003700ff0037005d00370023
:10d610005c0037005b0037005a00370059003700c4
:10d620005800370057003700ac003700550037006e
:10d6300054003700530037005200370051003700c4
:10d64000500037004f0037004e0037004d003700c4
:10d650004c0037004b0037004a00370049003700c4
:10d660005300370047003700460037009b00370063
:10d6700044003700430037004200370041003700c4
:10d68000400037003f0037003e0037003d003700c4
:10d690003c0037003b0037003a00370039003700c4
:10d6a00038003700370037003600370035003700c4
:10d6b00034003700330037003200370031003700c4
:10d6c000300037002f0037002e0037002d003700c4
:10d6d0002c0037002b0037002a00370029003700c4
:10d6e000280037002700370026003700c600370023
:10d6f00024003700230037002200370021003700c4
:10d70000200037001f0037001e0037001d003700c3
:10d710001c0037001b0037001a00370019003700c3
:10d7200018003700170037001600370015003700c3
:10d7300014003700130037001200370011003700c3
:10d74000100037000f0037000e0037000d003700c3
:10d750000c0037000b0037000a0037000fb99700a4
:10d76000880078000e007800588502000000000054
:10d770000000e00003003a007cf092000014a000da
:10d7800070f69a007cf09200620060000000cf000a
:10d790000000e9004f00de004f0778004f06be0092
:10d7a0004f05be004f04be004f03b100000006004d
:10d7b0005e80fb00ee050200000000000000e000bb
:10d7c0001c003a008000eb000e0078009502070074
:10d7d0000fb997000089be00f2ff2f00f3f7270072
:10d7e000ec240200000000000000e000e5ff320031
:10d7f00069074700110020000e0078008902070029
:10d800000fb997002001980031019800f2ff2f0016
:10d81000f3f72700ec240200000000000000e00005
:10d82000d8ff32007cf092000034a00070f69a001d
:10d83000d1ff3700820020008e00780000fc2f000e
:10d840000f00400044040200000000008044eb0090
:10d8500089cf9f008000eb0000fc2f000f004000ec
:10d86000f30007000fb997000089be00f2ff2f00f8
:10d87000f3f72700ec240200000000000000e000a5
:10d88000c0ff32006907470080fd2f000084470079
:10d89000920020008e007800080078004404020006
:10d8a0000000000099e79f001100200008007800a8
:10d8b000df0007000fb997002001980031019800a0
:10d8c000f2ff2f00f3f72700ec2402000000000015
:10d8d0000000e000abff3200a7ff37000e07e800b2
:10d8e0006e449000f0c2b300804f54002300320019
:10d8f000a0c7b300804f54002000320080c6b300a0
:10d90000804f54009fff3a00210020000e00780055
:10d9100072370200000000000fb99700005998000c
:10d92000f74f500097ff3e000e87e80021002000cf
:10d930000e00780072370200000000000fb9970057
:10d9400010599800b8c3b300804f54008dff3900c0
:10d950000e87e800210020000e00780072370200d8
:10d96000000000000fb9970020599800804f540024
:10d9700084ff390063074700aeff37002100200015
:10d980000e00780072370200000000000fb9970007
:10d99000705198000040e900fe4f500079ff3e00b2
:10d9a0000e87e800210020000e0078007237020088
:10d9b000000000000fb9970000599800f74f500081
:10d9c00070ff3e000e87e800210020000e00780066
:10d9d00072370200000000000fb99700105998003c
:10d9e000b2c3b300804f510066ff3900a0c7b30037
:10d9f000804f5400dfff3a007cf092000044a0000a
:10da000070f69a00dbff37007cf092000024a00043
:10da100070f69a000c4890008d0207006a00b90069
:10da2000800678001c489000890207008086460026
:10da30006168b9006a210200000000000fb9970078
:10da40000089be002c489000810207006a00b900de
:10da5000800678003c4890007d02070080864600e2
:10da60000fb997001200be00581e0200000000000f
:10da70000004be000205be006168b9006a21020010
:10da800000000000581e0200000000006022b800e4
:10da900006002000e7042400aa1e02000000000087
:10daa0000002be000203be000800be000a01be0064
:10dab0005e1f02000000000058200200000000006d
:10dac0000fb997000089be004c4890006002070023
:10dad0006a00b900800678005c4890005c0207008c
:10dae000808646000fb997001200be00581e020043
:10daf000000000000004be000205be006168b9001d
:10db00006a21020000000000581e02000000000010
:10db10006022b80006002700770b2400aa1e02002e
:10db2000000000000002be000203be000800be00ac
:10db30000a01be005e1f0200000000005820020023
:10db4000000000000fb997000089be003c4890001b
:10db5000580207000000e00004003a000fb99700e7
:10db60001200be0001f0a2000089be005c489000d7
:10db700050020700000478004c4890004d02070056
:10db8000800078000e00e800084178005502070088
:10db90000fb997002001980031019800f6fe370078
:10dba0007cf092000074a00070f69a00a10320009f
:10dbb0000e0078004406020000000000000178001a
:10dbc000100020000200e000f3fe320002005700c7
:10dbd000000044000004e9000207e80072fe37007c
:10dbe0007cf092000064a00070f69a0066fe370098
:10dbf00020fa2c00801f780040002000fc7c0200ee
:10dc0000000000000003eb00e504200044002000b9
:10dc100013042000e2fc2c0051032000c0fd2c0066
:10dc2000967c0200000000008f87e90044fe370068
:10dc30000c00fa00889fbe008a9fbe008c9fbe0029
:10dc400000067800010478000000e00002003200c5
:10dc50001004e0000f003a0030fe2c00801f780016
:10dc600010012000fc7c0200000000000003eb001b
:10dc7000e50420001401200013042000b2002d0050
:10dc800081182000c0fd2c00967c020000000000de
:10dc90008f87e9000800e00083003a00210020009f
:10dca0000c00780072370200000000008006780047
:10dcb000a105200080804000f2ff2f00f3f727002d
:10dcc000400b2000808f50006e003e000c86e80064
:10dcd000210020000c0078007237020000000000d4
:10dce00000047800b103200080804000f2ff2f0084
:10dcf000f3f7270060072000808f500061003e008e
:10dd000063064600210020000c00780072370200f4
:10dd100000000000000578006140b9006a2102009f
:10dd2000000000000004be006150b9006a2102003a
:10dd30000000000002002000832c2400f0240200d8
:10dd4000000000000001be000800be00b02002007c
:10dd500000000000e0b79f00f1b79f00581e0200ce
:10dd6000000000000004be000205be006022b800f2
:10dd700006002000e7042c00961e020000000000b0
:10dd80000000e000450034006022b80006002000da
:10dd9000e70424000800be000a01be00a01e020025
:10dda000000000000000e0003c003d006168b90098
:10ddb0006a210200000000000004be0002002000f2
:10ddc000032724006fb09700ffb09700f0240200f3
:10ddd000000000000001be000800be00b0200200ec
:10dde00000000000c0b79f00d1b79f00581e02007e
:10ddf000000000000004be000205be006022b80062
:10de00000600280067052c00961e02000000000096
:10de10000000e000210035006022b8000600280064
:10de2000670524000800be000a01be00a01e020013
:10de3000000000000000e00018003c00ac40900032
:10de4000e0c4b30080cf50000c003200f2ff2f007e
:10de5000f3f727006540400080cf500009003a00ea
:10de60000800be000a01be0003f0a2005820020014
:10de700000000000c0b79f00d1b79f004fb19700ce
:10de8000dfb197000200be004f06be004f05be0086
:10de90004f04be000080fa0000000600f2ff2f00d1
:10dea000f3f72700f7ff3700310020000c0078005f
:10deb000723702000000000080067800410b20004d
:10dec00080804000f2ff2f00f3f72700801620002b
:10ded000808f5000ebff3e006306460021002000cb
:10dee0000c00780072370200000000000004780087
:10def000b103200080804000f2ff2f00f3f72700dd
:10df000060072000808f5000deff3e006306460061
:10df1000210020000c007800723702000000000091
:10df2000000578006140b9006a210200000000008d
:10df30000004be006150b9006a2102000000000028
:10df400002002000832c2400f024020000000000c6
:10df50000001be000800be00b0200200000000006a
:10df600080bf9f0091bf9f00581e0200000000006c
:10df70000004be000205be006022b80006002000ba
:10df8000e7042c00961e0200000000000000e000e4
:10df9000c2ff34006022b80006002000e70424001d
:10dfa0000800be000a01be00a01e02000000000022
:10dfb0000000e000b9ff3d006168b9006a2102007d
:10dfc000000000000004be0002002000032724001f
:10dfd0000fb897009fb89700f024020000000000df
:10dfe0000001be000800be00b020020000000000da
:10dff000c0b79f00d1b79f00581e0200000000006c
:10e000000004be000205be006022b8000600280021
:10e0100067062c00961e0200000000000000e000d1
:10e020009eff35006022b800060028006706240025
:10e030000800be000a01be00a01e02000000000091
:10e040000000e00095ff3c00ac40900050c4b300dd
:10e0500080cf500089ff3200f2ff2f00f3f7270036
:10e06000724040007cff3700889fbe008a9fbe0040
:10e070008c1f78000005be000204be000406780074
:10e080000200e00057003200e48f540044003600e4
:10e090000c00e00036003a000a00be00581e0200e4
:10e0a000000000000002be000203be006000b800d5
:10e0b000020028006305240018240200000000006c
:10e0c0006022b80086ff230077112400c0210200df
:10e0d00000000000942402000000000032fa270033
:10e0e000b30020009c040200000000000203be00f8
:10e0f0000002be0010c2b300004c42009205220094
:10e10000030020000600be009c0402000000000086
:10e110000203be000002be0011c2b3000140420073
:10e1200010449800b2052000030020000600be0045
:10e130009c040200000000000203be000002be00ba
:10e1400011c2b30001404200204498000140430046
:10e15000304498000040eb004044980008007800ec
:10e160004f0678004f05be004f04be0000000600b9
:10e170000a00be00581e0200000000006022b80025
:10e1800006002800670624005e1f02000000000051
:10e190006022b80086ff230077102400cbff3700f1
:10e1a000891f780081012d00811f78001001200057
:10e1b000fc7c02000000000009037800e504200058
:10e1c000140120001304200092042d00512120008e
:10e1d000c0fd2c00967c020000000000e487570080
:10e1e000abff370060052d00801f78001001200074
:10e1f000fc7c0200000000000003eb00e5042000ae
:10e20000140120001304200092042d00112120008d
:10e21000c0fd2c00967c0200000000008f87e90002
:10e2200099ff3700889fbe008a9fbe008c9fbe006a
:10e230000004be000000e00003003200104078003f
:10e240000004e00010003a00d0072d00801f780085
:10e2500010012000fc7c0200000000000003eb0025
:10e26000e50420001401200013042000520a2d00b0
:10e27000a1242000c0fd2c00967c020000000000bc
:10e280008f87e900184078000000fb00b4052000eb
:10e290000480b90052442f00020040006101b9001f
:10e2a000184090000000fb00cf80de00020040001c
:10e2b000838048000401b8000488b90080814100cf
:10e2c00056442f00f7ff2f000201430083814b00cb
:10e2d000284090000000fb00cf80de0002004000dc
:10e2e000838048000401b800048ab9008481410099
:10e2f0000201430083814b00384090000000fb0086
:10e30000cf80de0002014000838148001202b1008c
:10e310000380b1000900e0002e003a000200be00b8
:10e320001c240200000000006022b80086ff2300c9
:10e3300077112400aa1e0200000000000002be00a7
:10e340000203be006000b80002002800630524003c
:10e350001824020000000000582002000000000005
:10e360000006be00581e0200000000000004be00af
:10e370000205be006022b8000600280067052c00d8
:10e38000961e0200000000006022b800060028006f
:10e39000670524000000e000060035000800be000c
:10e3a0000a01be00a01e0200000000000000e00004
:10e3b00006003400f0ff2f00f1f727004f06be00e3
:10e3c0004f05be004f04be00000006000c00be005a
:10e3d000faff37000200be001c240200000000000b
:10e3e0006022b80086ff230077102400aa1e0200d6
:10e3f000000000006022b8000600280067062c001c
:10e400005e1f020000000000582002000000000013
:10e410000006be00581e0200000000000004be00fe
:10e420000205be006022b8000600280067062c0026
:10e43000961e0200000000000000e000ddff350035
:10e440006022b8000600280067062400d3ff3700ca
:10e450000041780000cdb30000404100e94f50007a
:10e4600005003e000280fb0002fd2f0082004000fc
:10e470000100780000000600f0cbb300004041002e
:10e48000e94f500003003e000280fb00f2fb2f002a
:10e49000f6ff370000cbb300004041008000eb00e6
:10e4a000e94f5000f2ff3e000280fb0002fb2f000c
:10e4b000eeff37008040780000cdb30000c0400080
:10e4c000e94f50000400360042062000c0c4b300eb
:10e4d00080cf500001003a000001eb0002007800fc
:10e4e00000000600889fbe008a9fbe008c9fbe0071
:10e4f0008e1f78008004780001447800024778007d
:10e500000000e00062003200994044007cc45000ea
:10e5100002c3b30002c04000e94f500056003e0065
:10e5200000cbb30000444400194090007c465000ea
:10e53000b0c3b300804f56000200360040ccb30099
:10e540000046460029409000fc4650000800fb00b1
:10e55000cf80de006a210200000000000804e00015
:10e5600040003500581e0200000000000004be00fc
:10e570000205be000c00fb00cf80de006a21020015
:10e58000000000000c04e00031003500581e0200bd
:10e59000000000006022b80006002000e70424000c
:10e5a000aa1e0200000000000002be000203be001e
:10e5b0000800be000a01be005e1f0200000000004d
:10e5c0000004be000205be000d00fb00cf80de008f
:10e5d0006a210200000000000d04e0001700350071
:10e5e000581e0200000000006022b800060027004c
:10e5f000770b2400aa1e0200000000000002be00eb
:10e600000203be000800be000a01be005e1f020039
:10e610000000000058200200000000000e04e0008e
:10e620000100320001f0a2004f0778004f06be0043
:10e630004f05be004f04be0000000600020020008f
:10e6400003382400b020020000000000e4ff37007f
:10e650000200200003382400b02002000000000067
:10e66000caff37000200200003382400b020020057
:10e6700000000000bbff370062c2b30002c04000d0
:10e68000e94f5000a8ff3e0000447800a6ff370085
:10e69000200b2d00801f7800c0012000fc7c0200b0
:10e6a000000000000003eb00e5042000c40120008e
:10e6b00013042000c20d2d0001292000c0fd2c00f4
:10e6c000967c0200000000008f87e9008eff370073
:10e6d000581e0200000000006022b8000600200062
:10e6e00007fd2300c02102000000000022240200d8
:10e6f000000000001002b000000006000042780098
:10e70000f602200042de2c008001eb00e5ef2c0039
:10e71000850f510009003100924f52001000320065
:10e7200012409000804f5200060032006301410009
:10e730008301e800850f5100f7ff390006007800db
:10e74000000006002240900080cf5000f7ff3a0002
:10e7500010022000030040000003ea00f7ff37002a
:10e760002240900080cf5000edff3a0016022000ba
:10e7700003034300f1ff3700ec874700889fbe008a
:10e780008a9fbe008c9fbe008e1f78008006780096
:10e79000010778000000e000730132000100e00092
:10e7a00069013200621520000201400082bf9f0013
:10e7b00029802000e0ff2f00800878000006eb0091
:10e7c00028938000e00f14001900310009599000cf
:10e7d0008280fb0090022000808f50003e013200ba
:10e7e00062003c000080e900808f50004100320050
:10e7f0000000e800808f5000150032000280fb000e
:10e80000801f780060172d00801f780050032000c3
:10e81000fc7c020000000000e48757002893800081
:10e820000c06e800fc844400880f5600e7ff39001e
:10e83000008feb00109380004f0778004f06be005a
:10e840004f05be004f04be00cf00b100000006001f
:10e85000195890000080fb000058a3000c003a00fb
:10e860000048a3000e003200090078008e04020068
:10e8700000000000000178008d0078000900780099
:10e88000243b0200000000000000e000e3ff3a002b
:10e890000c0f7800195890006f006000e6ff3700f9
:10e8a0000d0078008e0402000000000000017800d6
:10e8b0008d00780009007800243b02000000000071
:10e8c0000000e000d5ff3a00195890000068a3004e
:10e8d000efff3200e94090008180fb007d40900016
:10e8e0000000d1006f006000808f5000cbff3a0025
:10e8f000e7ff3700195890000080fb000058a30084
:10e90000e3ff3a000048a300060032000900780047
:10e910008e0402000000000000017800e88046003c
:10e92000d6ff370068844600080078008e04020095
:10e9300000000000000178008800780009007800dd
:10e94000243b0200000000000000e000b3ff3a009a
:10e95000195890000068a300cdff3200e9409000f4
:10e960008180fb007d489000ddff3700b002200071
:10e97000808f5000b4003200500035000000e800e5
:10e98000808f50009dff3a007df092000018a30098
:10e99000a3ff32005212e2004300320082a5800041
:10e9a00093a58000a0a58000b1a580008fba970034
:10e9b00025029000b5029000849fbe006fb29700c0
:10e9c0001403be000002be00fc8057007880570090
:10e9d000e239020000000000e48757000000e00078
:10e9e0002a003a004fb59700dfb597001901be0025
:10e9f0000a00be0074250200000000000000e000d4
:10ea000086ff350039019000c90190000a00be0060
:10ea1000ec240200000000000000e0007fff3c004a
:10ea20006fb59700ffb5970069019000f90190005c
:10ea30000a00be0074250200000000000000e00093
:10ea400076ff350019089000a9089000581e0200b2
:10ea5000000000006022b8006033b8007825020092
:10ea6000000000000000e00089ff3200190990005a
:10ea7000a90990000a00be00ec240200000000007a
:10ea80000000e00065ff3c0081ff3700c51a2d0043
:10ea9000851f780030032000fc7c0200000000008d
:10eaa0008f87e9005dff3700c2918000d39180001d
:10eab000e0918000f1918000bcff37007df0920072
:10eac0000018a30056ff3200194078008080fb0038
:10ead000e48f50005000320023003c00e28f5000d1
:10eae0001800320011003c00e18f50000600320097
:10eaf0000080fb00801f7800f01c2d00801f780034
:10eb00002003200042ff37000fb997001200be001b
:10eb100039019000c9019000742502000000000036
:10eb20000000e0003eff340059ff37008fba970025
:10eb300025009000b500900069019000f901900057
:10eb4000f5ff37000fba97001400be00390190009e
:10eb5000c901900074250200000000000000e000e0
:10eb60002fff3400f1ff3700e68f50002100320004
:10eb7000e58f50001a003400e78f50001400320077
:10eb8000e88f5000daff3a000fba97001400be0079
:10eb900039019000c90190007425020000000000b6
:10eba0000000e0001eff34008fba9700250090009f
:10ebb000b500900069019000f9019000ec2402007a
:10ebc000000000000000e00015ff3d0030ff3700ae
:10ebd0000fb9970022009000b2009000f5ff3700b7
:10ebe0000fba97001400be0039019000c9019000cf
:10ebf000f2ff37008fba97001500be003901900070
:10ec0000c9019000ec240200000000000000e000b8
:10ec100003ff3d00eeff37000fb997001200be0062
:10ec200039019000c9019000ec24020000000000ae
:10ec30000000e000fafe3d000fba970024009000ab
:10ec4000b4009000bcff37007df092000018a300d4
:10ec5000f3fe32008fb897001105be001901be0007
:10ec60000a00be00ec240200000000000000e000ea
:10ec7000ebfe3c0069019000f90190000a00be0023
:10ec800074250200000000000000e000e4fe3500f2
:10ec90000fb9970022059000b2059000390190004d
:10eca000c90190000a00be007425020000000000a7
:10ecb0000000e000dafe350019099000a909900073
:10ecc0000a00be00ec240200000000000000e0008a
:10ecd000d3fe3c00eefe37007df092000018a3004a
:10ece000cffe320069029000f902900039019000d5
:10ecf000c90190008fb8970021009000b1009000ea
:10ed0000809fbe006fb097001003be00fc805700cc
:10ed100078805700e239020000000000e4875700c5
:10ed20000000e00004003a001901be006fb0970037
:10ed3000ffb0970050ff3700c11a2d00811f7800e7
:10ed40001003200054ff3700b1202d00811f7800f0
:10ed5000e0022000fc7c0200000000001000200007
:10ed60008f87e900b4fe370070232d00801f7800e4
:10ed7000d0022000f7ff3700889fbe008a9fbe00a8
:10ed80008c9fbe000004be00820578000000e000f9
:10ed9000810032000900e0006f0032000b08a30080
:10eda0005c003a00fc0720000c00780032e0b7005d
:10edb0004d0320009d467800f00f200034e0b7009e
:10edc0000005eb008b05d100e08f15004b003100f2
:10edd000183b88000c00780064e7b700400424006a
:10ede000003b880021042000914078008180fb00d6
:10edf000c508de00010078006ff5b70000ceb30053
:10ee00004260b70050c5b30066e7b700a0cab300c0
:10ee100066e7b70061e7a800c508dd0042c0bf0093
:10ee20007f4060000140700042e0b7006007e200f0
:10ee3000feff350019017800020cbb0040002400e1
:10ee4000003b880021042000914078008180fb0075
:10ee5000c508de00010078006ff5b70000ceb300f2
:10ee60004260b70050c5b30066e7b700a0cab30060
:10ee700066e7b70061e7a800c508dd0042c0bf0033
:10ee80007f4060000140700042e0b7006007e20090
:10ee9000feff350018007800820f5000120032008b
:10eea000821f7800801f7800881f780010262d00b0
:10eeb000801f780050172000fc7c0200000000003a
:10eec0001803780065052000541720006304200013
:10eed000a22b2d0021192000802c2d00967c0200f1
:10eee00000000000e88757000884e8008984e800f3
:10eef0000a05e8008b0f5500b5ff39000d007800ba
:10ef000034e0b7004f06be004f05be004f04be0000
:10ef1000000006008b1f7800002d2d00801f780058
:10ef200080052000fc7c0200000000000b0378003c
:10ef3000650520008405200063042000a22b2d001d
:10ef4000a1142000802c2d00967c020000000000ff
:10ef5000e487570093ff370040302d00801f780072
:10ef600080052000fc7c0200000000000003eb0094
:10ef7000e50420008405200063042000a22b2d005e
:10ef800061142000802c2d00967c020000000000ff
:10ef90008f87e90081ff370080322d00801f7800c5
:10efa00080052000fc7c0200000000000003eb0054
:10efb000e50420008405200063042000a22b2d001e
:10efc00021142000802c2d00967c020000000000ff
:10efd0008f87e9006fff37005000fa00889fbe005e
:10efe0008a9fbe008c1f7800209380000000e00004
:10eff00013003a0010938000c1342d00e40f50003c
:10f000000400320011352d00e80f500001003200dd
:10f0100061352d00811f780080352d00801f78001c
:10f02000b67d020000000000e48757004f0678001c
:10f030004f05be004f04be000080fa00000006002d
:10f04000801f7800e1382d00811f7800b67d020016
:10f0500000000000b03a2d00801f7800013b2d0019
:10f06000811f7800803b2d00801f7800f13b2d0030
:10f07000811f7800b67d020000000000903d2d0049
:10f08000801f780011352d0010938000e80f50008c
:10f0900001003200c1342d00811f7800213e2d0077
:10f0a000811f7800b67d0200000000008005eb00a3
:10f0b00028802000f28757006412e200dbff320054
:10f0c00074054700890220008e844400cc03200090
:10f0d0000e0646000e007800090009000018eb003b
:10f0e0000a007800090009000018eb000900780008
:10f0f000090009000018eb000c0078000900090065
:10f100000018eb00085990008280fb00900220005c
:10f11000808f5000d100320052003c000080e90096
:10f12000808f5000270032000000e800808f5000e0
:10f1300024003200004eeb00804ceb00004deb0051
:10f14000004feb00985890008c1f7800891f7800c2
:10f150008a1f78008e1f780001007800000fb2002f
:10f16000801f78000280fb00de000700801f78000f
:10f17000185890006f00600011352d00e80f500006
:10f1800004003200c1342d00e40f500001003200b1
:10f1900061352d00811f7800d13e2d00811f780040
:10f1a000b67d020000000000f08757008b05e800e4
:10f1b0007c04440020938000808f5500c5ff3900f7
:10f1c0009aff3700985890000180fb000058a30078
:10f1d00003003200a0022000000f7800daff3700a1
:10f1e0000048a3001a003a000068a3000e00320095
:10f1f000684090000080fb00801f7800881f780026
:10f2000060002000801f7800b1402d00811f780031
:10f210000e0078006006020000000000e88757003a
:10f2200008599000c7ff3700881f78006000200051
:10f23000801f780031412d00811f78000e0078007a
:10f240006006020000000000e6875700f4ff370068
:10f25000881f780060002000801f780081412d0009
:10f26000f5ff3700b0022000808f500052003200be
:10f27000300035000000e800808f5000adff3a00fc
:10f280001800be00581e020000000000809fbe0053
:10f29000829fbe00e0412d00801f78000e007800a4
:10f2a000600602000000000038009000c8009000d6
:10f2b000581e020000000000809fbe00829fbe001a
:10f2c000c1422d00811f78000a007800600602000c
:10f2d0000000000068009000f8009000581e020036
:10f2e00000000000809fbe00829fbe00a0432d0052
:10f2f000801f78000900780060060200000000000e
:10f3000018089000a8089000581e02000000000095
:10f31000809fbe00829fbe0061442d00811f780047
:10f320000c00780060060200000000008f02b100af
:10f33000bbff37001880fb000000d00041162d00f5
:10f34000e09f780020452d00801f78000e00780097
:10f35000600602000000000038009000c800900025
:10f36000581e020000000000809fbe00829fbe0069
:10f37000c1452d00811f78000a0078006006020058
:10f380000000000068009000f8009000581e020085
:10f3900000000000809fbe00829fbe00b0462d008e
:10f3a000801f78000900780060060200000000005d
:10f3b000f88757009aff37001800be00581e020059
:10f3c00000000000809fbe00829fbe0091472d007c
:10f3d000811f78000e007800600602000000000027
:10f3e00038009000c8009000581e02000000000085
:10f3f000809fbe00829fbe0090482d00801f780035
:10f400000a0078006006020000000000680090001a
:10f41000f8009000581e020000000000809fbe000f
:10f42000829fbe0091492d00811f7800090078005d
:10f43000600602000000000018089000a808900074
:10f44000581e020000000000809fbe00829fbe0088
:10f45000904a2d00801f7800b1ff37001800be00d1
:10f46000581e020000000000809fbe00829fbe0068
:10f47000804b2d00801f78000e007800600602008f
:10f480000000000038009000c8009000581e0200e4
:10f4900000000000809fbe00829fbe00c1452d007d
:10f4a000811f78000a00780060060200000000005a
:10f4b00068009000f8009000581e02000000000054
:10f4c000809fbe00829fbe00b0462d00801f780046
:10f4d000090078006006020000000000fe87570067
:10f4e0004fff3700800178000082eb000001eb0045
:10f4f0006410b80085122d0005004000908f510067
:10f500000b0032000201e800e80f5100f8ff36005e
:10f51000c0572100e10f4200040032006420b8000f
:10f5200062122d0060007900000006000000060055
:10f5300002027800f6ff3700410320009140780076
:10f54000f00f200034e0b7002280200000002f00e0
:10f5500077050900305978000100780034e0b700e1
:10f5600000000600881f7800480320001844780037
:10f57000f30f20008001fd0034e0b7008001fd00a2
:10f5800018050200000000000800780034e0b70011
:10f590004f04780000000600f0874700889fbe00f7
:10f5a0008a9fbe008c9fbe008e1f7800c1b79f004f
:10f5b000a2002000110009000280d800e1e79f00ae
:10f5c000110009000280d800d1e79f001100090056
:10f5d0000280d800c1e79f00f0aa800001ab800044
:10f5e000f0b79f0081bf9f00c27020000300200081
:10f5f0006e24020000000000d0b79f00e1b79f001a
:10f60000d4a2a8006000b8005fb19700efb19700e6
:10f61000820f5000838f58000300310061004000ca
:10f62000e0804800f8ff3700d4a2a9006044b80089
:10f63000c2702000030020007fb097008fb89700b1
:10f640006e24020000000000800f5400818f5c00d7
:10f650000300310061044400e0844c00faff3700ed
:10f66000d4a2a8006044b800c270200003002000ab
:10f670007fb097008fb897006e2402000000000052
:10f68000800f5400818f5c0003003100610444004e
:10f69000e0844c00faff3700d4a2a9006044b8000f
:10f6a000c2702000030020007fb097008fb8970041
:10f6b0006e24020000000000800f5400818f5c0067
:10f6c0000300310061044400e0844c00faff37007d
:10f6d000d4a2a8006044b800c2702000030020003b
:10f6e0007fb097008fb897006e24020000000000e2
:10f6f000800f5400818f5c000300310061044400de
:10f70000e0844c00faff3700d4a2a9006044b8009e
:10f71000c2702000030020007fb097008fb89700d0
:10f720006e24020000000000800f5400818f5c00f6
:10f730000300310061044400e0844c00faff37000c
:10f74000d4a2a8006044b800c270200003002000ca
:10f750007fb097008fb897006e2402000000000071
:10f76000800f5400818f5c0003003100610444006d
:10f77000e0844c00faff3700d4a2a9006044b8002e
:10f78000c2122000030020007fb097008fb89700be
:10f790006e24020000000000800f5400818f5c0086
:10f7a0000300310061044400e0844c00faff37009c
:10f7b0000007eb00fc815700830647001d407800de
:10f7c0000004e000490032000006eb002100320096
:10f7d00062382000030020007fb097008fb89700a8
:10f7e0006e240200000000000005be00d4a2a800a4
:10f7f0006000b8008a0f50008b8f58000300310062
:10f8000061004000e0804800faff3700d4a2a90060
:10f810006044b80062382000030020007fb09700e9
:10f820008fb897006e24020000000000800f540083
:10f83000818f5c000300310061044400e0844c00cf
:10f84000faff37000c06e8001d80fb00800f560011
:10f85000e6ff35006044b800c2122000030020001b
:10f860007fb097008fb897006e2402000000000060
:10f87000800f5400818f5c0003003100610444005c
:10f88000e0844c00faff37000e07e800e20f570053
:10f89000c8ff34004fb097000000e0000d003200b8
:10f8a0006044b800c2122000030020007fb097001f
:10f8b0008fb897006e24020000000000800f5400f3
:10f8c000818f5c004eff310061044400e0844c00f5
:10f8d000faff37004f0778004f06be004f05be0005
:10f8e0004f04be000f01b10000000600d4a2a80022
:10f8f0006044b800120e2000030020007fb0970083
:10f900008fb897006e24020000000000800f5400a2
:10f91000818f5c000300310061044400e0844c00ee
:10f92000faff3700d4a2a900caff3700889fbe00a3
:10f930008a9fbe008c9fbe008e1f78000007780053
:10f940008106780002067800830578008404780038
:10f950000505780006047800010220001000200050
:10f96000984b0200000000000000e000130032008d
:10f970005812e20011003200a15621009140780097
:10f9800040c4b30080cf50000c003200881f7800c4
:10f990008a1f7800891f78008b1f78008c1f7800e1
:10f9a0008d1f78008e1f7800404c2d00801f78003e
:10f9b000b67d020000000000f0875700d192800061
:10f9c00009007800f4fe07000000fe004f077800f1
:10f9d0004f06be004f05be004f04be0000000600eb
:10f9e000d422ef00f0f02f0090168800d4a2a900d6
:10f9f000d4e2a900000006000000fa00881f780089
:10fa0000000478005812e2000b003200a1562100d9
:10fa10009140780040c4b30080cf5000060032000f
:10fa20000102200010002000984b0200000000009e
:10fa30000000e0000b003a00301f2000800f54004f
:10fa4000030036004f0478000080fa000000060032
:10fa50008000eb0008007800cc7a02000000000073
:10fa6000f8ff37003fb897000000e0003000320098
:10fa7000823e2000110009000284d800301f2000bf
:10fa8000808f50002400360002102100804f2d008e
:10fa900005000900305978005800200002102100ac
:10faa000020244006108b8008001eb00320020002f
:10fab00060380200000000006304440001102100cf
:10fac00001004400a1c3b30001587800fac05000ff
:10fad000015878000048eb000884e800c1122000bb
:10fae000888050000210210002004400ea81570083
:10faf0003fb99700a4060200000000000004440083
:10fb0000080178000110210010002000804302004d
:10fb100000000000cbff370002102100e04f2d0055
:10fb2000060009003059780068002000dbff37002c
:10fb300051502d00811f7800c0122000aeff070039
:10fb400008037800e5042000c4122000030520000b
:10fb500002522d005104200060522d00967c0200bc
:10fb6000000000008f87e900c1ff37000000fa00a5
:10fb70005812e2001a003200a1562100914078008c
:10fb800040c4b30080cf50001500320001022000b5
:10fb900010002000984b0200000000000000e00070
:10fba0000f0032004fb897000000e0000e00320056
:10fbb000c0122000e88157004fb9970080007800fc
:10fbc00000102100a40602000000000000017800df
:10fbd00001102100100020008043020000000000fe
:10fbe0000080fa0000000600e0522d00801f78001f
:10fbf000d012200080ff07000003eb00e504200086
:10fc0000d412200003052000a2542d00e10720009b
:10fc100060522d00967c0200000000008f87e900f2
:10fc2000e3ff37000c00fa00889fbe008a9fbe00e9
:10fc30008c1f7800000478000000e0008e00320085
:10fc40000081eb000802780063002000c810dd008e
:10fc50003480fb00808070004810de000000d0007f
:10fc6000826d290002004000108168008301e900d4
:10fc7000e18f4100f5ff3a00680244006300200074
:10fc8000c810dd003480fb00808070004810de006a
:10fc90000000d000866d2900060040001081680039
:10fca0008301e900e18f4100f5ff3a00820178000d
:10fcb00072024400080990000201e900e10f4100ce
:10fcc0000b003200c818dd003480fb00808070001b
:10fcd0004818de000000d000836d290003004000ba
:10fce000908168000201e900e10f4100f5ff3a0050
:10fcf000784090000000d1006f406000a0ef9f00ae
:10fd00000040eb00b0ef9f00c0ef9f0003057800bc
:10fd1000f681570022002000c850dd003380fb0030
:10fd2000808070004850de000000d000846d290003
:10fd300004004000108568000201e900e10f410065
:10fd4000f5ff3a0002067800abd720008000eb00f8
:10fd5000520920002b009000800f55004400320013
:10fd60008100e800e6854500828f5000f9ff3600eb
:10fd7000c850020000000000f0b79f0081bf9f0044
:10fd800092bf9f00a3bf9f00f8aa800009ab80002c
:10fd90000800be001c24020000000000e00f540018
:10fda000e08f5c002c0035000002be000203be00a4
:10fdb0007fb097008fb897001fb99700afb9970031
:10fdc000aa1e020000000000222402000000000021
:10fdd0000002be00e10f4600100032001b01be0011
:10fde000a092800000004100e08049001200200045
:10fdf000840f5000858f580002003e00848dbe00a5
:10fe00000001eb00020078004f0678004f05be00ad
:10fe10004f04be000080fa0000000600f387800057
:10fe20006618b800e6d72000060140000a097800ed
:10fe3000a2d72000020040000488be008301e80031
:10fe4000f387880050092000808f5100ecff3400b8
:10fe5000fe30ef00eaff37006022b8000600200005
:10fe6000071f24005e1f020000000000ceff3700c5
:10fe700001067800beff370020552d00801f780056
:10fe800050192000fc7c0200000000000003eb0081
:10fe9000e5042000541920004304200092572d004f
:10fea0006103200040582d00967c020000000000f5
:10feb0008f87e90062ff37000002be000201e900ff
:10fec000e10f41000a003200c820dd003580fb0050
:10fed000808070004820de000000d0006080790043
:10fee000008268000201e900e10f4100f6ff3a00dc
:10fef00004007800000006004200200081572f0017
:10ff0000c02221007300070042002000c1572f00cb
:10ff1000002321006f0007004200200001582f003d
:10ff2000402321006b0007004200200041582f00b1
:10ff300080232100670007004200200081582f0025
:10ff4000c02321006300070082002000c1582f0059
:10ff5000002421005f0007002200200041592f00eb
:10ff6000802421005b0007002200200061592f003f
:10ff7000a0242100570007002200200081592f00f3
:10ff8000c02421005300070022002000a1592f00a7
:10ff9000e02421004f00070022002000c1592f005b
:10ffa000002521004b00070022002000e1592f000e
:10ffb000202521004700070022002000015a2f00c1
:10ffc000402521004300070022002000215a2f0075
:10ffd000602521003f00070022002000415a2f0029
:10ffe000802521003b00070022002000615a2f00dd
:10fff000a02521003700070022002000815a2f0091
:020000040001f9
:10000000c02521003300070022002000a15a2f0044
:10001000e02521002f00070022002000c15a2f00f8
:10002000002621002b00070022002000e15a2f00ab
:1000300020262100270007001193800000052000e2
:10004000808f50002100320006003600400620005c
:10005000808f5000030032006c004000808f500001
:100060001a00320040002000109388002200200077
:10007000015b2f004026210016000700020420002b
:10008000215b2f0060262100120007000001eb0019
:100090006810b80063262100030040001004e0004f
:1000a000030032000201e800e70f5100f8ff3400be
:1000b00002007800d2f2b7004673ef00c2022000bf
:1000c000215f2f00602a21000200370080002000fd
:1000d000e5ff3700881f78004803200018447800a7
:1000e000f30f20008001fd0034e0b7008001fd0027
:1000f00018050200000000000800780034e0b70096
:100100004f04780000000600889fbe008a9fbe0052
:100110008c9fbe000004be00820578000000e00055
:10012000810032000900e0006f0032000b08a300dc
:100130005c003a00fc0720000c00780032e0b700b9
:100140004d0320009d467800f00f200034e0b700fa
:100150000005eb008b05d100e08f15004b0031004e
:10016000183b88000c00780064e7b70040042400c6
:10017000003b880021042000914078008180fb0032
:10018000c508de00010078006ff5b70000ceb300af
:100190004260b70050c5b30066e7b700a0cab3001d
:1001a00066e7b70061e7a800c508dd0042c0bf00f0
:1001b0007f4060000140700042e0b7006007e2004d
:1001c000feff350019017800020cbb00400024003e
:1001d000003b880021042000914078008180fb00d2
:1001e000c508de00010078006ff5b70000ceb3004f
:1001f0004260b70050c5b30066e7b700a0cab300bd
:1002000066e7b70061e7a800c508dd0042c0bf008f
:100210007f4060000140700042e0b7006007e200ec
:10022000feff350018007800820f500012003200e7
:10023000821f7800801f7800881f7800c0582d002a
:10024000801f780050172000fc7c02000000000096
:10025000180378006505200054172000630420006f
:10026000425e2d00f1152000105f2d00967c0200eb
:1002700000000000e88757000884e8008984e8004f
:100280000a05e8008b0f5500b5ff39000d00780016
:1002900034e0b7004f06be004f05be004f04be005d
:1002a000000006008b1f7800805f2d00801f780003
:1002b00080052000fc7c0200000000000b03780099
:1002c000650520008405200063042000425e2d00a7
:1002d00061112000105f2d00967c020000000000dc
:1002e000e487570093ff3700b0622d00801f78002d
:1002f00080052000fc7c0200000000000003eb00f1
:10030000e50420008405200063042000425e2d00e7
:1003100021112000105f2d00967c020000000000db
:100320008f87e90081ff3700e0642d00801f78008f
:1003300080052000fc7c0200000000000003eb00b0
:10034000e50420008405200063042000425e2d00a7
:10035000e1102000105f2d00967c020000000000dc
:100360008f87e9006fff3700881f7800a1562100b2
:100370009140780070c4b30080cf500089003200f3
:10038000a1562100914078006340500080cf50007a
:10039000840032000102200010002000984b02006f
:1003a000000000000000e0007e0032004e12e2007b
:1003b0008c00320010672d00801f78005012e20080
:1003c0008600320010672d00801f78005612f8005a
:1003d0005412f8004c12f8004a12f800a091800064
:1003e000b1918000809fbe0080918000919180003b
:1003f000809fbe006091800071918000809fbe0050
:10040000e0918000f1918000581e02000000000081
:10041000809fbe00829fbe00c0918000d19180006d
:10042000581e020000000000809fbe00829fbe0098
:100430004812f80001242100811f7800620020008a
:10044000821f780040672d00801f7800b67d020073
:10045000000000000f03b100d2d2bf0041742d0094
:1004600001003a0051742d00811f78000080fb00cc
:10047000801f7800c2742d00821f7800b67d0200b4
:10048000000000000004eb00e6875700d2d2bf0056
:100490000080fb00e00f100015003d000000e900a7
:1004a00041742d00800f540001003200e1752d00d1
:1004b000811f78006840b80062262100821f40003a
:1004c00080002000801f780001762d00811f7800b9
:1004d000b67d020000000000e88757000804e8002d
:1004e000d2d2bf000080fb00800f5400ebff35002c
:1004f000622a2100821f780070762d00801f78000c
:10050000b67d02000000000010938000c1772d002e
:10051000e40f50000400320011782d00e80f500065
:100520000100320061782d00811f78006412f8000c
:100530005c12e2002700320080782d00801f7800d6
:100540005a12e2002100320080782d00801f7800ce
:100550006012e2001b00320080782d00801f7800be
:100560005e12e2001500320080782d00801f7800b6
:100570005212e2000f00320080782d00801f7800b8
:100580005812e2000900320080782d00801f7800a8
:10059000c1782d00811f7800b67d020000000000a8
:1005a000f68757004f04780000000600e0822d0017
:1005b000f6ff3700e0822d00f0ff3700e0822d00cb
:1005c000eaff3700e0822d00e4ff3700e0822d00d3
:1005d000deff3700e0822d00d8ff370010832d00aa
:1005e00079ff370010832d0073ff3700889fbe000e
:1005f0008a9fbe008c1f78005101200000db210083
:100600009900070000057800f50f5000090032003e
:100610000003780065052000c41a2000730520003f
:1006200082832d007103200010842d00967c02002f
:100630000000000051002000e0db210072370200c2
:10064000000000000004be00000678002bdb210043
:1006500042002000c1842d000b007800d00502006c
:10066000000000000000e0003400320052002000d2
:1006700011852d000b007800d0050200000000005d
:100680000000e00018003a000800e00002003a0014
:100690000028ef00d8ff3700880078002080200075
:1006a00032000700880f5000090032000003780074
:1006b00065052000d41a20007305200082832d00d8
:1006c000b104200010842d00967c02000000000080
:1006d000c2012000110009000286d8000001780044
:1006e00002408800c4ff3700a200200071852d0061
:1006f0000b007800d0050200000000000000e000c0
:100700000a0032000a03780065052000e41a200080
:100710007305200082832d008300780010842d0053
:10072000967c020000000000b3ff37004f067800ff
:100730004f05be004f04be00000006008800780090
:10074000c022210009000700880f5000aaff3200d4
:100750000003780065052000c41a200073052000fe
:1007600082832d0011042000ecff3700889fbe001b
:100770008a9fbe0000057800010478000000e000b8
:100780002f0032000800e0002300320088047800c7
:100790008005eb000800e00011003400011020008b
:1007a00000db21003000070000047800e40f500057
:1007b0000f003400640454000801780021db21009c
:1007c0000a00780018050200000000000805450036
:1007d00088854500888454004240a900efff3c0012
:1007e0000b0078004f05be004f04be00000006005d
:1007f0000003780065052000d41a2000730520004e
:1008000022862d003108200010842d00967c0200e5
:1008100000000000e7ff37000003eb006505200043
:10082000c41a20007305200022862d002107200015
:1008300010842d00967c020000000000d3ff3700da
:100840000003eb00e5042000c41a2000730520001b
:1008500022862d00d106200010842d00967c0200f7
:1008600000000000c7ff37000800fa00889fbe00a4
:100870008a9fbe008c9fbe000005be000000e00005
:1008800081003200e48f5500750036005c002000c6
:10089000615bb80004d420000430b8006331b900b3
:1008a0000281400004bab9008400410062918000d6
:1008b000739180006e2402000000000080bf9f0042
:1008c00091bf9f00e90f5000e08f580004003c00ea
:1008d000a00020000100200080bf9f0091bf9f006a
:1008e000800c200001002000e0b79f00f1b79f00be
:1008f0008a86e80028002000f4815700080178006b
:100900008a00780010002000dc4102000000000096
:10091000880f5000090032000003780065052000b0
:10092000e41a20007305200002872d00610c2000ce
:1009300010842d00967c0200000000009a80fb00cd
:10094000c808dd001a4090000080fb008084700021
:100950008b8f540038003e000984e900f081570075
:10096000080178008d00780010002000dc410200b2
:1009700000000000880f50000900320000037800da
:1009800065052000041b20007305200002872d0050
:10099000210d200010842d00967c02000000000034
:1009a0000080eb00836d2900090178008a0078003f
:1009b0005c7f0200000000000000e0001700320031
:1009c0000c06e9001200200071832d00020078005f
:1009d00080430200000000000c00e000c5ff3c0066
:1009e0000003eb0065052000f41a200073052000c9
:1009f00002872d00d10e200010842d00967c02006d
:100a0000000000000000eb004f06be004f05be00d6
:100a10004f04be000080fa00000006001200200013
:100a200061832d0002007800804302000000000076
:100a300009007800f4ff37000903780065052000fd
:100a4000f41a20007305200002872d00b10c20004d
:100a500010842d00967c020000000000beff3700cd
:100a60000003eb0065052000d41a20007305200068
:100a700002872d00e10a200010842d00967c0200e0
:100a80000000000081ff37000003eb00e5042000b8
:100a9000c41a20007305200002872d00810a20005f
:100aa00010842d00967c02000000000075ff3700c6
:100ab000f2874700889fbe008a9fbe008d1f780086
:100ac0008e1f780000047800010578008206780007
:100ad0000000e00032023200e90f55001f0234002e
:100ae0000d00e0000d023200630744001e41780053
:100af00070c4b300804f51001301320020c5b30011
:100b0000804f510004003a009e4090006540500024
:100b100080cf50000c0032000040eb00c05e980017
:100b200000c0eb00b05e9800d1ff2f0001007800fc
:100b30004f077800cf0678004f05be004f04be0077
:100b40002f01b10000000600ae4090006a40500046
:100b500080cf5000f0ff3a008a00e9000800e8006a
:100b60001f0207008080eb000000e000efff35006f
:100b7000c10220000e0078004406020000000000c0
:100b80000007e8001e80fb006a00b9001e419000cb
:100b90000041410070415100825e98002e4090005b
:100ba0000080fb006a00b9003e4190000041410016
:100bb00070415100925e98004e4090000080fb0012
:100bc0006a00b9005e41900000414100704151004f
:100bd000a25e9800c10220000e00780044060200c8
:100be000000000000007e8009e40780010c4b30039
:100bf00080cf5000d200320060c5b30080cf5000db
:100c0000cd0032000040eb00b05e9800c102200031
:100c10000e00780044060200000000000004780086
:100c20000007e8001e81fb006a11b9001e40900019
:100c30000080fb00020040000021b100cf80de00f8
:100c40006a210200000000000005be0063044400a9
:100c50006011b8008000eb0008007800c2020200ba
:100c6000000000005820020000000000e0b79f00d4
:100c7000f1b79f00c10220000e0078004406020078
:100c8000000000000007e8000a00be00581e020035
:100c9000000000000004be000205be006fb0970017
:100ca000ffb09700581e0200000000006022b8004c
:100cb00006002000e7042400aa1e02000000000035
:100cc0000002be000203be000800be000a01be0012
:100cd0005e1f02000000000058200200000000001b
:100ce0000001be00808ebe0030c5b3009e4f1000d4
:100cf00089003200c10220000e0078004406020084
:100d000000000000000478000007e8001e81fb00de
:100d1000400620000091b9001e4090000080fb00ba
:100d20006a00b900000141002e4090000080fb00e5
:100d30000001410000b32e00000141006110b90024
:100d40006a210200000000000005be0064044400a7
:100d50006011b8008000eb0008007800c2020200b9
:100d600000000000582002000000000080bf9f002b
:100d700091bf9f00c10220000e00780044060200cf
:100d8000000000000007e8000a00be00581e020034
:100d9000000000000004be000205be000fb897006e
:100da0009fb89700581e0200000000006022b800a3
:100db00006002000e7042400aa1e02000000000034
:100dc0000002be000203be000800be000a01be0011
:100dd0005e1f02000000000058200200000000001a
:100de0000001be00a0069800b106980070c5b300cf
:100df0009e4f10003f003200c10220000e0078001c
:100e000044060200000000000007e8006011b8007e
:100e10008000eb000e007800c2020200000000001b
:100e20005820020000000000e0069800f10698003b
:100e3000c10220000e0078004406020000000000fd
:100e40000007e8006011b8008000eb000e00780099
:100e5000c202020000000000582002000000000052
:100e6000800e9800910e9800c10220000e007800bc
:100e700044060200000000000007e8001e80fb009e
:100e80006a00b9001e4190000041410070415100cc
:100e9000f25698002e4090000080fb006a00b900d6
:100ea0003e4190000041410070415100e2569800df
:100eb0004e4190000281fb006a11b9005e40900033
:100ec0000080fb0002004000015c200001004000a7
:100ed000a00e98000000200001082000c006980025
:100ee000d106980030c0b300c05e98008000eb00cf
:100ef0000eff37000200be00581e02000000000076
:100f000003f0a2005820020000000000a006980094
:100f1000b1069800b8ff37000200be00581e02005c
:100f20000000000003f0a2005820020000000000b2
:100f3000808ebe006fff370000c0eb0032ff37002d
:100f400010c0b30030ff37001e409000824f5000a9
:100f5000eafe3a00ae40900010c4b30080cf5000cb
:100f6000e6fe3a008a00e9000800e8001c010700dc
:100f70008080eb000000e000ecfe3500c1022000a4
:100f80000e00780044060200000000000007e800a0
:100f90001e80fb006a00b9001e4190000041410024
:100fa00070415100825e98002e4090000080fb004e
:100fb0006a00b9003e41900000414100704151007b
:100fc000925e98004e4090000080fb006a00b900dd
:100fd0005e4190000041410070415100a25e9800c6
:100fe000c10220000e00780044060200000000004c
:100ff000000478000007e8001e81fb006a11b900b8
:101000001e4090000080fb00020040000021b10063
:10101000cf80de006a210200000000000005be0053
:10102000630444006011b8008000eb000800780001
:10103000c202020000000000582002000000000070
:10104000a0b79f00b1b79f00c10220000e0078003a
:1010500044060200000000000007e8000a00be008d
:10106000581e0200000000000004be000205be0081
:101070002fb09700bfb09700581e0200000000007c
:101080006022b80006002000e7042400aa1e020027
:10109000000000000002be000203be000800be0007
:1010a0000a01be005e1f020000000000582002007e
:1010b000000000000001be00808ebe0030c5b300fd
:1010c0009e4f10008d003200c10220000e007800fb
:1010d0004406020000000000000478000007e80059
:1010e0001e81fb00400620000091b9001e409000c8
:1010f0000080fb006a00b900000141002e40900012
:101100000080fb000001410000b32e0000014100ff
:101110006110b9006a210200000000000005be0055
:10112000640444006011b8008000eb0008007800ff
:10113000c20202000000000058200200000000006f
:10114000c0b79f00d1b79f00c10220000e007800f9
:1011500044060200000000000007e8000a00be008c
:10116000581e0200000000000004be000205be0080
:101170004fb09700dfb09700581e0200000000003b
:101180006022b80006002000e7042400aa1e020026
:10119000000000000002be000203be000800be0006
:1011a0000a01be005e1f020000000000582002007d
:1011b000000000000001be00a0069800b1069800e3
:1011c00070c5b3009e4f100043003200c1022000e2
:1011d0000e00780044060200000000000007e8004e
:1011e0001e40780001c3b300814f50003800320028
:1011f00001405000b05e9800c10220000e0078004f
:1012000044060200000000000007e800c1022000c0
:101210000e00780044060200000000000007e8000d
:10122000c10220000e007800440602000000000009
:101230000007e8006011b8008000eb000e007800a5
:10124000c20202000000000058200200000000005e
:10125000c0069800d1069800c10220000e00780058
:10126000440602000000000090409000d0c4b3008b
:1012700080cf50000d0032000040eb00f056980087
:10128000e05698000000eb00a00e9800000020003f
:1012900001082000e0069800f1069800800e9800f2
:1012a000910e980010c0b3000fff37004d00900062
:1012b000dd00900052b82e0013052400ae2202007b
:1012c00000000000c0069800d1069800eaff370031
:1012d00000c0eb00c7ff37000200be00581e02002e
:1012e0000000000003f0a2005820020000000000ef
:1012f000a0069800b1069800b4ff37000200be00b7
:10130000581e02000000000003f0a2005820020056
:1013100000000000808ebe006bff370020882d008b
:10132000801f7800e0042000fc7c02000000000028
:101330000003eb00e5042000050278008501780039
:10134000f28a2d0021032000b08b2d00967c020034
:10135000000000008f87e900e3fd37008a1f780056
:10136000218c2d00811f7800f0042000fc7c0200fd
:10137000000000000a03780065052000f404200046
:10138000e3042000f28a2d00e1022000b08b2d0042
:10139000967c020000000000e4875700d0fd370073
:1013a000d08e2d00801f7800d0042000fc7c02002d
:1013b000000000000003eb00e5042000d40420003e
:1013c00085017800f28a2d00a1022000b08b2d004b
:1013d000967c0200000000008f87e900befd370008
:1013e000889fbe000004be000000e00046003200fe
:1013f000e58f540033003400090044008000e90008
:10140000888f50002d00390011417800a0c2b30030
:10141000804f5100060032008100e900888f5000a3
:101420002600390011417800804f5100faff3a0040
:101430008081eb00a0c2b300804f510018003a0039
:101440000041eb0008007800810f540003003100d8
:1014500030416900810f5000fdff39000280fb0020
:10146000c401de00e9cf510012003e000343b0008a
:101470006f416100e94f51000c003e000243b00093
:101480001140900080cf510004003a0021409000ac
:1014900088815000804f510001003200e3ff2f008f
:1014a000030078004f04be00000006007243b00045
:1014b000f3ff37007343b000edff370011417800b0
:1014c000dbff3700891f7800a0912d00801f780076
:1014d000d0322000fc7c0200000000000003eb0082
:1014e000e50420003402200073042000f2942d0053
:1014f00041122000b08b2d00967c020000000000fd
:10150000e4875700bcff370040962d00801f78000d
:1015100030022000fc7c0200000000000003eb0011
:10152000e50420003402200073042000f2942d0012
:10153000f1112000b08b2d00967c0200000000000d
:101540008f87e900aaff37008c02fa00889fbe004f
:101550008a9fbe008c9fbe000006780080d62f00b8
:101560000f004000bb0009000018eb0080d62f00e0
:101570000f004000a60007000000e0009d003a00b8
:101580001c00be00f09f9e0081a79e002c009000d2
:10159000bc00900090a79e00a1a79e00a1d72f009d
:1015a000818647002c009000bc009000581e02006d
:1015b000000000006022b8006033b800a01e0200e6
:1015c000000000000000e00088003500500420000a
:1015d000801f78002c059000bc0590000a00be001a
:1015e00082250200000000000004be00cf80de0063
:1015f0006a210200000000000001be000a00be00d7
:10160000ae2002000000000001f0a1000200200056
:1016100003272400ae22020000000000581e020032
:1016200000000000809fbe00829fbe00080078007e
:101630000800e0006b003500801f78001c00be0031
:10164000581e0200000000006022b8006033b8009d
:10165000a01e0200000000000000e0005f00350056
:10166000e0042000801f78001c05be000a00be00b8
:1016700082250200000000000004be00cf80de00d2
:101680006a210200000000000001be000a00be0046
:10169000ae2002000000000001f0a10002002000c6
:1016a00003272400ae22020000000000581e0200a2
:1016b00000000000809fbe00829fbe0008007800ee
:1016c0000800e00043003500801f78001c5890009f
:1016d0000080fb00801f78000c5890000080fb0009
:1016e000801f78007c5090000080fb00801f7800f5
:1016f000c09a2d00801f78000d007800600602005f
:10170000000000000f02b100612a21000d007800e6
:10171000c6060200000000000d0078008e040200e2
:1017200000000000c03f9d0000ee2f000085470034
:10173000421120008a00780080d62f000f00400060
:10174000c05e020000000000000478000000e0001d
:101750001b003500000178008a007800200020007e
:101760007262020000000000880f50000d0032007d
:10177000801f7800509d2d00801f780000072000fa
:10178000fc7c02000000000010002000e4875700ed
:101790004f06be004f05be004f04be000080fa0099
:1017a00000000600419f2d0080d62f000f00400052
:1017b00062650200000000000000eb00f4ff37004b
:1017c000801f7800e19f2d00811f7800f006200027
:1017d000ebff37000800ea00bbff370030052000b0
:1017e000a0ff37000800ea0093ff370070052000d3
:1017f00077ff3700f202200041a32d0010002000e7
:1018000080430200000000000080eb00e0ff370092
:10181000889fbe008a9fbe008c9fbe008006780015
:101820000000e0006b0032004653e200120032007c
:101830000d0078004135210007000900315878007b
:1018400068804600c1342100070009003158780043
:10185000401120000d004000c1352100400009006a
:10186000315878000000eb004f06be004f05be0067
:101870004f04be000000060041a62d0000242100f8
:10188000863b0200000000000000e0004d00320036
:10189000222d2100124178000204e00041003200b4
:1018a0000006eb00220032006865b80063262100c4
:1018b000030445008084eb008000eb00d2c2b3003b
:1018c00068c07800824f5000340032008100e80088
:1018d000e68f5000faff3400e18f44002900320007
:1018e000c135210001004500090178008800780019
:1018f000180502000000000009004400104090009c
:101900000080fb0002fd2f008200400033362100e2
:10191000030045000148d0000c06e800222d2100fc
:10192000124178000280fb00800f5600deff350078
:101930000280fb006800b800b335210003004000be
:101940001004a000020078009cf3b7008200200081
:101950000124210040352100440402000000000061
:101960004852d4005bf3b700419a2d00c0342100e7
:10197000260502000000000010c0b30046f3b700c7
:10198000abff3700c035210080004500080078001b
:1019900005000900b0587800dfff370081047800a7
:1019a000cdff3700b2a62d00821f7800a0062000d0
:1019b000fc7c0200000000000080eb008f87e90043
:1019c000a9ff370011a92d00811f7800d006200043
:1019d000f7ff3700d0ab2d00801f7800a006200055
:1019e000fc7c0200000000000003eb00e504200086
:1019f000a40620004305200032ae2d00710820000f
:101a000040af2d00967c0200000000008f87e900a7
:101a100085ff3700e28057001101be000370a1006e
:101a20008040a9000000eb00020180000278e10084
:101a30000d003500100020000b003700e280570039
:101a40001101be000370a1008080a90020002000c9
:101a500005003700e28057001101be000370a100ad
:101a60008060a900300020006ff7800028d5280092
:101a7000881f7800090020001a0280004855dd0008
:101a80008a8474002a028000630565004455dd00e5
:101a90008a847400891f7800004006000000fe0060
:101aa0000000fe00889fbe00e20f500031003200af
:101ab000e10f50001b003600e30f50001000320011
:101ac0006044b800120e200003002000f0aa80003d
:101ad00001ab80006e24020000000000800f540063
:101ae000818f5c000300310061044400e0844c00fd
:101af000faff37000000fe004f04be0000000600a1
:101b0000831f7800821f7800811f7800e0af2d00ce
:101b1000801f7800b67d020000000000e8875700b3
:101b2000e7ff3700831f7800821f7800811f78004d
:101b3000c1b22d00e10f50000100320051b32d0061
:101b4000811f7800f0b32d00801f7800b67d020061
:101b500000000000f827f800ec1ef800f0b62d0099
:101b6000801f7800b67d020000000000f08757005b
:101b7000d3ff3700831f7800821f7800811f780011
:081b8000f0b92d00e2ff37006f
:020000040000fa
:020000040001f9
:101b8800646d0000637400006f6400006567000006
:101b98003a20000045720000726f0000723a00009f
:101ba800206100007267000020700000747200005d
:101bb800206900006e70000020690000732000009a
:101bc8006e7500006c6c0000206f00007220000031
:101bd800656d000070740000793a0000202500004f
:101be800700a0000006400006d630000746f00005c
:101bf800646500006700000075740000696c0000ef
:101c0800732e000063000000646d00006374000020
:101c18006f640000656700003a200000496e00000c
:101c280074650000726e0000616c000020450000c1
:101c3800727200006f7200003a20000073650000a5
:101c48006320000025660000206900007320000062
:101c58006f750000742000006f660000207200009d
:101c6800616e000067650000205b00002d350000f4
:101c7800392e0000393900002e2e000035390000b9
:101c88002e390000395d00000a000000646d000074
:101c9800637400006f640000656700003a2000006c
:101ca800496e000074650000726e0000616c0000ef
:101cb80020450000727200006f7200003a20000098
:101cc8006d6900006e200000256600002069000094
:101cd800732000006f750000742000006f6600001c
:101ce80020720000616e000067650000205b000044
:101cf8002d350000392e0000393900002e2e000045
:101d0800353900002e390000395d00000a00000056
:101d1800646d0000637400006f6400006567000074
:101d28003a20000064650000672000002566000076
:101d380020690000732000006f7500007420000007
:101d48006f66000020720000616e00006765000089
:101d5800205b00002d330000363000002e2e0000de
:101d680033360000305d00000a000000646d00009a
:101d7800637400006f640000656700003a2000008b
:101d8800496e000074650000726e0000616c00000e
:101d980020450000727200006f7200003a200000b7
:101da800706f0000696e000074650000722000000a
:101db8006d690000736d00006174000063680000c5
:101dc8002c200000737400007020000025700000b3
:101dd800202100003d200000702000002570000038
